:100000000C948A180C94B5180C94B5180C94B51867
:100010000C94B5180C94B5180C94B5180C94B5182C
:100020000C94B5180C94B5180C94B5180C94B5181C
:100030000C94B5180C9437190C94B5180C94B51889
:100040000C94B5180C947A7B0C94B5180C94B518D4
:100050000C94B5180C94B5180C9434840C9496191F
:100060000C94B5180C944D510C94B5180C94B5180B
:100070000C94B5180C94B5180C94B5180C94B518CC
:100080000C94B5180C94B5180C94B5180C94B518BC
:100090000C94B5180C94B5180C94B5180C94639680
:1000A0000C94B5180C94B5180C94B5180C94B5189C
:1000B0000C94B5180C94B5180C94B5180C94B5188C
:1000C0000C94B5180C94B5180C94B5180C94B5187C
:1000D0000C94B5180C94B5180C94B5180C94B5186C
:1000E0000C94B518084AD73B3BCE016E84BCBFFDCB
:1000F000C12F3D6C74319ABD56833DDA3D00C77FF8
:1001000011BED9E4BB4C3E916BAAAABE0000008090
:100110003F05A84CCDB2D44EB93836A9020C50B91F
:10012000918688083CA6AAAA2ABE000000803F0249
:1001300000002100240027002A002D003000330099
:1001400001010000040107010A010000220025004E
:1001500028002B002E0031003400020100000501B0
:1001600008010B01000020002300260029002C00BC
:100170002F003200000100000301060109010505FE
:100180000505070508080808020202020A0A08080D
:10019000040404040101010101010101030303033B
:1001A00003030303040707070C0C0C0C0C0C0C0CCA
:1001B0000202020206060606060606060B0B0B0BDB
:1001C0000B0B0B0B01021020200808102040102000
:1001D000408002010201080402010102040810200B
:1001E0004080804020100804020180040201804009
:1001F0002010080402010804020101020408102072
:10020000408001020408102040800000090A020812
:100210000B0C0D07060304010000000000000000A5
:1002200000000000000000000000000000000000CE
:1002300000000000000011100F000000000000008E
:1002400000000000000000000000000000000000AE
:100250004D383420582059205A2045006563686F76
:100260003A0043616E6E6F7420656E746572207320
:1002700075626469723A20004D3234004D32332089
:100280002573006175746F25692E67004572726F62
:10029000723A006572726F722077726974696E6764
:1002A00020746F2066696C6500436172642065721A
:1002B000726F723A004E6F74205344207072696EF0
:1002C00074696E67002F005344207072696E746900
:1002D0006E67206279746520002E0044656C657439
:1002E000696F6E206661696C65642C2046696C6577
:1002F0003A200046696C652064656C657465643AF3
:10030000002E006F70656E206661696C65642C203C
:1003100046696C653A200057726974696E6720748B
:100320006F2066696C653A20002E006F70656E2044
:100330006661696C65642C2046696C653A20002E04
:10034000006F70656E206661696C65642C2046697B
:100350006C653A200046696C652073656C65637452
:100360006564002053697A653A200046696C65200F
:100370006F70656E65643A20002E006F70656E20A8
:100380006661696C65642C2046696C653A2000538F
:10039000442063617264206F6B006F70656E526FF2
:1003A0006F74206661696C656400766F6C756D654D
:1003B0002E696E6974206661696C6564005344201F
:1003C000696E6974206661696C006563686F3A00E4
:1003D00048617264636F6465642044656661756C2E
:1003E000742053657474696E6773204C6F61646523
:1003F000640053746F7265642073657474696E670A
:10040000732072657472696576656400204400200B
:1004100049002020204D33303120500050494420E5
:1004200073657474696E67733A00205A002059002E
:1004300020204D323036205800486F6D65206F66A1
:100440006673657420286D6D293A00204500205A96
:100450000020580020420020540020204D3230352A
:10046000205300416476616E636564207661726931
:1004700061626C65733A20533D4D696E2066656517
:10048000647261746520286D6D2F73292C20543D92
:100490004D696E2074726176656C20666565647264
:1004A00061746520286D6D2F73292C20423D6D6984
:1004B0006E696D756D207365676D656E7420746906
:1004C0006D6520286D73292C20583D6D6178696D0C
:1004D000756D205859206A65726B20286D6D2F73D9
:1004E000292C20205A3D6D6178696D756D205A2048
:1004F0006A65726B20286D6D2F73292C2020453D75
:100500006D6178696D756D2045206A65726B202874
:100510006D6D2F73290020540020204D323034207F
:100520005300416363656C65726174696F6E3A2054
:10053000533D616363656C65726174696F6E2C20F5
:10054000543D7265747261637420616363656C65A8
:10055000726174696F6E00204500205A00205900B6
:1005600020204D3230312058004D6178696D756D15
:1005700020416363656C65726174696F6E20286DDC
:100580006D2F7332293A00204500205A002059006F
:1005900020204D3230332058004D6178696D756DE3
:1005A0002066656564726174657320286D6D2F73B4
:1005B000293A00204500205A0020590020204D39BA
:1005C0003220580053746570732070657220756E08
:1005D00069743A0053657474696E67732053746F5D
:1005E000726564006563686F3A004572726F723AB3
:1005F000005072696E7465722073746F70706564F8
:100600002064756520746F206572726F72732E207E
:1006100046697820746865206572726F7220616E19
:100620006420757365204D39393920746F207265E7
:1006300073746172742E202854656D7065726174D4
:100640007572652069732072657365742E20536519
:1006500074206974206166746572207265737461B8
:100660007274696E6729005072696E7465722068D1
:10067000616C7465642E206B696C6C282920636141
:100680006C6C656421006F6B00526573656E643A33
:1006900020002200556E6B6E6F776E20636F6D6D5C
:1006A000616E643A2022002200556E6B6E6F776E89
:1006B00020636F6D6D616E643A2022007A5F6D6118
:1006C000783A2000795F6D61783A2000785F6D6933
:1006D0006E3A20005A3A00593A0020436F756E7402
:1006E00020583A2000453A005A3A00593A00583A00
:1006F000004649524D574152455F4E414D453A4D96
:1007000061726C696E2056313B20537072696E7451
:1007100065722F6772626C206D61736875702066F8
:100720006F722067656E36204649524D57415245DB
:100730005F55524C3A687474703A2F2F6669726D27
:10074000776172652E756C74696D616B65722E636D
:100750006F6D2050524F544F434F4C5F564552538C
:10076000494F4E3A312E30204D414348494E455F66
:10077000545950453A556C74696D616B65722045EA
:10078000585452554445525F434F554E543A310ADE
:100790000020423A0020453A00543A0020573A00DF
:1007A00020453A00543A002042403A0020403A00A6
:1007B000202F0020423A00202F006F6B20543A0077
:1007C0002569206D696E2C202569207365630045BD
:1007D0006E642066696C65206C697374004265679D
:1007E000696E2066696C65206C6973740000000096
:1007F00000000061430000664300000000000000AC
:100800000000000000000066430000614300006635
:10081000430000664300006143000066430000A0FF
:10082000400000A04000004040FF01012569206811
:100830006F757273202569206D696E75746573001C
:10084000446F6E65207072696E74696E67206669A8
:100850006C65005072696E7465722073746F70708D
:1008600065642064756520746F206572726F7273A1
:100870002E2046697820746865206572726F722038
:10088000616E6420757365204D39393920746F208D
:10089000726573746172742E202854656D70657270
:1008A00061747572652069732072657365742E209A
:1008B0005365742069742061667465722072657373
:1008C00074617274696E6729006F6B004E6F204C03
:1008D000696E65204E756D62657220776974682057
:1008E000636865636B73756D2C204C617374204C69
:1008F000696E653A20004E6F20436865636B7375BF
:100900006D2077697468206C696E65206E756D6204
:1009100065722C204C617374204C696E653A20001E
:10092000636865636B73756D206D69736D61746366
:10093000682C204C617374204C696E653A20004C21
:10094000696E65204E756D626572206973206E6FE9
:1009500074204C617374204C696E65204E756D6215
:1009600065722B312C204C617374204C696E653A92
:1009700020004D31313000446F6E6520736176691F
:100980006E672066696C652E006F6B004D32390012
:100990002020506C616E6E657242756666657242AB
:1009A000797465733A20002046726565204D656D47
:1009B0006F72793A20004F63742031352032303124
:1009C0003300436F6D70696C65643A200056657240
:1009D00073696F6E2031332E313000207C204175D9
:1009E00074686F723A20004F6374203135203230C2
:1009F00031332031343A33333A353700204C617388
:100A00007420557064617465643A2000312E302E74
:100A100030004D61726C696E200020536F667477F0
:100A20006172652052657365740020576174636854
:100A3000646F67205265736574002042726F776E31
:100A4000206F757420526573657400204578746555
:100A5000726E616C20526573657400506F776572B9
:100A60005570007374617274002200656E71756553
:100A7000696E672022002200656E717565696E6778
:100A80002022006563686F3A0020746F6F206C6FDE
:100A90006E6720657874727573696F6E2070726509
:100AA00076656E7465640020636F6C64206578748D
:100AB000727573696F6E2070726576656E746564A9
:100AC0000000002110422063308440A550C660E73A
:100AD00070088129914AA16BB18CC1ADD1CEE1EFF3
:100AE000F13112100273325222B5529442F772D68B
:100AF00062399318837BB35AA3BDD39CC3FFF3DE43
:100B0000E36224433420040114E664C774A44485DA
:100B1000546AA54BB528850995EEE5CFF5ACC58D92
:100B2000D55336722611163006D776F6669556B42A
:100B3000465BB77AA719973887DFF7FEE79DD7BCE2
:100B4000C7C448E5588668A778400861180228237A
:100B500038CCC9EDD98EE9AFF9488969990AA92B32
:100B6000B9F55AD44AB77A966A711A500A333A12CA
:100B70002AFDDBDCCBBFFB9EEB799B588B3BBB1A82
:100B8000ABA66C877CE44CC55C222C033C600C411A
:100B90001CAEED8FFDECCDCDDD2AAD0BBD688D49D2
:100BA0009D977EB66ED55EF44E133E322E511E706A
:100BB0000E9FFFBEEFDDDFFCCF1BBF3AAF599F7822
:100BC0008F8891A981CAB1EBA10CD12DC14EF16FD3
:100BD000E18010A100C230E3200450254046706738
:100BE00060B9839893FBA3DAB33DC31CD37FE35E64
:100BF000F3B1029012F322D2323542145277625688
:100C000072EAB5CBA5A89589856EF54FE52CD50D73
:100C1000C5E234C324A014810466744764245405D7
:100C200044DBA7FAB79987B8975FE77EF71DC73C03
:100C3000D7D326F2369106B0165766767615463427
:100C4000564CD96DC90EF92FE9C899E9898AB9AB13
:100C5000A94458654806782768C018E1088238A377
:100C6000287DCB5CDB3FEB1EFBF98BD89BBBAB9AA3
:100C7000BB754A545A376A167AF10AD01AB32A92C7
:100C80003A2EFD0FED6CDD4DCDAABD8BADE89DC9B3
:100C90008D267C076C645C454CA23C832CE01CC117
:100CA0000C1FEF3EFF5DCF7CDF9BAFBABFD98FF843
:100CB0009F176E367E554E745E932EB23ED10EF067
:100CC0001E7C3C3E5E2B3D3F2F5B5D3B2C2A225C15
:100CD0000045313A200045303A20005A3A20005968
:100CE0003A2000583A20004D53312C4D53322050B9
:100CF000696E730A0024F404D9201BC40C5C0E989E
:100D000004C4095F0265077101F405F900FB04B32F
:100D10000048048700C103690058035500030345D8
:100D200000BE023A008402310053022A0029022543
:100D30000004022000E4011C00C8011900AF0117E3
:100D4000009801140084011300710110006101106A
:100D50000051010E0043010D0036010B002B010B69
:100D60000020010B00150109000C01090003010816
:100D700000FB000800F3000800EB000700E4000699
:100D800000DE000600D8000600D2000600CC0005F8
:100D900000C7000500C2000500BD000400B9000442
:100DA00000B5000400B1000400AD000400A9000477
:100DB00000A5000300A20003009F0004009B0003A5
:100DC00000980003009500020093000300900003C8
:100DD000008D0002008B00030088000200860002E4
:100DE0000084000300810002007F0002007D0002F9
:100DF000007B00020079000200770001007600020B
:100E0000007400020072000100710002006F000215
:100E1000006D0001006C0002006A00010069000220
:100E20000067000100660001006500010064000227
:100E3000006200010061000100600001005F00022B
:100E4000005D0001005C0001005B0001005A000130
:100E50000059000100580001005700010056000130
:100E60000055000100540001005300000053000130
:100E7000005200010051000100500001004F00012C
:100E8000004E0000004E0001004D0001004C00012A
:100E9000004B0000004B0001004A00010049000126
:100EA0000048000000480001004700010046000023
:100EB000004600010045000000450001004400011B
:100EC0000043000000430001004200000042000116
:100ED000004100000041000100400001003F00000F
:100EE000003F0001003E0000003E0001003D000008
:100EF000003D0001003C0000003C0000003C0001FF
:100F0000003B0000003B0001003A0000003A0001F5
:100F100000390000003900010038000000380000EE
:100F200000380001003700000037000100360000E3
:100F300000360000003600010035000000350000DA
:100F400000350001003400000034000000340001CE
:100F500000330000003300000033000100320000C5
:100F600000320000003200010031000000310000BA
:100F700000310001003000000030000000300001AE
:100F8000002F0000002F0000002F0000002F0001A4
:100F9000002E0000002E0000002E0001002D000099
:100FA000002D0000002D0000002D0001002C00008D
:100FB000002C0000002C0000002C0001002B000081
:100FC000002B0000002B0000002B0001002A000075
:100FD000002A0000002A0000002A00010029000069
:100FE000002900000029000000290000002900015C
:100FF0000028000000280000002800000028000051
:101000000028000100270000002700000027000042
:101010000027000000270001002600000026000035
:101020000026000000260000002600010025000028
:10103000002500000025000000250000002500001C
:10104000002500010024000000240000002400000E
:101050000024000000240001002300000023000001
:1010600000230000002300000023000000230000F4
:1010700000230001002200000022000000220000E6
:1010800000220000002200000022000100210000D8
:1010900000210000002100000021000000210000CC
:1010A00000210000002100010020000000200000BD
:1010B00000200000002000000020000000200000B0
:1010C0000020000000200001001F0000001F0000A1
:1010D000001F0000001F0000001F0000001F000094
:1010E000001F0001001E0000001E0000001E000086
:1010F000001E00000024F4D43050C38E20C2A24051
:1011000017828B7011127A910D816CD90AA861E156
:1011100008C7586607615143061E4B5D05C145A7C8
:10112000041A411104093D9803713931034036DB3B
:101130000265339102D4305402802E1D02632CEEDE
:1011400001752AC501B028A001102781018F2564EF
:10115000012B244B01E0223401AC211F018D200D15
:1011600001801FFC00841EED00971DDF00B81CD21B
:1011700000E61BC600201BBC00641AB200B219A80E
:10118000000A19A0006A189900D117910040178B26
:1011900000B516840031167E00B31579003A157338
:1011A00000C7146F0058146A00EE136600881363BA
:1011B0000025135E00C7125B006C12570015125415
:1011C00000C111510070114F0021114B00D6104980
:1011D000008D1047004610440002104200C00F402E
:1011E00000800F3E00420F3C00060F3B00CB0E3844
:1011F00000930E37005C0E3500270E3400F30D32DD
:1012000000C10D3100900D3000600D2E00320D2D0B
:1012100000050D2C00D90C2B00AE0C2900850C29E3
:10122000005C0C2700350C27000E0C2600E80B2470
:1012300000C40B2400A00B23007D0B23005A0B21BC
:1012400000390B2100180B2000F80A1F00D90A1ED4
:1012500000BB0A1E009D0A1D00800A1D00630A1CB7
:1012600000470A1B002C0A1B00110A1A00F7091A72
:1012700000DD091900C4091900AB0919009209170A
:10128000007B091800630917004C0916003609167F
:1012900000200916000A091500F5081500E00814D9
:1012A00000CC081400B8081400A408140090081317
:1012B000007D0812006B081300580812004608123F
:1012C0000034081100230811001208110001081150
:1012D00000F0071000E0071000D0071000C0071052
:1012E00000B0070F00A107100091070E0083070F41
:1012F0000074070F0065070E0057070E0049070E20
:10130000003B070D002E070E0020070D0013070DF0
:101310000006070D00F9060C00ED060D00E0060CB6
:1013200000D4060C00C8060C00BC060C00B0060C6D
:1013300000A4060B0099060C008D060B0082060B1C
:101340000077060B006C060B0061060A0057060BBF
:10135000004C060A0042060A0038060A002E060A59
:101360000024060A001A060A001006090007060AE9
:1013700000FD050900F4050900EB050900E2050977
:1013800000D9050900D0050900C7050900BE0509F7
:1013900000B5050800AD050800A50509009C050875
:1013A00000940508008C050800840508007C0508E9
:1013B00000740508006C050700650508005D050759
:1013C00000560508004E05070047050700400508C0
:1013D0000038050700310507002A05070023050727
:1013E000001C050600160507000F05070008050686
:1013F0000002050700FB040600F5040700EE0406E2
:1014000000E8040600E2040700DB040600D5040639
:1014100000CF040600C9040600C3040600BD04068C
:1014200000B7040600B1040500AC040600A60406DB
:1014300000A00405009B0406009504050090040626
:10144000008A04050085040500800406007A04056E
:101450000075040500700405006B040500660405B2
:1014600000610405005C04050057040500520405F2
:10147000004D04050048040500430405003E040433
:10148000003A04050035040500300404002C04056E
:101490000027040400230405001E0404001A0404A9
:1014A0000016040500110404000D040400090405DD
:1014B000000404040000040400FC030400F8030416
:1014C00000F4030400F0030400EC030400E8030448
:1014D00000E4030400E0030400DC030400D8030478
:1014E00000D4030400D0030400CC030400C80303A9
:1014F00000C50303006563686F3A00205A3A002074
:10150000593A0020583A00656E6473746F70732006
:101510006869743A20004572726F723A0054656DC2
:1015200070657261747572652068656174656420A8
:10153000626564207377697463686564206F6666AA
:101540002E204D415854454D50207472696767658F
:10155000726564202121003A2045787472756465B3
:1015600072207377697463686564206F66662E20E5
:101570004D494E54454D50207472696767657265D8
:10158000642021003A204578747275646572207376
:1015900077697463686564206F66662E204D4158D4
:1015A00054454D50207472696767657265642021E7
:1015B00000202D20496E76616C6964206578747214
:1015C00075646572206E756D626572202100000081
:1015D0000000300E0100C00E0A00500F1400D00FA2
:1015E0001E0060102800E010320070113C00F01165
:1015F00046007012500000135A008013640000145B
:101600006E00901478001015820090158C00101652
:1016100096009016A0001017AA009017B40010189A
:10162000BE009018C8001019D2009019DC00101AE2
:10163000E600801AF000001BFA00801B0401F01B7A
:101640000E01701C1801F01C2201601D2C01E01D10
:101650003601501E4001D01E4A01401F5401B01FE8
:101660005E0130206801A020720110217C019021D0
:101670008601002290016026F401902A5802802EF3
:10168000BC0250322003E03584035039E803803C2B
:101690004C04504944204175746F74756E65206622
:1016A000696E69736865642120507574207468657B
:1016B000204B702C204B6920616E64204B642063AA
:1016C0006F6E7374616E747320696E746F20436FF4
:1016D0006E66696775726174696F6E2E6800504935
:1016E00044204175746F74756E65206661696C6520
:1016F00064212074696D656F75740020403A006F35
:101700006B20543A006F6B20423A0050494420410C
:1017100075746F74756E65206661696C65642120EF
:1017200054656D706572617475726520746F6F2099
:101730006869676800204B643A2000204B693A20B2
:1017400000204B703A200020436C61736963205085
:10175000494420002054753A2000204B753A20005F
:10176000206D61783A2000206D696E3A2000206477
:101770003A200020626961733A20004D41494E547D
:10178000454E414E4345004D4154455249414C0060
:101790005052494E5400737570706F727440756C7E
:1017A00074696D616B65722E636F6D00436F6E744B
:1017B0006163743A0053616665747920636972638A
:1017C0007569740054656D702073656E736F722057
:1017D0004245440054656D702073656E736F7200EE
:1017E0004552524F52202D2053544F5050454400E3
:1017F000801506060606FEFEFEFEFC000000000048
:101800000000FCFEFEFEFC0000000EFEFEFEFE00E0
:1018100000E0FCFEFEFCE0E0000000CECECE0000CA
:1018200000C0C0C0C0C0C08000000000000080C078
:10183000C0800000000000008080C0C0C0C0C0C0E8
:10184000C080800000000006FEFEFEFE00000000DA
:1018500080C0C0C00000000000008080C0C0C08008
:10186000808000000000C0C0C0C00080C0C0C0C0F8
:101870008000000000007FFFFFFFFF8000000000ED
:101880000080FFFFFFFFFF00000000FFFFFFFF00E1
:101890000000FFFFFFFF0000000000FFFFFF00004F
:1018A0000081F1FFFF3F0F3FFFFCF0F0FCFF3F0F17
:1018B0003FFFFEF880000000C1E1F1F1713101014C
:1018C00083FFFFFFFC000000FFFFFFFF000C3EFF57
:1018D000FFF7C301000000FCFEFF87031131313325
:1018E0003F3F3F1E000001FFFFFFFF070301010113
:1018F00001000000000000010307070F0F0F0F0F8A
:101900000F0F0707070F0F06000000070F0F070054
:101910000000070F0F0700000000000F0F0F00006E
:10192000060F0F070100000001070F0F070100005D
:101930000001070F0F06000003070F0F0E0E06072A
:1019400003070F0F07000000070F0F07000000003C
:10195000030F0F0F060000000307070F0E0E0E0EF9
:101960000E0E06000000000F0F0F0F000000000019
:1019700000008015090909F90101010103FE0000B9
:10198000000000FE0301010103FE001FF10101013F
:1019900001FFF01E030101031E10F000FF31313181
:1019A000FF00E020202020202060C080000080C0B8
:1019B00060202060C000000000C040602020202087
:1019C0002020206040C080000FF901010101FF00CC
:1019D00080C060202020E000000080C04060202007
:1019E00020604040C08000E020202020E0602020D7
:1019F000202060C0000000FF80000000007FC08049
:101A00008080C07F0000000000FF0000FF00000099
:101A100000FF01FF00000000FF010100FF000000C7
:101A2000FF00C37A0E0000C070C000030E0E03005A
:101A3000C070C00001077CC000E3321A0A0A8ACADB
:101A4000FAC67C00000003FE00FF00000000FF73E8
:101A5000C10000083CE68300FE03010078FCEE4A6A
:101A60004E4C404040613F03FE00000000F80C0671
:101A7000020202030000000003060C0818101010F8
:101A8000101010101808181010190F000F1810104F
:101A9000180F000F181010180F0000001F10101062
:101AA0001F0F191010180E0300030E181010180E37
:101AB0000300030E181010190F070C181010111145
:101AC00019080C181010180F000F181010180F001C
:101AD00001071C101010190F01070C081810111124
:101AE00011111111190F00001F101010101F00000C
:101AF000000000002F400000000000000000000077
:101B00000000808080C0E0FEFF191E989898181889
:101B1000181818189E9F991E38F0E0000000000069
:101B200000000000000000000000000000003CFE7B
:101B3000FFFF99F1E1C3FFFF000063636360606032
:101B40006060606363630000FFFF7C38000000009A
:101B50000000000000000080C060B0D8D81CFCFF6E
:101B60003F0F8FCFC7C7C7C6C6C6C6C6C6C6C6C67E
:101B7000C6C6C6C6C6C6C6C7C7C4CC0C1CF8F87055
:101B8000C00000000EFFF92A2B2B2828FCFFFF00C5
:101B900000FFFFFFFFFFFFFFBFB717B5BDB500B5E3
:101BA000B5F717FFBFBFFFFFFFFF0000FFFFFCFF00
:101BB0000700C0F0FFFFFDDD1D19193FFFFF00000A
:101BC000FFFFFFFFFFFFFFFBF1FBFBEAEEC0EEEACA
:101BD000FAF0FAFAFFFFFFFFFF0000FFFF0F1FF808
:101BE000E00003070F0F1B1819FBFEFFFFF0E0C01A
:101BF000C1E1F1F1F1F1F1F1F1F1F1F1F1F9F9F9FD
:101C0000F9F9F9797979F1F010181F070603030043
:101C100000000000000000F8FFEFDFBF7FFFFFFFC4
:101C2000404143437F212020217FFFFFFF3FB091B0
:101C3000D1DFD050581F1FF0F0000000000000005E
:101C4000000000000003070F1E3D7B77EED1DEDEB3
:101C5000CF4B4B6969686868603F3F373737353429
:101C600030101018181A1B0F060000000000100F8B
:101C7000FC0E0FCFCFCFCECCCCCCCCCCCCDCC0C0EC
:101C800007707E7F7F7F7F7F7F7F7F7F7F7F0F01DA
:101C90007120FFFFFFFFFFFFFFFFFFFFFCE00000E1
:101CA0000000000000000000E0FCFFFFFFFFFFFF5E
:101CB000FFFFFFFF00000000000000000000000028
:101CC0000000000000000000000000000000FFFF16
:101CD000FFFFFFFFFF000000000000000000000009
:101CE00000000000000000000000000000000000F4
:101CF00000000000000000000000000000000000E4
:101D0000000000FFFFFFFFFFFFFF7FFFFFFFFFFF60
:101D1000F8800000000080F0FFFFFFFFFF3FFFFFA3
:101D2000FFFFFFFFFF00000030F8F8FCFC7E7E7E26
:101D30003E3E3E3E7E7EFEFEFCFCF8E0800000FF64
:101D4000FFFFFFFFFFFF000080C0E0F0F8FCFEFE99
:101D50007E3E1E0E06C0E0F0F8FCFCFE7E3E3E3EDF
:101D60003E3E7EFEFCFCF8F0C0800000FEFEFEFE63
:101D7000FEFEFEFEFFFFFFFFFFFFFF00031FFFFF52
:101D8000FFFFFFFCE0E0FCFFFFFFFFFF1F0100FF84
:101D9000FFFFFFFFFFFF0000C0E0F0F0F8F8FC7C61
:101DA0007C3C3C3E1E1E1EFFFFFFFFFFFFFF0000AE
:101DB000FFFFFFFFFFFFFFFEFFFFFFFFFFFFFFF142
:101DC000C080000000FFFFFFFFFFFFFF3C3C3C3CEA
:101DD0003C3C3C3C3C3F3F3F3F3F3F00000000005D
:101DE0000000000000FFFFFFFFFFFFFF00000000FA
:101DF000073FFFFFFFFFFFFFFFFF3F07000000005F
:101E0000FFFFFFFFFFFFFF00003F7FFFFFFFFFFC23
:101E1000FCF8F8F87C7C3C3EFFFFFFFFFFFFFF0073
:101E200000FFFFFFFFFFFFFF0301000003071F7F0D
:101E3000FFFFFFFEFCF0E38F1F3F3F7F7FFEFCF8BC
:101E4000F8F0F0F0F8F8FCFC7E7E3C300000FEFE7E
:101E5000FEFEFEFEFEFE43414E43454C00207365F0
:101E60006300206D696E0020686F75720020686FD6
:101E700075727300000000000000005F00000007A2
:101E8000000700147F147F14242A7F2A12231308CA
:101E9000646236495522500005030000001C2241AF
:101EA000000041221C00082A1C2A0808083E0808D5
:101EB000005030000008080808080060600000209A
:101EC000100804023E5149453E00427F40004261F5
:101ED0005149462141454B311814127F1027454581
:101EE00045393C4A49493001710905033649494998
:101EF00036064949291E00363600000056360000D5
:101F0000000814224114141414144122140800026D
:101F100001510906324979413E7E1111117E7F49F6
:101F20004949363E414141227F4141221C7F494976
:101F300049417F090901013E414151327F080808AA
:101F40007F00417F41002040413F017F0814224132
:101F50007F404040407F0204027F7F0408107F3EA4
:101F60004141413E7F090909063E4151215E7F09F9
:101F7000192946464949493101017F01013F404045
:101F8000403F1F2040201F7F2018207F631408142B
:101F9000630304780403615149454300007F4141D4
:101FA000020408102041417F0000040201020440A5
:101FB00040404040000102040020545454787F48BF
:101FC0004444383844444420384444487F385454C6
:101FD0005418087E090102081454543C7F08040474
:101FE0007800447D40002040443D00007F1028449C
:101FF00000417F40007C041804787C080404783891
:10200000444444387C14141408081414187C7C08C4
:102010000404084854545420043F4440203C4040A9
:10202000207C1C2040201C3C4030403C4428102890
:10203000440C5050503C4464544C44000836410019
:1020400000007F0000004136080008082A1C08082C
:102050001C2A08087072696E746572206265642EAD
:10206000006F662061646A757374696E6720796FAA
:1020700075720074726F756768742074686520707B
:10208000726F6365737300492077696C6C206775A4
:1020900069646520796F7500434F4E54494E55452C
:1020A00000473120462569205A2569205825692096
:1020B00059256900473238205A302058302059308D
:1020C0000066726F6D20746865206275696C64705B
:1020D0006C6174652E0061206D696C6C696D65744E
:1020E0006572206177617900756E74696C2074681F
:1020F00065206E6F7A7A6C6520697300526F746127
:1021000074652074686520627574746F6E00342F76
:10211000323100434F4E54494E554500434F4E54C3
:10212000494E554500473120462569205A30004721
:1021300031204625692058256920592569004731F5
:1021400020462569205A350066726F6D20746865D7
:10215000206275696C64706C6174652E006973200F
:1021600061206D696C6C696D657465722061776161
:10217000790073637265772074696C6C207468658C
:10218000206E6F7A7A6C65005475726E206C65668D
:1021900074206275696C64706C61746500352F32EF
:1021A0003100434F4E54494E554500473120462596
:1021B00069205A300047312046256920582569207A
:1021C00059256900473120462569205A3500667235
:1021D0006F6D20746865206275696C64706C6174E1
:1021E000652E0069732061206D696C6C696D657482
:1021F0006572206177617900736372657720746915
:102200006C6C20746865206E6F7A7A6C650054750A
:10221000726E207269676874206275696C64706C94
:1022200061746500362F323100434F4E54494E558C
:10223000450074686520626564206C6576656C2E67
:1022400000706170657220746F2066696E652D7410
:10225000756E65006E6F77207573652061207368F9
:10226000656574206F6600526570656174207468DE
:10227000697320737465702C2062757400372F3277
:102280003100434F4E54494E5545004731204625B5
:1022900069205A3000473120462569205825692099
:1022A00059256900473120462569205A3500626961
:1022B0007420726573697374616E63652E00796F43
:1022C00075206665656C2061206C6974746C6500AE
:1022D000746865206265642026206E6F7A7A6C656A
:1022E0002074696C6C00536C6964652061207061B6
:1022F000706572206265747765656E00382F3231C3
:1023000000434F4E54494E554500434F4E54494E9D
:10231000554500746865206C65667420636F726E45
:1023200065722E2E2E005265706561742074686986
:102330007320666F7200392F323100434F4E54497B
:102340004E55450074686520726967687420636F34
:10235000726E65722E2E2E00526570656174207447
:1023600068697320666F720031302F323100434F3D
:102370004E54494E554500444F4E4500746F2069F8
:102380006E73657274206D6174657269616C2E0084
:10239000746865206E657874207374657020697345
:1023A00000746865206275696C64706C61746500A6
:1023B0004E6F772074686174207765206C65766550
:1023C0006C65640031312F323100434F4E54494E19
:1023D00055450047312046313230303020583131B8
:1023E00030205930006D6174657269616C206C6FCA
:1023F0006164696E67007072696E746865616420FB
:1024000068656174696E6720666F7200506C656103
:10241000736520776169742C0031322F323100618D
:10242000626F766520746865206172726F772E0026
:10243000796F757220556C74696D616B6572322CA1
:102440000066726F6D207468652072656172206F1E
:102450006600496E73657274206E6577206D6174D5
:10246000657269616C0031332F323100434F4E5435
:10247000494E5545004C6F6164696E67206D61740B
:10248000657269616C2E2E2E0031342F3231006658
:10249000726F6D206E6F7A7A6C652E2E2E006D61D4
:1024A00074657269616C2065786974730050757326
:1024B0006820627574746F6E207768656E003135C0
:1024C0002F323100434F4E54494E554500556C74E0
:1024D000696D616B6572322E00696E736572746529
:1024E0006420696E2074686520006D61746572698E
:1024F000616C20796F752068617665004E6578742F
:102500002C2073656C656374207468650031362F08
:1025100032310052454144590031372F32310041A8
:10252000425300504C4100697320746869732072F3
:10253000696768743F00414253206173206D617484
:10254000657269616C2C00596F7520686176652031
:1025500063686F73656E0031382F3231004E4F0063
:10256000594553006974206973207573696E672E2D
:10257000006F66206D6174657269616C006B6E6FCF
:1025800077732077686174206B696E64004E6F7793
:1025900020796F757220556C74696D616B6572324C
:1025A0000031392F323100434F4E54494E554500CA
:1025B0006D616B652061203344205072696E742117
:1025C0000049276D207265616479206C65742773FA
:1025D0000032302F32310041524520594F552052A0
:1025E000454144593F00746F207072696E742069D0
:1025F000742100616E642070726573732074686565
:1026000020627574746F6E006F6E2074686520535D
:10261000442D636172640053656C656374206120AE
:102620007072696E742066696C650032312F3231C8
:10263000004C45542753205052494E540052656176
:1026400064696E6720636172642E2E2E0032312F12
:10265000323100796F757220556C74696D616B65EC
:1026600072322E2E2E00746861742063616D6520B5
:102670007769746800506C6561736520696E736575
:1026800072742053442D636172640032312F3231F1
:1026900000697320746869732072696768743F0009
:1026A000504C41206173206D6174657269616C2CBE
:1026B00000596F7520686176652063686F73656E79
:1026C0000031382F3231004E4F0059455300473208
:1026D00038205A3000627574746F6E20746F2063F6
:1026E0006F6E74696E756500556C74696D616B65AC
:1026F0007221205072657373207468650073746171
:1027000072747570206F6620796F75720057656CF2
:10271000636F6D6520746F207468652066697273DD
:102720007400312F323100434F4E54494E5545000D
:10273000612066697273742072756E2077697A61A0
:1027400072642E0077616C6B20796F7520746872EB
:102750006F75676800666972737420737461727450
:10276000757020492077696C6C00426563617573F0
:102770006520746869732069732074686500322F5E
:10278000323100434F4E54494E55450047312046A3
:102790002569205A256900473238205A3000676F72
:1027A000696E6720746F20646F2074686174206E96
:1027B0006F772E0061646A7573746D656E74732C27
:1027C00020776520617265007765206E65656420FD
:1027D000746F20646F20736F6D650041667465725D
:1027E000207472616E73706F72746174696F6E00C1
:1027F000332F323100434F4E54494E554500473137
:1028000020462569205A25692058256920592569BF
:1028100000473238205830205930004300432F0001
:10282000436C69636B20746F2072657475726E00FF
:102830004265642074656D70657261747572653A85
:10284000004300432F00436C69636B20746F207258
:10285000657475726E00486561642074656D70659D
:102860007261747572653A0052455455524E00417A
:102870004456414E43454400424544204C4556454C
:102880004C004731205A343000473238205A30004B
:10289000473238205A3000473238205830205930DB
:1028A00000414456414E43454400746F20646566C0
:1028B00061756C743F00526573657420657665724E
:1028C000797468696E67004E4F005945530056652C
:1028D0007273696F6E2031332E3130004F63742074
:1028E000313520323031332031343A33343A3032DA
:1028F0000052657475726E006D6D2F736563004DC7
:102900006178207370656564205A006D6D2F736562
:1029100063004D61782073706565642059006D6DAA
:102920002F736563004D617820737065656420586E
:10293000006D6D2F73656300582F59204A65726BC7
:102940000030306D6D2F7365635E320041636365E7
:102950006C65726174696F6E004D4F54494F4E0043
:102960006D6D2F736563006D6D2F736563006D6D05
:102970002F736563006D6D2F736563006D6D2F732D
:1029800065635E32003F3F3F004D617820737065A4
:102990006564205A004D6178207370656564205924
:1029A000004D6178207370656564205800582F5978
:1029B000204A65726B00416363656C65726174697E
:1029C0006F6E003C2052455455524E006D6D2F7372
:1029D0006563005265747261637420737065656429
:1029E000006D6D0052657472616374206C656E6772
:1029F00074680052455452414354494F4E006D6D26
:102A00002F736563006D6D003F3F3F005265747228
:102A100061637420737065656400526574726163EC
:102A200074206C656E677468003C205245545552A2
:102A30004E004300432F00436C69636B20746F208A
:102A400072657475726E00526F7461746520746F74
:102A500020657874727564650048656164207465EA
:102A60006D70657261747572653A00250042726915
:102A70006768746E657373004C45440025003F3FE2
:102A80003F0020476C6F77207768656E20646F6E1B
:102A90006500204F6E207768696C65207072696EE2
:102AA00074696E670020416C77617973204F6666A8
:102AB0000020416C77617973204F6E004272696724
:102AC00068746E657373003C2052455455524E0035
:102AD0003F3F3F00466163746F7279207265736592
:102AE000740056657273696F6E004D6F74696F6E16
:102AF0002073657474696E677300526574726163E4
:102B000074696F6E2073657474696E6773004D6FBE
:102B10007665206D6174657269616C0052616973DC
:102B20006520626564004C6F7765722062656400A1
:102B3000486F6D65206865616400486561747570F3
:102B40002062656400486561747570206865616421
:102B5000004C45442073657474696E6773003C20B3
:102B600052455455524E0041425300504C41005280
:102B7000455455524E0053455454494E4753004313
:102B800048414E4745004D4154455249414C005340
:102B9000656C6563746564206D6174657269616CF0
:102BA0003A004F4B0025004D6174657269616C20DD
:102BB000666C6F7700250046616E207370656564F2
:102BC000006D6D004D6174657269616C20446961CE
:102BD0006D657465720043004265642054656D70D4
:102BE0006572617475726500430054656D7065723D
:102BF0006174757265004D4154455249414C002540
:102C00000025006D6D00430043003F3F3F00466CD0
:102C10006F7720250046616E004469616D657465BB
:102C20007200486561746564206265640054656D76
:102C30007065726174757265003C2052455455523E
:102C40004E004D6F64696679207468652073657401
:102C500074696E677300250046616E3A2000430078
:102C600043002500466C6F773A006D6D0043757325
:102C7000746F6D697A65003C2052455455524E0080
:102C8000666F72206D6174657269616C2072656D2A
:102C90006F76616C0048656174696E672070726957
:102CA0006E746865616400526576657273696E67FB
:102CB000206D6174657269616C0052656D6F766537
:102CC000206D6174657269616C0043414E43454CEF
:102CD0000052454144590047312046256920582576
:102CE0006920592569004732382058302059300072
:102CF00061626F766520746865206172726F772EED
:102D000000796F7572206D616368696E652C00666D
:102D1000726F6D20746865206261636B73696465AE
:102D2000206F6600496E73657274206E6577206D42
:102D30006174657269616C0043414E43454C0052B9
:102D40004541445900466F7277617264696E67202D
:102D50006D6174657269616C00636F6D6573206F7E
:102D6000757420746865206E6F7A7A6C650057619F
:102D700069742074696C6C206D6174657269616C32
:102D80000043414E43454C00524541445900534491
:102D90002043415244003B464C41564F523A556CF9
:102DA000746947436F6465003B464C41564F523A45
:102DB000556C746947436F6465004E6F2066696C9B
:102DC000657320666F756E6421004F4B004F4B009A
:102DD00052656164696E6720636172642E2E2E00F5
:102DE000506C6561736520696E73657274206361F0
:102DF0007264004E6F205344204341524421003CF2
:102E0000204241434B003C2052455455524E0066EF
:102E1000726F6D2074686520736C696365722E0033
:102E200073657474696E672077697468207365745C
:102E300074696E67006F76657272696465206D6192
:102E40006368696E6500546869732066696C652003
:102E500077696C6C0043414E43454C00434F4E54E0
:102E6000494E5545004731204631353030204530F8
:102E70000047393220452D25690047323800473256
:102E80003800473120463135303020453000473951
:102E900032204525690063617264210072656164B6
:102EA000696E67205344004572726F7220776869BB
:102EB0006C650052455455524E20544F204D4149A7
:102EC0004E00746865207072696E742E00596F75BB
:102ED0002063616E2072656D6F7665005072696E59
:102EE000742066696E697368656400430050726996
:102EF0006E74657220636F6F6C696E6720646F77A4
:102F00006E004241434B20544F204D454E550054D6
:102F1000696D65206C6566740054696D65206C652B
:102F2000667420756E6B6E6F776E004300430048C9
:102F3000656174696E672062656400430043004800
:102F4000656174696E67005072696E74696E673A84
:102F50000041424F52540054554E450041626F7239
:102F60007420746865207072696E743F004E4F0063
:102F70005945530025004D6174657269616C206686
:102F80006C6F7700250046616E2073706565640084
:102F900025005072696E7420737065656400545525
:102FA0004E45006D6D2F73656300526574726163E9
:102FB00074207370656564006D6D00526574726194
:102FC0006374206C656E67746800524554524143C7
:102FD00054494F4E006D6D2F736563006D6D003F5A
:102FE0003F3F00526574726163742073706565645D
:102FF0000052657472616374206C656E677468005A
:103000003C2052455455524E0025002500430043B4
:103010000043004300250052657472616374696F58
:103020006E004D6174657269616C20666C6F77002B
:1030300046616E2073706565640042656420746546
:103040006D70657261747572650054656D7065723E
:103050006174757265005370656564003C2052456B
:103060005455524E00507265706172696E672074DB
:103070006F207072696E743A0048656174696E679A
:103080002075702E2E2E0041424F52540054554E42
:1030900045004E6F20696E666F20617661696C61D4
:1030A000626C65006D006D004D6174657269616CE4
:1030B0003A200054696D653A20003B4D4154455219
:1030C00049414C3A003B54494D453A00466F6C64C7
:1030D000657200494E46494E4954594E414ECDCC39
:1030E000CC3D0AD7233C17B7D13877CC2B329595F6
:1030F000E6241FB14F0A000020410000C8420040F2
:103100001C4620BCBE4CCA1B0E5AAEC59D74BD2FBA
:10311000DD51B82F11241FBECFEFD1E2DEBFCDBFEE
:1031200000E00CBF14E0A0E0B2E0E8E8F6EA01E05D
:103130000BBF02C007900D92AC32B107D9F715E171
:10314000ACE2B4E001C01D92A73CB107E1F711E386
:10315000C2E1D1E304C02297FE010E9434D3CE30F5
:10316000D107C9F704D00C943FCA0C940000CF9348
:10317000DF9332D10E94CF4EC0E0D0E00E94464E95
:103180002097E1F30E940000F9CFCF92DF92EF92F7
:10319000FF920F931F93CF93DF937C016B018A0102
:1031A000C0E0D0E00FC0D6016D916D01D701ED9167
:1031B000FC910190F081E02DC7011995C80FD91F2E
:1031C000015010400115110571F7CE01DF91CF912B
:1031D0001F910F91FF90EF90DF90CF900895823074
:1031E000B9F0833028F4882351F0813051F50AC0BA
:1031F000843011F18430E8F0853019F520C0109248
:103200006E00089580916F008D7F80936F00089508
:10321000809170008D7F8093700081E08093B0007A
:103220008091B100887F84608093B1001092B300D8
:1032300008951092710008951092720008951092EE
:10324000730008951F93182F80913603811711F092
:103250009FEF06C0EFE2F1E094918FEF8093360389
:10326000892FBDDF812F60E0AAD21F9108951F92A0
:103270000F920FB60F920BB60F9211242F933F931C
:103280004F935F936F937F938F939F93AF93BF936E
:10329000EF93FF9380912C0490912D04A0912E0424
:1032A000B0912F040097A105B10551F1E0913004D0
:1032B000F09131048081909132048927808380913C
:1032C0002C0490912D04A0912E04B0912F04181677
:1032D00019061A061B06BCF480912C0490912D044B
:1032E000A0912E04B0912F040197A109B1098093F8
:1032F0002C0490932D04A0932E04B0932F0403C0AC
:10330000809136039FDFFF91EF91BF91AF919F9125
:103310008F917F916F915F914F913F912F910F907E
:103320000BBE0F900FBE0F901F9018951F920F921B
:103330000FB60F9211242F933F938F939F93AF93C8
:10334000BF938091370490913804A0913904B091D3
:103350003A0430913B040196A11DB11D232F2D5F2E
:103360002D3720F02D570196A11DB11D20933B0450
:103370008093370490933804A0933904B0933A04AF
:103380008091330490913404A0913504B0913604B7
:103390000196A11DB11D8093330490933404A09332
:1033A0003504B0933604BF91AF919F918F913F91B7
:1033B0002F910F900FBE0F901F9018958FB7F89414
:1033C00020913704309138044091390450913A04E7
:1033D0008FBFB901CA010895789484B5826084BD15
:1033E00084B5816084BD85B5826085BD85B5816009
:1033F00085BDEEE6F0E0808181608083E1E8F0E069
:103400001082808182608083808181608083E0E897
:10341000F0E0808181608083E1EBF0E08081846076
:103420008083E0EBF0E0808181608083E1E9F0E07F
:10343000808182608083808181608083E0E9F0E028
:10344000808181608083E1EAF0E080818260808316
:10345000808181608083E0EAF0E080818160808308
:10346000E1E2F1E0808182608083808181608083FD
:10347000E0E2F1E0808181608083EAE7F0E0808132
:10348000846080838081826080838081816080838A
:103490008081806880831092C10008951F93CF932C
:1034A000DF93182FEB0161E0D7D0209709F4CAC051
:1034B000CF3FD10509F4C9C0E12FF0E0E65FFD4F31
:1034C0008491893009F466C08A30B0F48430F1F117
:1034D000853040F4823059F1833070F5813009F045
:1034E000AEC020C0873009F443C0883008F048C01F
:1034F000863009F0A4C034C08D3009F478C08E3015
:1035000038F48B3009F45AC08C3008F066C04CC0D7
:10351000803109F480C0813109F487C08F3009F00F
:103520008EC06FC084B5806884BDC7BD91C084B5AE
:10353000806284BDC8BD8CC080918000806880930B
:103540008000D0938900C093880082C08091800061
:10355000806280938000D0938B00C0938A0078C0F3
:103560008091B00080688093B000C093B30070C0B9
:103570008091B00080628093B000C093B40068C0B6
:1035800080919000806880939000D0939900C093C0
:1035900098005EC080919000806280939000D093EC
:1035A0009B00C0939A0054C08091900088608093E3
:1035B0009000D0939D00C0939C004AC08091A000D1
:1035C00080688093A0008091A0008F7B8093A000F2
:1035D000D093A900C093A8003BC08091A000806256
:1035E0008093A000D093AB00C093AA0031C080911B
:1035F000A00088608093A000D093AD00C093AC0081
:1036000027C080912001806880932001D0932901F8
:10361000C09328011DC08091200180628093200109
:10362000D0932B01C0932A0113C0809120018860A0
:1036300080932001D0932D01C0932C0109C0C03884
:10364000D1051CF4812F60E002C0812F61E0B7D06A
:10365000DF91CF911F910895CF93DF93482F50E0D2
:10366000CA018C539E4FFC01349142585E4FFA01BF
:103670008491882369F190E0880F991FFC01E05D37
:10368000FE4FA591B491FC01E65BFE4FC591D4912C
:10369000662351F42FB7F8948C91932F909589233A
:1036A0008C93888189230BC0623061F42FB7F89422
:1036B0008C91932F909589238C938881832B888379
:1036C0002FBF06C09FB7F8948C91832B8C939FBF1C
:1036D000DF91CF910895893009F449C08A30A0F470
:1036E000843051F1853040F4823079F1833000F537
:1036F000813009F063C026C0873079F1883098F5B1
:10370000863009F05BC025C08D3009F442C08E3090
:1037100028F48B30B1F18C30C0F52DC0803109F424
:1037200042C0813109F445C08F3009F047C037C02D
:10373000809180008F7703C0809180008F7D80937F
:103740008000089584B58F7702C084B58F7D84BDD5
:1037500008958091B0008F7703C08091B0008F7D75
:103760008093B0000895809190008F7707C080917A
:1037700090008F7D03C080919000877F80939000A0
:1037800008958091A0008F7707C08091A0008F7D61
:1037900003C08091A000877F8093A000089580914E
:1037A00020018F7703C0809120018F7D80932001BD
:1037B000089580912001877F809320010895FF92D2
:1037C0000F931F93F62E482F50E0CA01865F9D4F3E
:1037D000FC012491CA018C539E4FFC011491425864
:1037E0005E4FFA0104910023C1F0222311F0822FD1
:1037F00072DFE02FF0E0EE0FFF1FE65BFE4FA591BA
:10380000B4919FB7F894FF2021F48C9110958123F7
:1038100002C08C91812B8C939FBF1F910F91FF90C1
:103820000895AC01DB01FA0190E02EE28C91803228
:1038300029F0983009F421938C9181939F5F119620
:103840009B30A1F71082CA010895FC01128216A6CE
:103850000895FC0186A5882311F081E082830895F4
:10386000FC018281811112820895CF93DF93EC01D4
:10387000FC01EB55FE4F8081882309F461C0815023
:103880008083DE01AC5ABF4FFE01ED58FF4F8BE144
:1038900001900D928150E1F7FE01EE5AFF4FCF5893
:1038A000DF4F88819981C157D0409183808330E078
:1038B000BE016B557E4F3FC0832F90E0AC014F5F40
:1038C0005F4FDC01E5E0AA0FBB1FEA95E1F7A81BFB
:1038D000B90BAC0FBD1FFA0125E0EE0FFF1F2A95B3
:1038E000E1F7E41BF50BEC0FFD1FAD58BF4FED5892
:1038F000FF4F2BE101900D922150E1F7FC0125E0F3
:10390000EE0FFF1F2A95E1F7E81BF90BEC0FFD1FE7
:10391000EF58FF4FDA0185E0AA0FBB1F8A95E1F748
:10392000A41BB50BAC0FBD1FAF58BF4F8D919C9121
:10393000918380833F5FFB018081381708F4BCCFFF
:10394000DF91CF910895FC0184E294E0918380831C
:103950008781882321F0CF0104960C94006D08958F
:103960000F931F938C010E94667B0E94627AC801AC
:1039700083539E4F0E94006DF801128280E592E011
:103980000E945B501F910F910895CF92DF92EF92AA
:10399000FF920F931F93DF93CF93CDB7DEB76F974F
:1039A0000FB6F894DEBF0FBECDBF8C016B01095A74
:1039B0001F4FD8018C9107551040882321F48FE2C6
:1039C000E82EF12C03C0B0E5EB2EF12CE00EF11E39
:1039D00084E294E09A8389831C821B8218861D826C
:1039E000B7016C5F7F4FCE010596A60121E00E94D2
:1039F0003874882391F5ECE5F2E0949108C0809149
:103A0000C00085FFFCCF9093C60031969491992316
:103A1000B1F7E2E6F2E0949108C08091C00085FF22
:103A2000FCCF9093C600319694919923B1F709C0C9
:103A30008091C00085FFFCCF0894C11CD11C9093DD
:103A4000C600F6019081992399F78091C00085FF07
:103A5000FCCF8AE08093C60056C0F801EB55FE4FBC
:103A600080818A3008F03EC08F5F8083282F30E04D
:103A7000C9010197FC01A5E0EE0FFF1FAA95E1F730
:103A8000E81BF90BED58FF4FE00FF11F21503040BC
:103A9000AF01415E5F4FBF018BE1DB010D90BD01C6
:103AA000DA010D92AD018150C1F792918291329667
:103AB000968F858F7F972115310541F7D801AD5835
:103AC000BF4FF70134968BE101900D928150E1F7E1
:103AD0000F581F4FF70182819381D8018D939C93DA
:103AE00001571040D801AC5ABF4FFE0135968BE10B
:103AF00001900D928150E1F70E5A1F4F8B819C81EE
:103B0000F80191838083CE0101961DDF6F960FB679
:103B1000F894DEBF0FBECDBFCF91DF911F910F9103
:103B2000FF90EF90DF90CF900895EF92FF920F9368
:103B30001F938C019DECE92E91E0F92EE00EF11E11
:103B4000C7010E94B16CC7010E94006DF80110828C
:103B500011821F910F91FF90EF900895CF92DF9205
:103B6000EF92FF920F931F93CF93DF937C016B0132
:103B7000DB010D900020E9F78D0101501040061B7C
:103B8000170BEDECF1E0EE0EFF1ED7011C92E3E304
:103B9000FEEFEE0EFF1ECB016EE470E00E94CCCA79
:103BA000EC01009731F4F8013197EC0DFD1D860111
:103BB0000EC060E270E00E94CCCA8C010F5F1F4F04
:103BC000CE016AE270E00E94CCCAFC0131978DE020
:103BD00081838AE082831382C70187539E4FB80195
:103BE0000E9432758DEC91E0E80EF91ED7018C91A0
:103BF000882319F1ECE8F2E0949108C08091C000AC
:103C000085FFFCCF9093C600319694919923B1F72C
:103C1000E3E9F2E0949108C08091C00085FFFCCFF9
:103C20009093C600319694919923B1F78091C0008A
:103C300085FFFCCF8AE08093C600DF91CF911F9172
:103C40000F91FF90EF90DF90CF900895CF93DF9387
:103C5000EC018EA5882309F43DC0E7ECF2E09491D5
:103C600008C08091C00085FFFCCF9093C6003196BC
:103C700094919923B1F7C051DE4F488159816A81EF
:103C80007B81C05FD14084EC98E02AE030E00E9464
:103C90007452E5ECF2E0949108C08091C00085FF79
:103CA000FCCF9093C600319694919923B1F7C851F7
:103CB000DE4F488159816A817B81C85ED14084ECA6
:103CC00098E02AE030E00E9474528091C00085FFA5
:103CD000FCCF12C0E5EBF2E0949108C08091C000E7
:103CE00085FFFCCF9093C600319694919923B1F74C
:103CF0008091C00085FFFCCF8AE08093C600C95543
:103D0000DE4F68816623E1F0E9EAF2E0949108C0B1
:103D10008091C00085FFFCCF9093C60031969491AE
:103D20009923B1F784EC98E070E04AE050E00E94FB
:103D3000C3528091C00085FFFCCF8AE08093C6000B
:103D4000DF91CF9108952F923F924F925F926F92A1
:103D50007F928F929F92AF92BF92CF92DF92EF921B
:103D6000FF920F931F93DF93CF93CDB7DEB7AD973D
:103D70000FB6F894DEBF0FBECDBF5C014B014DA75F
:103D8000FC0186A5882309F4E1C13DEC432E31E016
:103D9000532E4A0C5B1CC2010E94006DF501128279
:103DA0001A8A1D8A198A188A84E294E09F878E876E
:103DB0002EE4C22ED12CCA0CDB1C8FE290E0A80EA0
:103DC000B91EF601B182A08281ED9FEFA80EB91E47
:103DD000F40180818F3209F08DC0C4016FE270E080
:103DE0000E94CCCA7C010894E11CF11C3E0108949D
:103DF000611C711C160178C0C7016FE270E00E945F
:103E0000CCCA6C01009709F483C0E816F90608F0E3
:103E10007FC08C010E191F09C301B701A8010E94C0
:103E2000ECCA060D171DF8011082F30107C080913E
:103E3000C00085FFFCCF31969093C60090819923F6
:103E4000B1F78091C00085FFFCCFFAE0F093C60087
:103E5000F101608171816115710519F460E070E014
:103E600002C06C5F7F4FCE014296A30121E00E9409
:103E70003874882371F5EBE7F3E0949108C08091E2
:103E8000C00085FFFCCF9093C60031969491992392
:103E9000B1F7FE01319607C08091C00085FFFCCFCD
:103EA00031969093C60090819923B1F7E9E7F3E04A
:103EB000949108C08091C00085FFFCCF9093C6000C
:103EC000319694919923B1F78091C00085FFFCCF82
:103ED00037C18EE090E08C0F9D1FF10191838083AC
:103EE00076010894E11CF11C92E0E916F10408F057
:103EF00083CF0BC0E0E5F0E0AE0EBF1EF601B1824D
:103F0000A08280EB9FEFA80EB91E082DF92C01C0EE
:103F10000E2DF501E25BFF4F9DA5992309F4ADC07D
:103F2000608171816115710519F460E070E002C073
:103F30006C5F7F4FC201402F5F2D21E00E943874DB
:103F4000882309F46AC0EEEDF1E0AE0EBF1EF50164
:103F500040815181628173818AE090E0A80EB91E90
:103F6000F501408351836283738388E19EEFA80E3D
:103F7000B91EEBE6F3E0949108C08091C00085FF84
:103F8000FCCF9093C600319694919923B1F7802F7E
:103F90009F2D9C01F90107C08091C00085FFFCCFD7
:103FA00031969093C60090819923B1F7E3E6F3E050
:103FB000949108C08091C00085FFFCCF9093C6000B
:103FC000319694919923B1F784EC98E02AE030E09F
:103FD0000E9474528091C00085FFFCCF8AE08093DC
:103FE000C600E0EFF1E0AE0EBF1EF50110821182B7
:103FF00012821382E5E5F3E0949108C08091C0003D
:1040000085FFFCCF9093C600319694919923B1F728
:104010008091C00085FFFCCF93C0E1E4F3E0949170
:1040200008C08091C00085FFFCCF9093C6003196F8
:1040300094919923B1F7802F9F2D9C01F90107C01E
:104040008091C00085FFFCCF31969093C60090818F
:104050009923B1F7EFE3F3E0949108C08091C00099
:1040600085FFFCCF9093C600319694919923B1F7C8
:104070008091C00085FFFCCF63C0608171816115B4
:10408000710519F460E070E002C06C5F7F4FC201FF
:10409000402F5F2D26E50E943874882381F5EBE2DE
:1040A000F3E0949108C08091C00085FFFCCF90930D
:1040B000C600319694919923B1F7802F9F2D9C01D2
:1040C000F90107C08091C00085FFFCCF3196909325
:1040D000C60090819923B1F7E9E2F3E0949108C01A
:1040E0008091C00085FFFCCF9093C60031969491DB
:1040F0009923B1F78091C00085FFFCCF21C081E0FA
:10410000F5018083E7E1F3E0949108C08091C0005D
:1041100085FFFCCF9093C600319694919923B1F717
:10412000F40107C08091C00085FFFCCF31969093C9
:10413000C60090819923B1F78091C00085FFFCCF24
:104140008AE08093C600CE010E96FDDBAD960FB6D9
:10415000F894DEBF0FBECDBFCF91DF911F910F91BD
:10416000FF90EF90DF90CF90BF90AF909F908F9097
:104170007F906F905F904F903F902F900895FC013B
:1041800081E08183CF0140E0DECD2F923F924F92BC
:104190005F926F927F928F929F92AF92BF92CF92D7
:1041A000DF92EF92FF920F931F93DF93CF93CDB7E0
:1041B000DEB7AC970FB6F894DEBF0FBECDBF5C0183
:1041C0004B01FC0186A5882309F437C1C50183533F
:1041D0009E4F0E94006DF50112821A8A1D8A198A6B
:1041E000188A84E294E09F878E875EE4C52ED12CE6
:1041F000CA0CDB1C2FE230E0A20EB31EF601B18226
:10420000A08221ED3FEFA20EB31EF40180818F3218
:1042100009F090C0C4016FE270E00E94CCCA7C013A
:104220000894E11CF11C3E010894611C711C2601DC
:1042300042E1242E312C2C0E3D1E77C0C7016FE2C7
:1042400070E00E94CCCA6C01009709F481C0E816A6
:10425000F90608F07DC08C010E191F09C301B701D2
:10426000A8010E94ECCA060D171DF8011082F30187
:1042700007C08091C00085FFFCCF31969093C600A7
:1042800090819923B1F78091C00085FFFCCFFAE0BF
:10429000F093C600F201608171816115710519F416
:1042A00060E070E002C06C5F7F4FC101A30121E0BC
:1042B0000E943874882371F5E3E0F3E0949108C01C
:1042C0008091C00085FFFCCF9093C60031969491F9
:1042D0009923B1F7FE01319607C08091C00085FF98
:1042E000FCCF31969093C60090819923B1F7E1E01D
:1042F000F3E0949108C08091C00085FFFCCF9093BB
:10430000C600319694919923B1F78091C00085FF42
:10431000FCCF8DC02EE030E02C0F3D1FF201318329
:10432000208376010894E11CF11CE114F10409F0EA
:1043300085CF0BC080E590E0A80EB91EF601B182D2
:10434000A08220EB3FEFA20EB31ED82C092D02C095
:10435000DE2C0F2D8EE490E0A80EB91EF5018081B1
:10436000918122EB3FEFA20EB31E009719F480E07B
:1043700090E001C004966D2D702F0E940475882373
:1043800039F1E3EFF2E0949108C08091C00085FF1D
:10439000FCCF9093C600319694919923B1F78D2D5F
:1043A000902F9C01F90107C08091C00085FFFCCFD0
:1043B00031969093C60090819923B1F780EF91E0F8
:1043C000A80EB91EF501108211821282138232C02A
:1043D000EBEDF2E0949108C08091C00085FFFCCF26
:1043E0009093C600319694919923B1F78D2D902F1B
:1043F0009C01F90107C08091C00085FFFCCF319678
:104400009093C60090819923B1F7E9EDF2E0949181
:1044100008C08091C00085FFFCCF9093C600319604
:1044200094919923B1F78091C00085FFFCCF8AE079
:104430008093C600CE010E9686DAAC960FB6F8943D
:10444000DEBF0FBECDBFCF91DF911F910F91FF90C7
:10445000EF90DF90CF90BF90AF909F908F907F9024
:104460006F905F904F903F902F900895EF92FF9242
:104470000F931F93CF93DF938C01FC0116A686A99F
:10448000882321F0C801C3960E94006D66EAE62EDB
:1044900061E0F62EE00EF11EC70160E045E30E94E8
:1044A000D46A882309F5ECE5F2E0949108C0809184
:1044B000C00085FFFCCF9093C6003196949199235C
:1044C000B1F7EDEBF3E0949108C08091C00085FF57
:1044D000FCCF9093C600319694919923B1F78091C7
:1044E000C00085FFFCCF7DC0E801C555DE4FCE0181
:1044F000B70141E00E94C375882341F5CE01B701A1
:1045000040E00E94C375882309F5ECE8F2E094913D
:1045100008C08091C00085FFFCCF9093C600319603
:1045200094919923B1F7EAEAF3E0949108C080915D
:10453000C00085FFFCCF9093C600319694919923DB
:10454000B1F78091C00085FFFCCF4BC0C801C39676
:10455000BE010E94D76F882309F5ECE8F2E0949140
:1045600008C08091C00085FFFCCF9093C6003196B3
:1045700094919923B1F7EAE9F3E0949108C080910E
:10458000C00085FFFCCF9093C6003196949199238B
:10459000B1F78091C00085FFFCCF23C081E0F80116
:1045A00086A7ECE5F2E0949108C08091C00085FFF9
:1045B000FCCF9093C600319694919923B1F7EFE820
:1045C000F3E0949108C08091C00085FFFCCF9093E8
:1045D000C600319694919923B1F78091C00085FF70
:1045E000FCCF8AE08093C600D801AC5ABF4FF801D7
:1045F000F3968BE101900D928150E1F7F80181A9CA
:1046000092A90E5A1F4FF8019183808302551040E2
:10461000C8018F96025B1F4FF80191838083DF9161
:10462000CF911F910F91FF90EF9008952F923F929D
:104630004F925F926F927F929F92AF92BF92CF9272
:10464000DF92EF92FF920F931F93DF93CF93CDB73B
:10465000DEB7CC55D0400FB6F894DEBF0FBECDBF4D
:104660006C01662311F524EF31E0C20ED31ED60192
:104670008C91ECE0FEEFCE0EDF1E882309F4E1C042
:104680002CEE31E0C20ED31ED601ED90FD900D91BF
:104690001C91E4E1FEEFCE0EDF1E0E94DE19E6164D
:1046A000F7060807190708F4CCC024EF31E0C20E62
:1046B000D31ED6011C92ECE0FEEFCE0EDF1ED6011B
:1046C0009E968C91882339F4C601D0DEF60186A52A
:1046D000882309F4B6C000D000D0EDB7FEB73196FC
:1046E0007E010894E11CF11CADB7BEB71296FC9296
:1046F000EE92119783E892E093838283D6019C9691
:104700008D919C919D97958384830E9421CB8701F5
:10471000EDB7FEB736960FB6F894FEBF0FBEEDBFED
:10472000570108C0D8018C9190E00E944ACAF80154
:1047300081938F01F50101900020E9F73197EA1983
:10474000FB09802F8E198E176CF3A3E3AA2EB12CD0
:10475000AC0CBD1CC50140E050E060E070E00E9480
:10476000E76B9924FDE3EF2EF12CEC0EFD1E2E01DC
:104770000894411C511CEFE16E2E712C6C0E7D1EB5
:104780007CE7272E72E0372E42C0D8018C9190E052
:104790000E944ACAF80181938F01F701019000201D
:1047A000E9F73197EE19FF09802F8E198E176CF3F8
:1047B00027968FAD27978E3751F1C701B20145E09B
:1047C00050E00E94DECA009711F500D000D0EDB78E
:1047D000FEB73196ADB7BEB712967C926E92119726
:1047E00033822282558244820E9421CBEDB7FEB7EC
:1047F00036960FB6F894FEBF0FBEEDBFC3010E9400
:10480000D45088E792E00E945B5099249394C501AC
:10481000B70140E050E00E94F66E181614F48701CC
:10482000BCCF992041F48FEF9FEFD6019D969C93CA
:104830008E939C9706C0F60184A595A5019695A731
:1048400084A7C45ADF4F0FB6F894DEBF0FBECDBFAA
:10485000CF91DF911F910F91FF90EF90DF90CF905C
:10486000BF90AF909F907F906F905F904F903F90E0
:104870002F9008952F923F924F925F926F927F9266
:104880008F929F92AF92BF92CF92DF92EF92FF9260
:104890000F931F93DF93CF93CDB7DEB7CD58D040A2
:1048A0000FB6F894DEBF0FBECDBF8C013B016A018D
:1048B00084E090E0C80ED91EF8017096C757DF4F0C
:1048C000F983E883C958D040C8010396C957DF4F20
:1048D00099838883C758D040CA57DF4F1882C6587B
:1048E000D04036E6E32EF12CEC0EFD1E25EF822E95
:1048F00021E0922E800E911E96EFA92E91E0B92E06
:10490000A00EB11E8EE0282E312C2C0E3D1EB7E4D9
:104910004B2E512C4C0E5D1EF2013496C557DF4FC5
:10492000F983E883CB58D040ECE5F2E08491C3579B
:10493000DF4F8883CD58D04021C1F7018385282FD0
:1049400030E0A901487150704031510509F024C18F
:10495000F4019081913009F41FC1923009F41CC117
:10496000CE010196B7010E94111C1E86F3018081C1
:10497000882329F4C10160E072E00E94C1CAC1012C
:10498000B3010E94C1CAC101BE016F5F7F4F0E9487
:10499000C1CAC10160E072E00E94C1CA1CA61FA684
:1049A0001BA61AA684E294E099A788A7CE018C964C
:1049B000B601AE014F5F5F4F21E00E94387488233B
:1049C00009F03EC0F40180818823D1F5C357DF4F41
:1049D0009881CD58D040ECE5F2E008C08091C0004D
:1049E00085FFFCCF9093C600319694919923B1F73F
:1049F000E2E0F2E007C08091C00085FFFCCF319675
:104A00009093C60090819923B1F78091C00085FFF3
:104A1000FCCFFAE0F093C600FE01319607C080910A
:104A2000C00085FFFCCF31969093C60090819923FA
:104A3000B1F78091C00085FFFCCF8AE08093C6006B
:104A4000C557DF4FA881B981CB58D040FE01BC9635
:104A50008BE101900D928150E1F78AA59BA5F201AF
:104A60009383828384E294E091838083C801B101BF
:104A7000A20100DFC2010E94A31CCE0188960E9401
:104A8000A31C7CC0953E09F479C09E3209F476C01F
:104A90009F3509F473C0F8019089992331F09E3253
:104AA00009F46CC09F3509F469C023FD67C080E03C
:104AB0004031510509F481E0F80183A7882349F4C6
:104AC000F7018085873409F059C081858E3709F454
:104AD00055C0C957DF4F88819981C758D040B70169
:104AE0000E94111CF4018081882329F5F30107C07D
:104AF0008091C00085FFFCCF31969093C6009081D5
:104B00009923B1F7C957DF4FE881F981C758D040E1
:104B100007C08091C00085FFFCCF31969093C600FE
:104B200090819923B1F78091C00085FFFCCFFAE016
:104B3000F093C60023C0813039F4F5018081918162
:104B40000196918380831AC08230C1F4CA57DF4F27
:104B5000F881C658D0402F2F30E0F5018081918137
:104B600028173907F1F0CA57DF4FF881C658D040EF
:104B7000FF5FCA57DF4FF883C658D040C601B70160
:104B8000C757DF4F48815981C958D0400E94F66EFF
:104B900018160CF4D2CE05C0F7019081992309F0C4
:104BA00071CFC357DF4F0FB6F894DEBF0FBECDBF36
:104BB000CF91DF911F910F91FF90EF90DF90CF90F9
:104BC000BF90AF909F908F907F906F905F904F902D
:104BD0003F902F900895EF92FF920F931F93DF93D2
:104BE000CF93CDB7DEB76F970FB6F894DEBF0FBE89
:104BF000CDBF7C018C01025B1F4F805B9F4FF80192
:104C00009183808325EF31E0E20EF31E21E0F7016E
:104C100021937F01118210822AE03EEFE20EF31E03
:104C2000049640E050E060E070E00E94E76BF8011D
:104C300020813181DE011596F90134968BE10190D6
:104C40000D928150E1F7F901828193819C838B83DE
:104C500084E294E09A838983C70165E172E08E0162
:104C60000F5F1F4FA80106DEC8010E94A31CF701B9
:104C7000EA50FE4F808191816F960FB6F894DEBFA7
:104C80000FBECDBFCF91DF911F910F91FF90EF909D
:104C90000895EF92FF920F931F93DF93CF93CDB7B9
:104CA000DEB76F970FB6F894DEBF0FBECDBF7C01A5
:104CB0008C01025B1F4F805B9F4FF80191838083C3
:104CC00025EF31E0E20EF31E22E0F70120832BE016
:104CD0003EEFE20EF31EF701EA50FE4F60831182B1
:104CE000049640E050E060E070E00E94E76BF8015D
:104CF00020813181DE011596F90134968BE1019016
:104D00000D928150E1F7F901828193819C838B831D
:104D100084E294E09A838983C70165E172E08E01A1
:104D20000F5F1F4FA801A6DDC8010E94A31C6F964C
:104D30000FB6F894DEBF0FBECDBFCF91DF911F91AC
:104D40000F91FF90EF900895EF92FF920F931F93B2
:104D5000DF93CF93CDB7DEB76F970FB6F894DEBF72
:104D60000FBECDBF7C0185EF91E0E80EF91EF70183
:104D700010828BE09EEFE80EF91E87010D5C1F4F3D
:104D8000C80140E050E060E070E00E94E76BDE01A7
:104D90001596F8018BE101900D928150E1F7F70132
:104DA00081A992A99C838B8384E294E09A8389836E
:104DB000C70165E172E08E010F5F1F4FA8015ADD48
:104DC000C8010E94A31C6F960FB6F894DEBF0FBEF9
:104DD000CDBFCF91DF911F910F91FF90EF9008957C
:104DE0000F931F93CF93DF93DC01D3961C92D3973D
:104DF000D6961C92D697D2961C921E92D19784E298
:104E000094E0D0969C938E939F97AC5ABF4F1C9280
:104E100013961C92A755B040FD01E05BFF4FAE5AC0
:104E2000BF4F11961C921E92A255B0409183808371
:104E3000ED01C159DF4FFE0120E030E0482F148220
:104E400017821382128240839183215E3F4F7F96A7
:104E500081E02633380799F7A955BE4F89E18C9335
:104E600013961C9258961C921B961C9213961C9299
:104E7000A05DB140FD01E753FE4FA553BE4F119613
:104E80001C921E92408391835D961D921D921D92ED
:104E90001C92139718961D921D921D921C921397A7
:104EA000A05FB14012961C9212979E961C929E97FC
:104EB0001C9211961C9211978D0104511E4FF801FE
:104EC0001082118212821382AB55BE4F1C92FE01DA
:104ED000C90111920197E9F7A15BBF4F81E08C9363
:104EE000A45FB1409D961C921E929C970E94DE1971
:104EF00068577C4E8F4F9F4FF80160837183828388
:104F00009383DF91CF911F910F910895DF93CF93FA
:104F1000CDB7DEB7E0970FB6F894DEBF0FBECDBFBA
:104F2000DE011196E4EDF3E080E101900D928150F5
:104F3000E1F7DE015196E4ECF3E080E101900D929F
:104F40008150E1F7DE019196E4EBF3E080E101901E
:104F50000D928150E1F789819A81AB81BC81809368
:104F6000D9089093DA08A093DB08B093DC0889890C
:104F70009A89AB89BC898093C9089093CA08A09389
:104F8000CB08B093CC0889A19AA1ABA1BCA1809316
:104F9000E9089093EA08A093EB08B093EC088D81A0
:104FA0009E81AF81B8858093DD089093DE08A09341
:104FB000DF08B093E0088D899E89AF89B88D809312
:104FC000CD089093CE08A093CF08B093D0088DA1C0
:104FD0009EA1AFA1B8A58093ED089093EE08A09391
:104FE000EF08B093F00889859A85AB85BC858093DE
:104FF000E1089093E208A093E308B093E408898D58
:105000009A8DAB8DBC8D8093D1089093D208A093DC
:10501000D308B093D40889A59AA5ABA5BCA5809365
:10502000F1089093F208A093F308B093F4088D85EB
:105030009E85AF85B8898093E5089093E608A09394
:10504000E708B093E8088D8D9E8DAF8DB8A1809351
:10505000D5089093D608A093D708B093D8088DA50B
:105060009EA5AFA5B8A98093F5089093F608A093E4
:10507000F708B093F8080E94255780E090E4ACE967
:10508000B5E48093FD089093FE08A093FF08B093C9
:1050900000098093010990930209A0930309B0933A
:1050A000040920E030E040E050E02093F90830931C
:1050B000FA084093FB085093FC0880E29EE4A0E0CD
:1050C000B0E08093C5089093C608A093C708B0933A
:1050D000C808209311093093120940931309509383
:1050E000140980E090E0A0EAB1E480930509909370
:1050F0000609A0930709B09308098DEC9CECACEC71
:10510000BEE38093090990930A09A0930B09B09319
:105110000C0980E090E0A0EAB0E480930D09909340
:105120000E09A0930F09B0931009209354063093F1
:1051300055064093560650935706209350063093D9
:105140005106409352065093530620934C063093D9
:105150004D0640934E0650934F0686E696E6A2E42F
:10516000B1E48093840390938503A0938603B09366
:10517000870360E070E080E89FE30E94758360939E
:1051800088037093890380938A0390938B036BE762
:1051900074E184E192E40E94818360938C037093B4
:1051A0008D0380938E0390938F030E947D8280E015
:1051B00090E0A0E8BFE38093900390939103A093C5
:1051C0009203B093930384E195E090937A038093E4
:1051D000790390937C0380937B0382EE94E0909319
:1051E0007E0380937D0384E68093A8031092DB10F6
:1051F000EAECF3E0949108C08091C00085FFFCCFF9
:105200009093C600319694919923B1F7E0EDF3E0C5
:10521000949108C08091C00085FFFCCF9093C60098
:10522000319694919923B1F78091C00085FFFCCF0E
:105230008AE08093C600E0960FB6F894DEBF0FBEFA
:10524000CDBFCF91DF910895CF93DF93CAECD3E028
:10525000FE01949108C08091C00085FFFCCF90931F
:10526000C600319694919923B1F7E4ECF5E094915E
:1052700008C08091C00085FFFCCF9093C600319696
:1052800094919923B1F78091C00085FFFCCF8AE00B
:105290008093C600FE019491EAECF3E008C080918F
:1052A000C00085FFFCCF9093C6003196949199235E
:1052B000B1F74091D9085091DA086091DB087091FC
:1052C000DC088CEB95E00E94C2334091DD085091E0
:1052D000DE086091DF087091E00889EB95E00E949C
:1052E000C2334091E1085091E2086091E308709167
:1052F000E40886EB95E00E94C2334091E5085091A6
:10530000E6086091E7087091E80883EB95E00E9459
:10531000C233E6E1F2E007C08091C00085FFFCCF18
:1053200031969093C60090819923B1F78091C00087
:1053300085FFFCCF8AE08093C600FE019491EAECE1
:10534000F3E008C08091C00085FFFCCF9093C600B9
:10535000319694919923B1F7E9E9F5E0949108C069
:105360008091C00085FFFCCF9093C6003196949148
:105370009923B1F78091C00085FFFCCF8AE080932C
:10538000C600FE019491EAECF3E008C08091C000F1
:1053900085FFFCCF9093C600319694919923B1F785
:1053A0004091C9085091CA086091CB087091CC080F
:1053B00080E995E00E94C2334091CD085091CE081B
:1053C0006091CF087091D0088DE895E00E94C233BB
:1053D0004091D1085091D2086091D3087091D408BF
:1053E0008AE895E00E94C2334091D5085091D608D2
:1053F0006091D7087091D80887E895E00E94C23381
:10540000E6E1F2E007C08091C00085FFFCCF319655
:105410009093C60090819923B1F78091C00085FFD9
:10542000FCCF8AE08093C600FE019491EAECF3E0A1
:1054300008C08091C00085FFFCCF9093C6003196D4
:1054400094919923B1F7E9E6F5E0949108C0809131
:10545000C00085FFFCCF9093C600319694919923AC
:10546000B1F78091C00085FFFCCF8AE08093C60031
:10547000FE019491EAECF3E008C08091C00085FF42
:10548000FCCF9093C600319694919923B1F7409147
:10549000E9085091EA086091EB087091EC0880E609
:1054A00095E00E94D5334091ED085091EE0860914F
:1054B000EF087091F0088DE595E00E94D53340919A
:1054C000F1085091F2086091F3087091F4088AE5B0
:1054D00095E00E94D5334091F5085091F60860910F
:1054E000F7087091F80887E595E00E94D533E6E16A
:1054F000F2E007C08091C00085FFFCCF3196909309
:10550000C60090819923B1F78091C00085FFFCCF40
:105510008AE08093C600FE019491EAECF3E008C0B3
:105520008091C00085FFFCCF9093C6003196949186
:105530009923B1F7E2E2F5E0949108C08091C000B0
:1055400085FFFCCF9093C600319694919923B1F7D3
:105550008091C00085FFFCCF8AE08093C600FE01E9
:105560009491EAECF3E008C08091C00085FFFCCF85
:105570009093C600319694919923B1F74091FD081C
:105580005091FE086091FF087091000989E195E053
:105590000E94C233409101095091020960910309B0
:1055A0007091040986E195E00E94C233E6E1F2E0E1
:1055B00007C08091C00085FFFCCF31969093C60054
:1055C00090819923B1F78091C00085FFFCCF8AE0DC
:1055D0008093C600FE019491EAECF3E008C080914C
:1055E000C00085FFFCCF9093C6003196949199231B
:1055F000B1F7E3E6F4E0949108C08091C00085FF24
:10560000FCCF9093C600319694919923B1F7809185
:10561000C00085FFFCCF8AE08093C600FE01949114
:10562000EAECF3E008C08091C00085FFFCCF9093C6
:10563000C600319694919923B1F74091F9085091A1
:10564000FA086091FB087091FC088AE594E00E94DA
:10565000C233409111095091120960911309709160
:10566000140987E594E00E94C2334091C508509127
:10567000C6086091C7087091C80884E594E00E944C
:10568000D533409105095091060960910709709141
:10569000080981E594E00E94C233409109095091C4
:1056A0000A0960910B0970910C098EE494E00E9444
:1056B000C23340910D0950910E0960910F0970910C
:1056C00010098BE494E00E94C233E6E1F2E007C0E7
:1056D0008091C00085FFFCCF31969093C6009081E9
:1056E0009923B1F78091C00085FFFCCF8AE08093B9
:1056F000C600FE019491EAECF3E008C08091C0007E
:1057000085FFFCCF9093C600319694919923B1F711
:10571000E9E3F4E0949108C08091C00085FFFCCFDC
:105720009093C600319694919923B1F78091C0006F
:1057300085FFFCCF8AE08093C600FE019491EAECDD
:10574000F3E008C08091C00085FFFCCF9093C600B5
:10575000319694919923B1F740914C0650914D06A2
:1057600060914E0670914F0680E394E00E94C23330
:105770004091500650915106609152067091530627
:105780008DE294E0FFD74091540650915506609108
:105790005606709157068AE294E0F4D7E6E1F2E00B
:1057A00007C08091C00085FFFCCF31969093C60062
:1057B00090819923B1F78091C00085FFFCCF8AE0EA
:1057C0008093C600FE019491EAECF3E008C080915A
:1057D000C00085FFFCCF9093C60031969491992329
:1057E000B1F7ECE1F4E0949108C08091C00085FF2E
:1057F000FCCF9093C600319694919923B1F7809194
:10580000C00085FFFCCF8AE08093C600FE01949122
:10581000EAECF3E008C08091C00085FFFCCF9093D4
:10582000C600319694919923B1F740918403509129
:105830008503609186037091870382E194E0A2D78B
:10584000609188037091890380918A0390918B0302
:105850000E947B83AB01BC018FE094E093D7609101
:105860008C0370918D0380918E0390918F030E9421
:105870008783AB01BC018CE094E084D7E6E1F2E0E1
:1058800007C08091C00085FFFCCF31969093C60081
:1058900090819923B1F78091C00085FFFCCF8AE009
:1058A0008093C600DF91CF910895EF92FF921F93EE
:1058B000CF93DF93EC017B01142F888199810E94A3
:1058C000B7D1F70181937F018881998101969983EE
:1058D0008883115091F7DF91CF911F91FF90EF9046
:1058E0000895EF92FF920F931F93DF93CF93CDB75D
:1058F000DEB766970FB6F894DEBF0FBECDBF84E665
:1059000090E09A8389838091170290911802A09168
:105910001902B0911A028B8B9C8BAD8BBE8B8E01C2
:10592000015F1F4F7E010894E11CF11CC701B80103
:1059300044E0BBDFCE014396B80143E050E00E9453
:10594000DECA009709F0A6C0C70169ED78E040E122
:10595000ACDFC70169EC78E040E1A7DFC70169EE81
:1059600078E040E1A2DF0E942557C7016DEF78E0A3
:1059700044E09BDFC70161E079E044E096DFC701C6
:1059800069EF78E044E091DFC70161E179E044E04C
:105990008CDFC70165EC78E044E087DFC70165E094
:1059A00079E044E082DFC70169E079E044E07DDF2F
:1059B000C7016DE079E044E078DFC7016CE476E090
:1059C0004CE073DFC701BE016D5F7F4F42E06DDFCA
:1059D000C701BE016B5F7F4F42E067DFC701BE01B9
:1059E000695F7F4F42E061DFC701BE01675F7F4FA4
:1059F00042E05BDFC701BE01655F7F4F42E055DFDC
:105A0000C701BE01635F7F4F42E04FDFC70164E81B
:105A100073E044E04ADFC70168E873E044E045DF33
:105A2000C7016CE873E044E040DFC70169E773E059
:105A300046E03BDFC70168EA73E041E036DFC701BB
:105A40006BED70E141E031DF0E947D82EAECF3E032
:105A5000949108C08091C00085FFFCCF9093C60050
:105A6000319694919923B1F7E2EFF3E0949108C055
:105A70008091C00085FFFCCF9093C6003196949131
:105A80009923B1F78091C00085FFFCCF8AE0809315
:105A9000C60001C03BDAD8DB66960FB6F894DEBFCD
:105AA0000FBECDBFCF91DF911F910F91FF90EF906F
:105AB0000895EF92FF921F93CF93DF93EC017B0148
:105AC000142F88819981F70161917F010E94D2D1C1
:105AD00088819981019699838883115091F7DF918C
:105AE000CF911F91FF90EF900895EF92FF920F9347
:105AF0001F93DF93CF93CDB7DEB766970FB6F894B9
:105B0000DEBF0FBECDBF80911B0290911C02A09101
:105B10001D02B0911E028F87988BA98BBA8B84E6E9
:105B2000E82EF12CFA82E9828E010F5F1F4FC80127
:105B3000BE01615F7F4F44E0BCDFC80169ED78E0E2
:105B400040E1B7DFC80169EC78E040E1B2DFC801AD
:105B500069EE78E040E1ADDFC8016DEF78E044E048
:105B6000A8DFC80161E079E044E0A3DFC80169EF84
:105B700078E044E09EDFC80161E179E044E099DF2C
:105B8000C80165EC78E044E094DFC80165E079E0A5
:105B900044E08FDFC80169E079E044E08ADFC801B2
:105BA0006DE079E044E085DFC8016CE476E04CE02C
:105BB00080DF84EB90E09C838B8386E490E09E837F
:105BC0008D8318861F8280EF90E09A878987FC86F4
:105BD000EB861E861D86C801BE016D5F7F4F42E0C9
:105BE00068DFC801BE016B5F7F4F42E062DFC80122
:105BF000BE01695F7F4F42E05CDFC801BE01675FA5
:105C00007F4F42E056DFC801BE01655F7F4F42E033
:105C100050DFC801BE01635F7F4F42E04ADFC80129
:105C200064E873E044E045DFC80168E873E044E0FD
:105C300040DFC8016CE873E044E03BDFC80169E77E
:105C400073E046E036DFC80168EA73E041E031DF27
:105C5000C8016BED70E141E02CDF8091170290915B
:105C60001802A0911902B0911A028B8B9C8BAD8BFC
:105C7000BE8BFA82E982C801BE016D5E7F4F44E0AF
:105C800018DFEAECF3E0949108C08091C00085FF32
:105C9000FCCF9093C600319694919923B1F7E4ED2F
:105CA000F5E0949108C08091C00085FFFCCF9093EF
:105CB000C600319694919923B1F78091C00085FF79
:105CC000FCCF8AE08093C60066960FB6F894DEBFDC
:105CD0000FBECDBFCF91DF911F910F91FF90EF903D
:105CE0000895DF93CF930F920F92CDB7DEB7209137
:105CF000BB153091BC15CE0101962115310519F463
:105D0000875C954102C0821B930B9A8389838981AA
:105D10009A810F900F90CF91DF91089520E08091AC
:105D20003E0890913F08181619060CF421E0822FC6
:105D30000895AF92BF92CF92DF92EF92FF920F93AE
:105D40001F938C01000F111F000F111FF801E35169
:105D5000F84F6591759185919491F801E45BF94F45
:105D6000C080D180E280F3803CE3A32E36E0B32EE6
:105D7000A00EB11EA70196010E9452CBF5016083CF
:105D8000718382839383F801E750F84F6591759191
:105D90008591949128E5A22E26E0B22EA00EB11E88
:105DA000A70196010E9452CBF50160837183828323
:105DB0009383F801EB5FF74F65917591859194910D
:105DC000055B1C4FA70196010E9452CBF80160832E
:105DD0007183828393831F910F91FF90EF90DF90E7
:105DE000CF90BF90AF900895EF92FF920F931F93C3
:105DF000CF93DF93EC01E0905806F09059060091A4
:105E00005A0610915B06688179818A819B81A8017D
:105E100097010E942BCC882324F4E882F9820A831C
:105E20001B83E0905C06F0905D0600915E06109189
:105E30005F066C817D818E819F81A80197010E9400
:105E40002BCC882324F4EC82FD820E831F83E09008
:105E50006006F09061060091620610916306688505
:105E600079858A859B85A80197010E942BCC882380
:105E700024F4E886F9860A871B87E0904B03F090AC
:105E80004C0300914D0310914E03688179818A8102
:105E90009B81A80197010E942ECE181624F4E88257
:105EA000F9820A831B83E0904F03F0905003009126
:105EB0005103109152036C817D818E819F81A801D5
:105EC00097010E942ECE181624F4EC82FD820E83D8
:105ED0001F83E0905303F0905403009155031091F9
:105EE0005603688579858A859B85A80197010E945C
:105EF0002ECE181624F4E886F9860A871B87DF91D0
:105F0000CF911F910F91FF90EF90089580917506AA
:105F1000811181E00895809175060895CF93DF93F4
:105F20008130910541F46F5F7F4FF9F48CE394E089
:105F30000E94F0261AC0892BC1F46F5F7F4FA9F42D
:105F400085E096E00E94A31CC2ECD5E0CE010E9441
:105F5000A31C6F9784E0CC38D807C1F7CE010E940C
:105F6000A31CCE0181970E94A31CDF91CF910895BD
:105F700080E090E06FEF7FEFD1CF81E090E06FEFB6
:105F80007FEFCCCF1F93182F0E94668380917506F8
:105F9000882309F035C0109375068091770690919B
:105FA0007806A0917906B0917A0680937B0690934B
:105FB0007C06A0937D06B0937E06EAEEF5E0949110
:105FC00008C08091C00085FFFCCF9093C600319639
:105FD00094919923B1F7E1EFF5E0949108C0809195
:105FE000C00085FFFCCF9093C60031969491992311
:105FF000B1F78091C00085FFFCCF8AE08093C60096
:106000001F910895F8940E946683159A469A439AC0
:10601000409A8CE060E00E942C1BEAEEF5E094913F
:1060200008C08091C00085FFFCCF9093C6003196D8
:1060300094919923B1F7E7E6F6E0949108C0809136
:10604000C00085FFFCCF9093C600319694919923B0
:10605000B1F78091C00085FFFCCF8AE08093C60035
:10606000FFCF0E94DE1960937F06709380068093B5
:10607000810690938206E091A806F091A906E65564
:10608000F94F80818823A9F4E6E8F6E0949108C0EE
:106090008091C00085FFFCCF9093C600319694910B
:1060A0009923B1F78091C00085FFFCCF8AE08093EF
:1060B000C6000895EF92FF920F931F930E94DE197E
:1060C000E0908306F0908406009185061091860684
:1060D00020917F0630918006409181065091820682
:1060E000621B730B840B950BE616F706080719075E
:1060F00030F4E114F1040105110509F083DF80910A
:10610000680390916903A0916A03B0916B030097B3
:10611000A105B105F9F00E94DE1920917F063091AA
:1061200080064091810650918206621B730B840B9E
:10613000950B209168033091690340916A03509157
:106140006B03261737074807590720F48091050E7F
:106150008091060E069B02C08AE014DF0E94A659B9
:106160001F910F91FF90EF9008956F927F928F9201
:106170009F92AF92BF92CF92DF92EF92FF920F93D6
:106180001F93F82E6091870670918806809189068A
:1061900090918A0620918B0630918C0640918D0655
:1061A00050918E060E943BCE3B014C0100D000D0A6
:1061B0000DB71EB70F5F1F4F6091470370914803E3
:1061C000882777FD8095982F0E94CDCC20916C0375
:1061D00030916D0340916E0350916F030E9400CF88
:1061E00020E030E040E752E40E9432CC20E030E092
:1061F00048EC52E40E9432CC5B016C01F8016082F1
:10620000718282829382F4828091640685838CE31A
:1062100096E063E976E047E856E020E001E0E2E05E
:10622000EE2E0E9498538091930690919406A0912F
:106230009506B091960680933C0690933D06A093F8
:106240003E06B0933F068091970690919806A091E4
:106250009906B0919A068093400690934106A093C8
:106260004206B093430680919B0690919C06A091B4
:106270009D06B0919E068093440690934506A09398
:106280004606B093470680919F069091A006A09184
:10629000A106B091A2068093480690934906A09368
:1062A0004A06B0934B068DB79EB706960FB6F89484
:1062B0009EBF0FBE8DBF0E94DE1960937F06709354
:1062C000800680938106909382061F910F91FF9024
:1062D000EF90DF90CF90BF90AF909F908F907F9086
:1062E0006F900895CF92DF92EF92FF920F931F93DA
:1062F00083E996E079DD0E94DE1960937F06709352
:106300008006809381069093820660913C0670918E
:106310003D0680913E0690913F0620919306309174
:10632000940640919506509196060E942BCC8823A6
:1063300009F07AC060914006709141068091420652
:1063400090914306209197063091980640919906C6
:1063500050919A060E942BCC882309F065C0609169
:106360006C0370916D0380916E0390916F0320E038
:1063700030E040E752E40E9432CC7B018C0183E99B
:1063800096E067E976E04BE956E02FE936E0F4E67F
:10639000CF2EF6E0DF2E0E948C5C809193069091C8
:1063A0009406A0919506B091960680933C06909332
:1063B0003D06A0933E06B0933F06809197069091CC
:1063C0009806A0919906B0919A0680934006909302
:1063D0004106A0934206B093430680919B0690919C
:1063E0009C06A0919D06B0919E06809344069093D2
:1063F0004506A0934606B093470680919F0690916C
:10640000A006A091A106B091A206809348069093A1
:106410004906A0934A06B0934B061F910F91FF9037
:10642000EF90DF90CF9008956091470370914803FB
:10643000882777FD8095982F0E94CDCC20916C0302
:1064400030916D0340916E0350916F030E9400CF15
:1064500020E030E040E752E40E9432CC20E030E01F
:1064600048EC52E488CF84EC98E00E94D451E9E8EB
:10647000F6E0949108C08091C00085FFFCCF909316
:10648000C600319694919923B1F7409177065091C7
:1064900078066091790670917A064F5F5F4F6F4F73
:1064A0007F4F84EC98E02AE030E00E949052809187
:1064B000C00085FFFCCF8AE08093C600D2CD2F922A
:1064C0003F924F925F926F927F928F929F92AF9284
:1064D000BF92CF92DF92EF92FF920F931F93DF93C1
:1064E000CF9300D000D0CDB7DEB79E838D838330AD
:1064F000910508F010C15C01AA0CBB1CAA0CBB1CC6
:10650000C501845C994F9A83898380E090E0A0E084
:10651000B0E0E981FA8180839183A283B3838CE325
:1065200096E060E476E044E456E028E436E00E9439
:106530007757F501EF5EF74F6591759185919491CD
:10654000ED81FE81E75DF74FD490B3E92B2EB6E0E5
:106550003B2E2A0C3B1C20E030E040EC5FE30E9425
:1065600000CF7B018C016D2D772767FD7095872FFC
:10657000972F0E94CDCC2B013C01C801B701A3018C
:1065800092010E9400CFD1016D937D938D939C93D6
:106590001397F501E95CFC4FFC83EB83608171810B
:1065A0008281938160936C0370936D0380936E037B
:1065B00090936F0320E030E040E752E40E9432CC39
:1065C0007B018C0183E996E067E976E04BE956E0D0
:1065D0002FE936E0A4E6CA2EA6E0DA2E0E948C5CF3
:1065E0000E94667B80E090E0A0E0B0E0E981FA8163
:1065F00080839183A283B3838CE396E060E476E0AA
:1066000044E456E028E436E00E9477578DE198E0B4
:10661000A80EB91EF50185909590A590B490C5017E
:10662000B4019058A30192010E9400CFD1016D9353
:106630007D938D939C93139760916C0370916D0380
:1066400080916E0390916F0320E030E040E752E4C8
:106650000E9432CC7B018C0183E996E067E976E009
:106660004BE956E02FE936E00E948C5C0E94667B85
:10667000C501B401A50194010E9452CBA30192016E
:106680000E9400CFF1016083718382839383AB8189
:10669000BC816D917D918D919C9120E030E040E432
:1066A00050E40E9432CC60936C0370936D0380932E
:1066B0006E0390936F0320E030E040E752E40E94C5
:1066C00032CC7B018C0183E996E067E976E04BE907
:1066D00056E02FE936E00E948C5C0E94667B8D813B
:1066E0009E8127DBE981FA8180819181A281B3813A
:1066F000F10180839183A283B38380E090E0A0E0E6
:10670000B0E080936C0390936D03A0936E03B093FD
:106710006F030E94F57926960FB6F894DEBF0FBE80
:10672000CDBFCF91DF911F910F91FF90EF90DF9040
:10673000CF90BF90AF909F908F907F906F905F9021
:106740004F903F902F900895682F2091A806309188
:10675000A90680E690E0AC01249FC001259F900D22
:10676000349F900D11248C54994F70E00E94CCCA34
:106770009C019093B3068093B20680E0232B09F02E
:1067800081E00895FC01949108C08091C00085FFCC
:10679000FCCF9093C600319694919923B1F784EC85
:1067A00098E022E030E00C949653FC01949108C0EC
:1067B0008091C00085FFFCCF9093C60031969491E4
:1067C0009923B1F784EC98E02AE030E00C947452FD
:1067D0008091B2069091B306019660E070E04AE0C5
:1067E00050E00C94EBC88091B2069091B3060196EC
:1067F00060E070E00C9485C7CF93DF93EC0180914B
:1068000064068093760684E59FDF882309F46EC0D2
:10681000EADF0E949FCC262F60937606662309F458
:1068200065C0E4EEF5E0949108C08091C00085FF5A
:10683000FCCF9093C600319694919923B1F7C93655
:10684000D10599F0CA36D10524F4C836D105F1F541
:106850000FC0CD36D10531F0CA3DD105B9F5EFE114
:10686000F2E031C0E6E3F2E023C0EDE4F2E015C06F
:10687000E4E6F2E007C08091C00085FFFCCF3196CE
:106880009093C60090819923B1F720C08091C000F9
:1068900085FFFCCF31969093C60090819923B1F784
:1068A00015C08091C00085FFFCCF31969093C60043
:1068B00090819923B1F70AC08091C00085FFFCCF79
:1068C00031969093C60090819923B1F784EC98E0BB
:1068D000622F40E050E00E947F528091C00085FF0F
:1068E000FCCF8AE08093C60081E001C080E0DF91A8
:1068F000CF9108955F926F927F928F929F92AF9205
:10690000BF92CF92DF92EF92FF920F931F93DF938C
:10691000CF9300D00F92CDB7DEB719821A821B82B7
:106920001C828CE3C82E86E0D82E03E9E02E06E018
:10693000F02E00E010E03E010894611C711C55240B
:106940005394F801EC51FC4F8081FEDE882359F10D
:106950004ADF4B015C01F801EA5CF94F8081882332
:1069600011F061E002C06091A30670E0882777FD16
:106970008095982F0E94CDCCF601208131814281F3
:1069800053810E9400CF9B01AC01C501B4010E945C
:1069900052CBF7016083718382839383F301E00F0D
:1069A000F11F50820AC0F60180819181A281B381DA
:1069B000F70180839183A283B3830F5F1F4F84E02D
:1069C00090E0C80ED91EE80EF91E0430110509F03A
:1069D000B8CF86E4B9DE8823D9F005DF7B018C01CE
:1069E0006093A4067093A5068093A6069093A706CD
:1069F00020E030E040E050E00E942ECE181644F433
:106A0000E0926C03F0926D0300936E0310936F039A
:106A100080916606882309F4C1C08981882309F022
:106A2000BDC08A81882309F0B9C08B81882309F011
:106A3000B5C08C81882309F4B1C0A0904806B090FD
:106A40004906C0904A06D0904B0660919F0670910F
:106A5000A0068091A1069091A206A60195010E9430
:106A600051CB7B018C012DEC3CEC4CEC5DEB0E949E
:106A70002BCC88230CF04EC080916706882309F048
:106A80008DC060919B0670919C0680919D069091AF
:106A90009E06209160033091610340916203509102
:106AA00063030E9452CB60939B0670939C06809375
:106AB0009D0690939E06C801B701905820915803F7
:106AC0003091590340915A0350915B030E9451CB7E
:106AD0009B01AC01C601B5010E9451CB60934806F1
:106AE0007093490680934A0690934B0680915C030D
:106AF00090915D03A0915E03B0915F0380936C035E
:106B000090936D03A0936E03B0936F0381E0809325
:106B1000670644C0C801B7012DEC3CEC4CEC5DE3CA
:106B20000E942ECE1816D4F5809167068823B1F105
:106B3000609158037091590380915A0390915B03BF
:106B4000A80197010E9451CB2091680630916906F7
:106B500040916A0650916B060E9452CB9B01AC019A
:106B6000C601B5010E9452CB609348067093490656
:106B700080934A0690934B0680916403909165033D
:106B8000A0916603B091670380936C0390936D03AB
:106B9000A0936E03B0936F03109267060F900F904F
:106BA0000F900F90CF91DF911F910F91FF90EF9079
:106BB000DF90CF90BF90AF909F908F907F906F901D
:106BC0005F90089597DE89E4BFDD882351F00BDEE6
:106BD00060938706709388068093890690938A064F
:106BE0000CC080E090E0A0E0B0E080938706909336
:106BF0008806A0938906B0938A068AE4A5DD8823D7
:106C000051F0F1DD60938B0670938C0680938D06B6
:106C100090938E06089580E090E0A0E0B0E080932D
:106C20008B0690938C06A0938D06B0938E060895E4
:106C30002F923F924F925F926F927F928F929F928C
:106C4000AF92BF92CF92DF92EF92FF920F931F937A
:106C5000DF93CF93CDB7DEB76E970FB6F894DEBF54
:106C60000FBECDBF10926C0687E46EDD882309F459
:106C700035C5B9DD0E949ACC6A30710509F48BC024
:106C80006B3071059CF46230710599F163307105C8
:106C900024F4772334F50C940D4A6330710581F1A7
:106CA0006430710511F00C940D4A33C06A357105DA
:106CB00009F4C3C46B35710554F46B30710509F4E4
:106CC000F0C06C31710511F00C940D4A4FC16B3559
:106CD000710509F4B6C46C35710511F00C940D4AB8
:106CE000B5C480917506882321F404DEFBDA0C9488
:106CF0002E4A80917506882319F464DF81E006C06E
:106D000080917506882329F45DDF80E02EDA0C94EB
:106D10002E4A80E519DD882321F4EE24FF24870123
:106D200005C061DD0E949FCC7B018C0183E50CDDF9
:106D3000882359F058DD20E030E04AE754E40E940F
:106D400000CF0E949FCC7B018C010E94667B0E9439
:106D5000DE195B016C01AE0CBF1CC01ED11E0E946F
:106D6000DE1960937F06709380068093810690936E
:106D7000820681E080936C0605C00E9482879AD9C2
:106D80000E94D0900E94DE196A157B058C059D0536
:106D9000A0F30C940D4A80916706882311F00C949F
:106DA0000D4A80913C0690913D06A0913E06B0911F
:106DB0003F068093930690939406A0939506B09314
:106DC00096068091400690914106A0914206B091AE
:106DD00043068093970690939806A0939906B093E4
:106DE0009A068091440690914506A0914606B0917E
:106DF000470680939B0690939C06A0939D06B093B4
:106E00009E06609158037091590380915A039091A6
:106E10005B03209171033091720340917303509191
:106E200074030E9432CC9B01AC01609148067091C2
:106E3000490680914A0690914B060E9451CB9B01D6
:106E4000AC0160939F067093A0068093A106909377
:106E5000A206609148067091490680914A06909179
:106E60004B060E9451CB609368067093690680932D
:106E70006A0690936B0680915C0390915D03A091EC
:106E80005E03B0915F0380936C0390936D03A093B6
:106E90006E03B0936F0381E08093670623DA0C944E
:106EA0000D4A80916706882311F40C940D4A809155
:106EB0003C0690913D06A0913E06B0913F0680931E
:106EC000930690939406A0939506B09396068091AE
:106ED000400690914106A0914206B09143068093EE
:106EE000970690939806A0939906B0939A0680917E
:106EF000440690914506A0914606B09147068093BE
:106F00009B0690939C06A0939D06B0939E0660916D
:106F100048067091490680914A0690914B0620914F
:106F200068063091690640916A0650916B060E948E
:106F300052CB60939F067093A0068093A106909316
:106F4000A2068091640390916503A0916603B091BD
:106F5000670380936C0390936D03A0936E03B093CB
:106F60006F0310926706BED90C940D4A85E080939A
:106F70006C0680916C0390916D03A0916E03B091AB
:106F80006F038093AE069093AF06A093B006B093C4
:106F9000B106809147039091480390933B068093FC
:106FA0003A0684E690E090934803809347030E945A
:106FB000DE1960937F06709380068093810690931C
:106FC000820681E00E94FC7980913C0690913D060A
:106FD000A0913E06B0913F0680939306909394064D
:106FE000A0939506B0939606809140069091410635
:106FF000A0914206B091430680939706909398061D
:10700000A0939906B0939A06809144069091450604
:10701000A0914606B091470680939B0690939C06EC
:10702000A0939D06B0939E068091480690914906D4
:10703000A0914A06B0914B0680939F069093A006BC
:10704000A093A106B093A20680E090E0A0E0B0E09B
:1070500080936C0390936D03A0936E03B0936F03C2
:1070600088E572DB882351F489E56EDB882331F4EF
:107070008AE56ADB882311F481E001C080E0809317
:107080007003882309F416C10F2EF0E08F2EF0E074
:107090009F2EF0E0AF2EF0E0BF2EF02D80923C0648
:1070A00090923D06A0923E06B0923F068092400626
:1070B00090924106A0924206B09243068092440606
:1070C00090924506A0924606B09247068CE396E061
:1070D00060E476E044E456E028E436E00E94775726
:1070E00080E090E8ACEAB3EC80939306909394062A
:1070F000A0939506B093960680E090ECA8EAB3E4DE
:107100008093970690939806A0939906B0939A0659
:1071100080E090E8ACEAB3E480939B0690939C06F1
:10712000A0939D06B0939E0660913703709138033B
:107130008091390390913A0360936C0370936D03CF
:1071400080936E0390936F0320E030E040E752E4B9
:107150000E9432CC7B018C0183E996E067E976E0FE
:107160004BE956E02FE936E0F4E6CF2EF6E0DF2ECD
:107170000E948C5C0E94667B0E94F57980E090E022
:107180000E94992E81E090E00E94992E82E090E08A
:107190000E94992E8CE396E060E476E044E456E0A9
:1071A00028E436E00E94775780913C0690913D0696
:1071B000A0913E06B0913F0680939306909394066B
:1071C000A0939506B0939606809140069091410653
:1071D000A0914206B091430680939706909398063B
:1071E000A0939906B0939A06809144069091450623
:1071F000A0914606B091470680939B0690939C060B
:10720000A0939D06B0939E0660916C0370916D03F0
:1072100080916E0390916F0320E030E040E752E4EC
:107220000E9432CC7B018C0183E996E067E976E02D
:107230004BE956E02FE936E00E948C5C80926C03AB
:1072400090926D03A0926E03B0926F030E94667BD2
:107250000E94F5798091930690919406A0919506ED
:10726000B091960680933C0690933D06A0933E060F
:10727000B0933F068091970690919806A091990649
:10728000B0919A068093400690934106A0934206DF
:10729000B093430680919B0690919C06A0919D0619
:1072A000B0919E068093440690934506A0934606AF
:1072B000B093470680917003882321F48AE544DA6D
:1072C000882319F082E090E0FAD880917003882337
:1072D00051F488E539DA882309F40DC189E534DAF7
:1072E000882309F408C180E090E0A0E0B0E080933A
:1072F0003C0690933D06A0933E06B0933F068093D4
:10730000400690934106A0934206B09343068CE357
:1073100096E060E476E044E456E028E436E00E943B
:10732000775780E090E8ACEAB3EC809393069093B3
:107330009406A0939506B093960680E090ECA8EA98
:10734000B3E48093970690939806A0939906B09320
:107350009A062091370330913803409139035091B8
:107360003A0320936C0330936D0340936E03509364
:107370006F03E0903B03F0903C0300913D031091BC
:107380003E03C801B7010E942BCC882344F4E0924D
:107390006C03F0926D0300936E0310936F03609182
:1073A0006C0370916D0380916E0390916F0320E0E8
:1073B00030E040E752E40E9432CC7B018C0183E94B
:1073C00096E067E976E04BE956E02FE936E0E4E63F
:1073D000CE2EE6E0DE2E0E948C5C0E94667B80E072
:1073E00090E00E94992E81E090E00E94992E8CE31B
:1073F00096E060E476E044E456E028E436E00E945B
:10740000775780913C0690913D06A0913E06B09141
:107410003F068093930690939406A0939506B093AD
:1074200096068091400690914106A0914206B09147
:1074300043068093970690939806A0939906B0937D
:107440009A0660916C0370916D0380916E03909128
:107450006F0320E030E040E752E40E9432CC7B0131
:107460008C0183E996E067E976E04BE956E02FE985
:1074700036E00E948C5C80E090E0A0E0B0E0809379
:107480006C0390936D03A0936E03B0936F030E94FF
:10749000667B0E94F5798091930690919406A09165
:1074A0009506B091960680933C0690933D06A09376
:1074B0003E06B0933F068091970690919806A09162
:1074C0009906B0919A068093400690934106A09346
:1074D0004206B093430680919B0690919C06A09132
:1074E0009D06B0919E068093440690934506A09316
:1074F0004606B093470680917003882321F488E5FF
:1075000023D9882321F080E090E00E945F328091AF
:107510007003882321F489E517D9882321F081E0BD
:1075200090E00E945F3288E50FD98823C9F050D9D6
:10753000611571058105910599F055D920914C0689
:1075400030914D0640914E0650914F060E9452CB0D
:1075500060933C0670933D0680933E0690933F06F1
:1075600089E5F2D88823C9F033D961157105810501
:10757000910599F038D920915006309151064091EB
:107580005206509153060E9452CB6093400670936E
:10759000410680934206909343068AE5D5D8882316
:1075A000C9F016D9611571058105910599F01BD9AE
:1075B0002091540630915506409156065091570639
:1075C0000E9452CB60934406709345068093460612
:1075D000909347068CE396E060E476E044E456E05E
:1075E00028E436E00E94775780E00E94FC79809181
:1075F000AE069091AF06A091B006B091B10680930F
:107600006C0390936D03A0936E03B0936F0380910E
:107610003A0690913B0690934803809347030E945B
:10762000DE1960937F0670938006809381069093A5
:1076300082060E94F5790C940D4A1092A3060C94D0
:107640000D4A81E08093A3060C940D4A85E47CD812
:10765000882311F40E94667B4CE3E42E46E0F42E6E
:107660003CE4C32E36E0D32E00E010E0F801EC51EC
:10767000FC4F808169D8882321F1033059F4B3D8B5
:10768000F701608371838283938388E496E00E948C
:10769000505717C0A8D8F60120813181428153810B
:1076A0000E9452CBF70160837183828393838CE3C2
:1076B00096E060E476E044E456E028E436E00E9498
:1076C00077570F5F1F4F24E030E0E20EF31EC20E2B
:1076D000D31E0430110551F60C940D4A8DE434D8B4
:1076E000882311F40C942F497ED80E949ACC6337DA
:1076F000710511F40C94E443643771050CF08DC0EE
:107700006A32710509F44AC36B3271050CF040C04E
:107710006831710509F495C169317105D4F464319A
:10772000710509F437C16531710554F46131710592
:1077300009F42AC16231710511F00C940D4A5DC73C
:107740006631710509F45CC1673171050CF05EC1E9
:1077500051C16B31710509F4AFC16C31710554F43D
:107760006931710509F47DC16A31710511F00C941C
:107770000D4A7DC16E31710509F4E0C16F317105AB
:1077800009F48BC26C31710511F00C940D4A9AC149
:107790006C35710509F493C76D357105FCF46235DC
:1077A000710509F423C76335710554F4603571051B
:1077B00009F416C76135710511F00C940D4A13C711
:1077C0006435710509F419C7643571050CF411C7E6
:1077D0006535710511F00C940D4A58C76A3671056C
:1077E00009F484C66B36710554F46836710509F4E2
:1077F0001DC36936710511F00C940D4A48C36D36EE
:10780000710509F416C46237710509F4FCC76B36BB
:10781000710511F00C940D4AE0C6613D710511F43B
:107820000C94B146623D71050CF049C0693C71058C
:1078300011F40C9486456A3C71050CF568377105A6
:1078400011F40C94F7446937710554F465377105E8
:1078500009F4C9C76737710511F00C940D4A90C03F
:107860006C38710509F402C36E3B710509F474C5E7
:107870006937710511F00C940D4A0C94FB446D3C72
:10788000710511F40C94E6456E3C710564F46B3C93
:10789000710511F40C94A8456C3C710511F00C9421
:1078A0000D4A0C94C6456F3C710511F40C94624668
:1078B000603D710514F00C9491460C94444631E0FF
:1078C0006039730711F40C940B4941E06139740776
:1078D0004CF551E06D32750711F40C94364781E098
:1078E0006E32780764F46C3D710511F40C941847FE
:1078F0006D3D710511F00C940D4A0C94274791E0F1
:107900006F32790711F40C94CB48E1E06F327E07B7
:1079100014F40C94BC486053714011F00C940D4A5F
:107920000C940E4821E0673F720711F40C9417493C
:1079300031E0683F73079CF441E0653F740711F440
:107940000C94114951E0663F750714F00C941449EA
:10795000645F714011F00C940D4A0C940E4993E051
:10796000603A790709F45EC1E3E0673E7E0711F4EF
:107970000C941A496B59734011F00C940D4A29C1AB
:10798000EBE7F2E00C94064515984698439840982A
:107990000C940D4AEDEDF7E0949108C08091C00081
:1079A00085FFFCCF9093C600319694919923B1F74F
:1079B0008091C00085FFFCCF8AE08093C6008CE3F5
:1079C00094E00E94A426EFECF7E0949108C0809127
:1079D000C00085FFFCCF9093C60031969491992307
:1079E000B1F78091C00085FFFCCF8AE08093C6008C
:1079F0000C940D4A8CE394E00E9436220C940D4ABC
:107A00008CE394E00E94251C0C940D4A8091B206F0
:107A10009091B30604966AE270E00E94CCCAFC0121
:107A2000009711F0319710826091B2067091B30601
:107A30006C5F7F4F8CE394E041E00E94A31E0C94A6
:107A40000D4A8CE394E00E94291C0E94DE19609389
:107A50006D0670936E0680936F06909370060C947B
:107A60000D4A8CE394E00E94301C0C940D4A8091E6
:107A70006A04882311F40C940D4A8091E30588234D
:107A800011F00C940D4A83E50E94A433882311F46D
:107A90000C940D4A0E94E833AB01BC0140932C06C4
:107AA00050932D0680932E0670932F0689E096E062
:107AB0000E94E76B0C940D4A8CE394E00E94261E12
:107AC0000C940D4A8091B2069091B30604966AE236
:107AD00070E00E94CCCA8C01009719F12091A80691
:107AE0003091A90680E690E0AC01249FC001259F5B
:107AF000900D349F900D11248C54994F6EE470E0DA
:107B00000E94CCCA60E270E00E94CCCA9C012F5F48
:107B10003F4F3093B3062093B20601501040F80156
:107B200010826091B2067091B3066C5F7F4F8CE358
:107B300094E040E00E94A31E0C940D4A80916A04D8
:107B4000882311F40C940D4A8091E305882311F0E9
:107B50000C940D4A8CE394E00E94951D8091B2062E
:107B60009091B30604966AE270E00E94CCCA8C0140
:107B7000009719F12091A8063091A90680E690E0BF
:107B8000AC01249FC001259F900D349F900D1124BE
:107B90008C54994F6EE470E00E94CCCA60E270E0B1
:107BA0000E94CCCA9C012F5F3F4F3093B3062093B5
:107BB000B20601501040F80110826091B206709137
:107BC000B3066C5F7F4F8CE394E00E94C5200C9459
:107BD0000D4A8091B2069091B30604966AE270E075
:107BE0000E94CCCAFC01009711F03197108260917D
:107BF000B2067091B3066C5F7F4F8CE394E041E076
:107C00000E94A31E8CE394E00E94291C0E94DE19AE
:107C100060936D0670936E0680936F069093700666
:107C20000C940D4A8091B2069091B30605966AE2D3
:107C300070E00E94CCCA8C01009719F12091A8062F
:107C40003091A90680E690E0AC01249FC001259FF9
:107C5000900D349F900D11248C54994F6EE470E078
:107C60000E94CCCA60E270E00E94CCCA9C012F5FE7
:107C70003F4F3093B3062093B20601501040F801F5
:107C800010826091B2067091B3066B5F7F4F8CE3F8
:107C900094E00E94BF200C940D4A0E94DE1960936C
:107CA0007106709372068093730690937406209108
:107CB0006D0630916E0640916F0650917006621B02
:107CC000730B840B950B28EE33E040E050E00E94EC
:107CD000F5D2F22EE32ED42EC52E2DB73EB7285066
:107CE00030400FB6F8943EBF0FBE2DBF0DB71EB784
:107CF0000F5F1F4FCE010196EDB7FEB792838183D0
:107D000080EC97E0F801938382836F2D7E2D842F82
:107D1000952F2CE330E040E050E00E94F5D2F801CE
:107D2000358324836F2D7E2D8D2D9C2D2CE330E00B
:107D300040E050E00E94F5D2F801778366830E940C
:107D400021CBE4EEF5E094912DB73EB7285F3F4F8D
:107D50000FB6F8943EBF0FBE2DBF08C08091C00083
:107D600085FFFCCF9093C600319694919923B1F78B
:107D7000FE01319607C08091C00085FFFCCF31968F
:107D80009093C60090819923B1F78091C00085FF40
:107D9000FCCF8AE08093C6000C940D4A83E50E94D4
:107DA000A433882311F40C940D4A0E94F3330E94EB
:107DB0009ACC7B018C016B0180E50E94A43388235F
:107DC00069F0F7FC0BC03FEFE316F10409F034F45F
:107DD0000E94F3330E949ACC8B0102C008E010E0AD
:107DE000E8EEF3E0808191818017910711F40C9403
:107DF0000D4A329644E0E835F407A1F70730110543
:107E000019F4C092650604C017FF02C00C940D4A15
:107E1000802F61E00E942C1B802F6C2D0E94DF1BA5
:107E2000802FB6010E944E1A0C940D4A88E690E00D
:107E30000E94FC33882311F00C940D4A83E50E94C4
:107E4000A433882379F00E94F33320917606022F21
:107E500010E0000F111F00591F4E0E949ACCF8012C
:107E6000718360830E9465830C940D4A83E50E94B0
:107E7000A433882311F40C940D4A0E94F3330E941A
:107E80009ACC70937310609372100C940D4A89E62B
:107E900090E00E94FC33882311F00C940D4AEAEB29
:107EA000F7E0949108C08091C00085FFFCCF9093CB
:107EB000C600319694919923B1F7E0917606F0E0EF
:107EC000EE0FFF1FEE0FFF1FEA58FF4E408151815A
:107ED0006281738184EC98E021E030E00E94965347
:107EE000E7EBF7E0949108C08091C00085FFFCCFDC
:107EF0009093C600319694919923B1F7E09176065C
:107F0000F0E0EE0FFF1FE059FF4E6081718188277E
:107F100077FD8095982F0E94CDCCAB01BC0184ECFD
:107F200098E021E030E00E949653E3EBF7E0949173
:107F300008C08091C00085FFFCCF9093C6003196A9
:107F400094919923B1F740917C1050917D106091EC
:107F50007E1070917F1084EC98E021E030E00E9468
:107F60009653E0EBF7E0949108C08091C00085FF44
:107F7000FCCF9093C600319694919923B1F760910C
:107F8000721070917310882777FD8095982F0E944A
:107F9000CDCCAB01BC0184EC98E021E030E00E9444
:107FA0009653ECEAF7E0949108C08091C00085FFF9
:107FB000FCCF9093C600319694919923B1F78091AC
:107FC00076060E94AA82BC0184EC98E04AE050E068
:107FD0000E94C352E7EAF7E0949108C08091C00084
:107FE00085FFFCCF9093C600319694919923B1F709
:107FF0008FEF9FEF0E94AA82BC0184EC98E04AE0D8
:1080000050E00E94C352E4E9F2E007C08091C00052
:1080100085FFFCCF31969093C60090819923B1F7EC
:108020008091C00085FFFCCF8AE08093C6000C944D
:108030002E4A8DE690E00E94FC33882311F00C94C8
:108040000D4A83E080936C0683E50E94A433882365
:1080500079F00E94F33320917606022F10E0000F92
:10806000111F00591F4E0E949ACCF8017183608342
:108070000E9465830E94DE194B015C012091760607
:10808000022F10E07724000F111FF801E059FF4E76
:1080900060817181882777FD8095982F0E94CDCCD3
:1080A000000F111F0A581F4EF801208131814281B3
:1080B00053810E942ECE181614F477247394CC2486
:1080C000CA94DC2C7601E4EAF7E04490E0EAF7E0B9
:1080D0005490ECE9F7E064905AE0352E30C1942DCD
:1080E000E4EAF7E008C08091C00085FFFCCF9093E0
:1080F000C600319694919923B1F7E0917606F0E0AD
:10810000EE0FFF1FEE0FFF1FEA58FF4E4081518117
:108110006281738184EC98E021E030E00E94965304
:10812000952DE0EAF7E008C08091C00085FFFCCF04
:108130009093C600319694919923B1F76091760699
:1081400084EC98E070E04AE050E00E94C352962D23
:10815000ECE9F7E008C08091C00085FFFCCF909368
:10816000C600319694919923B1F7F7FE03C0E5E973
:10817000F2E028C00E94DE19A70196012854344F6E
:108180004F4F5F4F261B370B480B590BCA01B901E4
:1081900028EE33E040E050E00E94F5D284EC98E015
:1081A000BA01A9012AE030E00E9474528091C00017
:1081B00085FFFCCF0EC08091C00085FFFCCF3196BB
:1081C0009093C60090819923B1F78091C00085FFFC
:1081D000FCCF3092C6000E94DE194B015C010E9468
:1081E00082870E945A300E94D090FFEFCF16FFEF97
:1081F000DF06FFEFEF06FFEFFF0609F050C0E0914A
:108200007606772031F1F0E08F01000F111F000F8B
:10821000111F0A581F4EEE0FFF1FE059FF4E6081DD
:108220007181882777FD8095982F0E94CDCC20E022
:1082300030E040E050E40E9451CB9B01AC01F801DA
:1082400060817181828193810E942ECE87FF5AC006
:1082500060C0F0E08F01000F111F000F111F0A58BE
:108260001F4EEE0FFF1FE059FF4E6081718188277E
:1082700077FD8095982F0E94CDCC20E030E040E043
:1082800050E40E9452CB9B01AC01F80160817181E6
:10829000828193810E942BCC1816A4F53AC0F7FC7A
:1082A00038C0E0917606F0E08F01000F111F000F3B
:1082B000111F0A581F4EEE0FFF1FE059FF4E60813D
:1082C0007181882777FD8095982F0E94CDCC9B01E6
:1082D000AC01F80160817181828193810E9451CB50
:1082E0000E949ACC97FF07C09095809570956195F4
:1082F0007F4F8F4F9F4F64307105810591054CF082
:10830000772039F40E94DE19AC01CB01DA016C014F
:108310007D01FFEFCF16FFEFDF06FFEFEF06FFEF68
:10832000FF0669F0F7FE02C00C94104A0E94DE19A5
:108330006C197D09685B7B4010F00C94104A0E9418
:10834000DE19681979098A099B09695E73408040C2
:10835000904008F0C4CE43CF84E080936C0683E560
:108360000E94A433882341F00E94F3330E949ACCE8
:1083700070937310609372100E94DE195B016C01A0
:10838000E9E9F7E07490E5E9F7E08490E1E9F7E0E6
:108390009490EAE06E2E7DC00E94DE196A197B0976
:1083A0008C099D09695E73408040904008F46BC061
:1083B000E0916406F0E0EE0FFF1FEE0FFF1FEA589A
:1083C000FF4E4081518162817381972DE9E9F7E089
:1083D00008C08091C00085FFFCCF9093C600319605
:1083E00094919923B1F784EC98E022E030E00E9468
:1083F0009653982DE5E9F7E008C08091C00085FF0D
:10840000FCCF9093C600319694919923B1F7609177
:10841000640684EC98E070E04AE050E00E94C352A9
:10842000992DE1E9F7E008C08091C00085FFFCCFFD
:108430009093C600319694919923B1F740917C10A6
:1084400050917D1060917E1070917F1084EC98E0C7
:1084500021E030E00E949653E4E9F2E007C0809109
:10846000C00085FFFCCF31969093C6009081992380
:10847000B1F78091C00085FFFCCF6092C6000E94DA
:10848000DE195B016C010E9482870E945A300E94B3
:10849000D0906091721070917310882777FD80954D
:1084A000982F0E94CDCC7B018C0160917C10709143
:1084B0007D1080917E1090917F1020E030E040E0B0
:1084C00050E40E9451CB9B01AC01C801B7010E944E
:1084D0002BCC87FD61CF0E94DE1960937F067093DD
:1084E0008006809381069093820697C783E50E9459
:1084F000A433882309F464C00E94F3337B018C0108
:108500006091570370E0882777FD8095982F0E942F
:10851000CDCC9B01AC01C801B7010E9400CF20E087
:1085200030E048EC52E40E9432CC20E030E040E001
:1085300050E00E942BCC882314F460E03EC00E94DF
:10854000F3337B018C016091570370E0882777FD3E
:108550008095982F0E94CDCC9B01AC01C801B7013A
:108560000E9400CF20E030E048EC52E40E9432CC80
:1085700020E030E04FE753E40E942ECE181614F4AA
:108580006FEF1BC00E94F3337B018C016091570396
:1085900070E0882777FD8095982F0E94CDCC9B01B5
:1085A000AC01C801B7010E9400CF20E030E048ECE8
:1085B00052E40E9432CC0E949FCC609365062DC786
:1085C000809157039FEF899FC001112464E670E0FA
:1085D0000E94E2D26093650620C7109265061DC70F
:1085E000269A2E981AC7269A2E9A17C710923906DD
:1085F00014C781E08093390610C783E50E94A43335
:10860000882399F00E94F33320E030E04AE754E4F5
:108610000E9400CF0E949FCC60936803709369030F
:1086200080936A0390936B03F8C688E50E94A43395
:10863000882309F00AC789E50E94A433882309F03A
:1086400004C78AE50E94A433882309F0FEC685E4A6
:108650000E94A433882309F0F8C60E94667B409AE2
:108660000E94747BDAC6159A89E50E94A4338111B1
:10867000469A8AE50E94A4338111439A85E40E94B8
:10868000A433882309F4C9C6409AC7C683E50E946B
:10869000A433882309F4C1C60E94F33320E030E0FC
:1086A0004AE754E40E9400CF0E949FCC6093830667
:1086B000709384068093850690938606AEC669ED16
:1086C000662E68E0762E59EC252E58E0352E45E1D1
:1086D000442E49E0542E88249924F401EC51FC4F97
:1086E00080810E94A433882309F45DC053E085167D
:1086F00009F052C00E94F3335B016C0120E030E0CE
:1087000040EA51E40E942BCC88230CF03FC0F301D7
:108710006081718182819381A60195010E9432CC92
:108720007B018C0160910D0970910E0980910F09F8
:1087300090911009A80197010E9400CF60930D0944
:1087400070930E0980930F0990931009F1016081D5
:10875000718182819381A80197010E9400CFF1016C
:108760006083718382839383F2016081718182814E
:1087700093810E94CBCCA80197010E9400CF0E9458
:108780009FCCF2016083718382839383F301A08283
:10879000B182C282D38207C00E94F333F3016083A7
:1087A0007183828393830894811C911C24E030E0C0
:1087B000620E731E220E331E420E531E34E08316C9
:1087C000910409F08ACF29C6E1EFF6E0949108C040
:1087D0008091C00085FFFCCF9093C60031969491A4
:1087E0009923B1F71AC68091B2069091B306059607
:1087F0006AE270E00E94CCCAFC01009709F40DC641
:10880000319710820AC6EEEEF6E0949108C080918E
:10881000C00085FFFCCF9093C600319694919923B8
:10882000B1F740913C0650913D0660913E06709133
:108830003F0684EC98E022E030E00E949653EBEE95
:10884000F6E0949108C08091C00085FFFCCF909322
:10885000C600319694919923B1F74091400650910A
:108860004106609142067091430684EC98E022E054
:1088700030E00E949653E8EEF6E0949108C08091B3
:10888000C00085FFFCCF9093C60031969491992348
:10889000B1F74091440650914506609146067091AB
:1088A000470684EC98E022E030E00E949653E5EE23
:1088B000F6E0949108C08091C00085FFFCCF9093B2
:1088C000C600319694919923B1F740914806509192
:1088D000490660914A0670914B0684EC98E022E0CC
:1088E00030E00E949653EAEDF6E0949108C0809142
:1088F000C00085FFFCCF9093C600319694919923D8
:10890000B1F780E00E94507A0E94CDCC2091D90826
:108910003091DA084091DB085091DC080E9432CC9B
:10892000AB01BC0184EC98E022E030E00E94965359
:10893000E7EDF6E0949108C08091C00085FFFCCF80
:108940009093C600319694919923B1F781E00E94EB
:10895000507A0E94CDCC2091DD083091DE08409104
:10896000DF085091E0080E9432CCAB01BC0184ECDE
:1089700098E022E030E00E949653E4EDF6E0949116
:1089800008C08091C00085FFFCCF9093C60031964F
:1089900094919923B1F782E00E94507A0E94CDCC45
:1089A0002091E1083091E2084091E3085091E408F9
:1089B0000E9432CCAB01BC0184EC98E022E030E0B4
:1089C0000E949653E4E9F2E007C08091C00085FF61
:1089D000FCCF31969093C60090819923B1F7809196
:1089E000C00085FFFCCF8AE08093C60016C580E0FA
:1089F0000E94FC7912C581E00E94FC790EC580912D
:108A0000C00085FFFCCF31969093C60090819923DA
:108A1000B1F78091C00085FFFCCF8AE08093C6004B
:108A2000ECECF6E0949108C08091C00085FFFCCF8B
:108A30009093C600319694919923B1F7009B03C09F
:108A4000E7E9F2E00AC0ECE9F2E007C08091C0007B
:108A500085FFFCCF31969093C60090819923B1F7A2
:108A60008091C00085FFFCCF8AE08093C600E4ECD3
:108A7000F6E0949108C08091C00085FFFCCF9093F0
:108A8000C600319694919923B1F7049B03C0E7E99E
:108A9000F2E00AC0ECE9F2E007C08091C00085FF77
:108AA000FCCF31969093C60090819923B1F78091C5
:108AB000C00085FFFCCF8AE08093C600ECEBF6E0B7
:108AC000949108C08091C00085FFFCCF9093C600B0
:108AD000319694919923B1F7079B03C0E7E9F2E03F
:108AE0000AC0ECE9F2E007C08091C00085FFFCCF2E
:108AF00031969093C60090819923B1F78091C00080
:108B000085FFFCCF8AE08093C60087C404EE13E0A3
:108B100039EEE32E38E0F32EF80180810E94A43371
:108B2000882349F00E94F3330E949FCCF7016083B1
:108B30007183828393830F5F1F4F24E030E0E20E46
:108B4000F31E33E0083E130739F70E94255765C42A
:108B500004EE13E029ECE22E28E0F22EF8018081E9
:108B60000E94A433882339F00E94F333F701608315
:108B70007183828393830F5F1F4F24E030E0E20E06
:108B8000F31E33E0083E130749F747C483E50E940C
:108B9000A433882351F00E94F3336093FD0870934F
:108BA000FE088093FF089093000984E50E94A43397
:108BB000882309F432C40E94F3336093010970934F
:108BC0000209809303099093040927C483E50E9456
:108BD000A433882351F00E94F3336093F908709313
:108BE000FA088093FB089093FC0884E50E94A43364
:108BF000882351F00E94F333609311097093120996
:108C0000809313099093140982E40E94A43388236B
:108C100061F00E94F3330E949FCC6093C50870936B
:108C2000C6088093C7089093C80888E50E94A433BB
:108C3000882351F00E94F33360930509709306096D
:108C400080930709909308098AE50E94A43388233A
:108C500051F00E94F3336093090970930A098093DD
:108C60000B0990930C0985E40E94A433882309F42E
:108C7000D4C30E94F33360930D0970930E0980935F
:108C80000F0990931009C9C304EE13E09CE4E92E88
:108C900096E0F92EF80180810E94A433882339F0F0
:108CA0000E94F333F70160837183828393830F5FA4
:108CB0001F4F24E030E0E20EF31E33E0073E1307BF
:108CC00049F7ABC383E50E94A433882351F00E9487
:108CD000F333609358037093590380935A0390932E
:108CE0005B0386E40E94A433882351F00E94F3338F
:108CF00060935C0370935D0380935E0390935F03C6
:108D00008AE50E94A433882309F487C30E94F333C1
:108D10006093600370936103809362039093630395
:108D20007CC383E50E94A433882351F00E94F3336F
:108D3000609368067093690680936A0690936B0649
:108D400086E40E94A433882309F467C30E94F333A6
:108D50006093640370936503809366039093670345
:108D60005CC383E50E94A433882309F456C30E94A0
:108D7000F3330E949ACC672B21F06130710561F4C6
:108D800005C0109266061092670647C381E0809383
:108D900066061092670641C3E4EEF5E0949108C0C0
:108DA0008091C00085FFFCCF9093C60031969491CE
:108DB0009923B1F7E9EAF6E0949108C08091C000E8
:108DC00085FFFCCF9093C600319694919923B1F71B
:108DD0002091A8063091A90680E690E0289FF00136
:108DE000299FF00D389FF00D1124EC54F94F07C066
:108DF0008091C00085FFFCCF31969093C600908192
:108E00009923B1F7E7EAF6E0949108C08091C00099
:108E100085FFFCCF9093C600319694919923B1F7CA
:108E20008091C00085FFFCCF8AE08093C600F5C228
:108E300083E50E94A433882309F4EFC20E94F33330
:108E40000E949ACC7093480360934703E6C283E57F
:108E50000E94A433882309F4E0C20E94F3330E94E5
:108E60009ACC70934A0360934903D7C280E50E946D
:108E7000A433882351F00E94F333609384037093EA
:108E80008503809386039093870389E40E94A4332B
:108E9000882361F00E94F3330E94758360938803F6
:108EA0007093890380938A0390938B0384E40E94D8
:108EB000A433882361F00E94F3330E94818360937E
:108EC0008C0370938D0380938E0390938F0383E4C0
:108ED0000E94A433882351F00E94F33360939003DF
:108EE0007093910380939203909393030E947D82E9
:108EF000E6EAF2E007C08091C00085FFFCCF319622
:108F00009093C60090819923B1F7E9EAF2E007C097
:108F10008091C00085FFFCCF31969093C600908170
:108F20009923B1F7409184035091850360918603A2
:108F30007091870384EC98E022E030E00E94965321
:108F4000EDEAF2E007C08091C00085FFFCCF3196CA
:108F50009093C60090819923B1F760918803709136
:108F6000890380918A0390918B030E947B83AB01DC
:108F7000BC0184EC98E022E030E00E949653E1EBE3
:108F8000F2E007C08091C00085FFFCCF319690933E
:108F9000C60090819923B1F760918C0370918D0385
:108FA00080918E0390918F030E948783AB01BC0157
:108FB00084EC98E022E030E00E949653E5EBF2E08A
:108FC00007C08091C00085FFFCCF31969093C6000A
:108FD00090819923B1F74091900350919103609152
:108FE00092037091930384EC98E022E030E00E94B9
:108FF0009653E4E9F2E007C08091C00085FFFCCF02
:1090000031969093C60090819923B1F78091C0006A
:1090100085FFFCCF8AE08093C600FFC180E50E94F7
:10902000A433882351F00E94F33360939403709328
:109030009503809396039093970389E40E94A43349
:10904000882361F00E94F3330E9475836093980334
:109050007093990380939A0390939B0384E40E94F6
:10906000A433882361F00E94F3330E9481836093CC
:109070009C0370939D0380939E0390939F030E9493
:109080007D82E6EAF2E007C08091C00085FFFCCF58
:1090900031969093C60090819923B1F7E9EAF2E006
:1090A00007C08091C00085FFFCCF31969093C60029
:1090B00090819923B1F74091940350919503609169
:1090C00096037091970384EC98E022E030E00E94D0
:1090D0009653EDEAF2E007C08091C00085FFFCCF17
:1090E00031969093C60090819923B1F760919803CF
:1090F0007091990380919A0390919B030E947B83C6
:10910000AB01BC0184EC98E022E030E00E94965371
:10911000E1EBF2E007C08091C00085FFFCCF319603
:109120009093C60090819923B1F760919C03709150
:109130009D0380919E0390919F030E948783AB01C2
:10914000BC0184EC98E022E030E00E949653E4E910
:10915000F2E007C08091C00085FFFCCF319690936C
:10916000C60090819923B1F78091C00085FFFCCFA4
:109170008AE08093C60051C183E50E94A43388230E
:1091800029F460E070E080E090E002C00E94F333D8
:109190000E941C5742C185E40E94A433882319F41D
:1091A000CC24DD2412C00E94F3330E949ACC6B01C0
:1091B00077FF0BC00F2EF0E0EF2EF0E0FF2EFCE863
:1091C0000F2FF2E41F2FF02D0AC00F2EF0E0EF2E2C
:1091D000F0E0FF2EF6E10F2FF3E41F2FF02D83E5D3
:1091E0000E94A433882321F00E94F3337B018C0179
:1091F00083E40E94A433882319F425E030E005C0FD
:109200000E94F3330E949ACC9B01C801B701A601CA
:109210000E94168A02C10E94667BFFC00E94752DC3
:10922000FCC00E94712CF9C00E948627F6C00E94E3
:109230002429F3C01092750680917B0690917C06DC
:10924000A0917D06B0917E06809377069093780674
:10925000A0937906B0937A060E943332DEC084E58B
:109260000E94A433882309F48DC00E94F3330E9426
:109270009FCC262F609376066623B9F1E4EEF5E0E5
:10928000949108C08091C00085FFFCCF9093C600E8
:10929000319694919923B1F7E9EBF2E007C0809100
:1092A000C00085FFFCCF31969093C6009081992332
:1092B000B1F784EC98E0622F40E050E00E947F52CA
:1092C000EBEBF2E007C08091C00085FFFCCF319648
:1092D0009093C60090819923B1F78091C00085FFDB
:1092E000FCCF8AE08093C60098C086E40E94A43335
:1092F0008823E1F00E94F3337B018C016093A40684
:109300007093A5068093A6069093A70620E030E010
:1093100040E050E00E942ECE181644F4E0926C0318
:10932000F0926D0300936E0310936F03E4EEF5E08B
:10933000949108C08091C00085FFFCCF9093C60037
:10934000319694919923B1F7ECECF2E007C080914B
:10935000C00085FFFCCF31969093C6009081992381
:10936000B1F76091640684EC98E070E04AE050E068
:109370000E94C3528091C00085FFFCCF8AE0809399
:10938000C6004BC0E4EEF5E0949108C08091C000A7
:1093900085FFFCCF9093C600319694919923B1F745
:1093A000E4E9F6E0949108C08091C00085FFFCCF0D
:1093B0009093C600319694919923B1F72091A80615
:1093C0003091A90680E690E0289FF001299FF00DDA
:1093D000389FF00D1124EC54F94F07C08091C00064
:1093E00085FFFCCF31969093C60090819923B1F709
:1093F000E2E9F6E0949108C08091C00085FFFCCFBF
:109400009093C600319694919923B1F78091C00052
:1094100085FFFCCF8AE08093C6000E9431301EC0D9
:109420000E94DE1960936D0670936E0680936F063E
:10943000909370060E94DE1960937F0670938006F9
:109440008093810690938206E8CF0E94667B88E530
:109450000E94A433882309F006C906C96E960FB688
:10946000F894DEBF0FBECDBFCF91DF911F910F915A
:10947000FF90EF90DF90CF90BF90AF909F908F9034
:109480007F906F905F904F903F902F9008952F9214
:109490003F924F925F926F927F928F929F92AF9284
:1094A000BF92CF92DF92EF92FF920F931F93DF93C1
:1094B000CF93CDB7DEB76E970FB6F894DEBF0FBE71
:1094C000CDBF80E6A82EB12CE3E5F8E084900AE059
:1094D000702EE9ECF8E094906624639409C22D3074
:1094E00071F02A3321F480913508882341F080916E
:1094F0003608909137088F3591050CF4D5C1E0916D
:109500003608F0913708309709F4E5C2A091380881
:10951000B0913908AA9D7001AB9DF00CBA9DF00C7A
:109520001124EE0DFF1DEC54F94F10828091350887
:10953000882309F0B4C110923508A655B94F1C9282
:1095400087010C54194FC8016EE470E00E94CCCA28
:109550009C01009709F4F4C09093B3068093B2067F
:109560002F5F3F4F201B310B2E0D3F1DC9018C5427
:10957000994F60E070E04AE050E00E94EBC86093D1
:109580003A0870933B0880933C0890933D08C09044
:109590007706D0907806E0907906F0907A06A701D9
:1095A00096012F5F3F4F4F4F5F4F6217730784073E
:1095B000950709F433C380913808909139089C01CC
:1095C0002A9DC0012B9D900D3A9D900D11248C5425
:1095D000994F62E779E00E9491CA892B09F01EC376
:1095E000EAEEF5E0949108C08091C00085FFFCCFC1
:1095F0009093C600319694919923B1F7EFE3F9E087
:10960000949108C08091C00085FFFCCF9093C60064
:10961000319694919923B1F784EC98E0B701A601B3
:109620002AE030E07DD78091C00085FFFCCF71C07B
:10963000FE264F5FFC01E40FF11DEC54F94FE08171
:10964000EA32B1F73093B3062093B206C90101960E
:1096500060E070E00E9485C70E949ACC2F2D30E018
:109660002617370709F45BC0EAEEF5E0949108C0CD
:109670008091C00085FFFCCF9093C60031969491F5
:109680009923B1F7E0E2F9E0949108C08091C0001D
:1096900085FFFCCF9093C600319694919923B1F742
:1096A00040917706509178066091790670917A061C
:1096B00084EC98E02AE030E033D78091C00085FF49
:1096C000FCCF27C0EAEEF5E0949108C08091C0007D
:1096D00085FFFCCF9093C600319694919923B1F702
:1096E000E6EFF8E0949108C08091C00085FFFCCFC0
:1096F0009093C600319694919923B1F784EC98E049
:10970000B701A6012AE030E00BD78091C00085FFA9
:10971000FCCF8AE08093C6000E94333249C080911A
:109720003A0890913B08A0913C08B0913D08809385
:10973000770690937806A0937906B0937A063DC099
:10974000C8016AE270E00E94CCCA009709F435C0F3
:10975000EAEEF5E0949108C08091C00085FFFCCF4F
:109760009093C600319694919923B1F7ECECF8E010
:10977000949108C08091C00085FFFCCF9093C600F3
:10978000319694919923B1F74091770650917806DC
:109790006091790670917A0684EC98E02AE030E0D6
:1097A000BFD68091C00085FFFCCF8AE08093C600C1
:1097B000109237081092360850C280913808909164
:1097C00039088A9D70018B9DF00C9A9DF00C112434
:1097D00087010C54194FC80167E470E00E94CCCA9D
:1097E0009C01009709F445C09093B3068093B2069C
:1097F0002F5F3F4F201B310B2E0D3F1DC9018C5495
:10980000994F60E070E00E9485C70E949ACC643056
:10981000710578F5809175068823B9F480913C0430
:10982000882339F5992DE9ECF8E008C08091C00053
:1098300085FFFCCF9093C600319694919923B1F7A0
:109840008091C00085FFFCCF12C0982DE3E5F8E0C1
:1098500008C08091C00085FFFCCF9093C600319670
:1098600094919923B1F78091C00085FFFCCF70924D
:10987000C6008091380890913908019664E070E044
:109880000E94E2D2909339088093380880913E0874
:1098900090913F08019690933F0880933E08109264
:1098A00037081092360824C02B3311F46092350823
:1098B000809135088823E1F42091360830913708EB
:1098C00080913808909139088A9DF0018B9DF00DA8
:1098D0009A9DF00D1124E20FF31FEC54F94F809183
:1098E000340880832F5F3F4F30933708209336082A
:1098F0008091C0089091C1082091C2083091C3089E
:10990000821B930B8F779070892B09F4A1C18091F2
:109910003E0890913F0804970CF09AC184EC98E0BF
:1099200025D5282F809334088A3009F0D8CDE7CD8B
:109930008091360890913708892B09F422C18DC196
:109940004D3089F04A3321F480913508882359F04D
:1099500080913608909137088F35910524F42F5F58
:109960003F4F09F0E9C020912C0630912D0640911F
:109970002E0650912F068091240690912506A091E5
:109980002606B0912706281739074A075B0708F40F
:109990009BC0962DE0E4F8E008C08091C00085FFF0
:1099A000FCCF9093C600319694919923B1F78091A2
:1099B000C00085FFFCCF3092C6000E94DE19609384
:1099C00071067093720680937306909374062091CB
:1099D0006D0630916E0640916F0650917006621BC5
:1099E000730B840B950B28EE33E040E050E00E94AF
:1099F000F5D2F22EE32ED42EC52EEDB7FEB7389752
:109A00000FB6F894FEBF0FBEEDBF0DB71EB70F5FC8
:109A10001F4FB282A182F80153824282622F732FBC
:109A2000842F952F20E13EE040E050E00E94F5D2E7
:109A3000F801358324836F2D7E2D8D2D9C2D2CE3F5
:109A400030E040E050E00E94F5D2CA01B9012CE3B9
:109A500030E040E050E00E94F5D2F8017783668361
:109A60000E9421CB972DE4EEF5E02DB73EB7285F9D
:109A70003F4F0FB6F8943EBF0FBE2DBF08C0809178
:109A8000C00085FFFCCF9093C60031969491992336
:109A9000B1F7F50107C08091C00085FFFCCF31967A
:109AA0009093C60090819923B1F78091C00085FF03
:109AB000FCCF3092C6008CE394E00E94B01C8CE393
:109AC00094E061E00E941623209136083091370817
:109AD0002115310519F410923508BFC0809138085E
:109AE00090913908889DF001899DF00D989DF00DA9
:109AF0001124E20FF31FEC54F94F1082FC01E655DC
:109B0000F94F208220913E0830913F082F5F3F4F50
:109B100030933F0820933E08019664E070E00E9475
:109B2000E2D2909339088093380810923508109249
:109B30003708109236083AC04B3311F4209235089A
:109B400080913508882391F52091360830913708A7
:109B50008091380890913908889DF001899DF00D19
:109B6000989DF00D1124E20FF31FEC54F94F8091F2
:109B7000340880832F5F3F4F309337082093360897
:109B800015C010E6812E912C22242394E0E4F8E005
:109B90006490BAE03B2E5E010894A11CB11CACE2BB
:109BA0004A2EA8E05A2EE4EEF5E0749020912C069F
:109BB00030912D0640912E0650912F06809124065B
:109BC00090912506A0912606B091270628173907FF
:109BD0004A075B0708F041C080913E0890913F081A
:109BE0000497DCF58091110690911206A09113065E
:109BF000B091140680932C0690932D06A0932E0608
:109C0000B0932F0689E096E00E94856F9C01482F53
:109C1000809334088A3009F093CEA5CE809138081D
:109C2000909139088A9D80018B9D100D9A9D100D91
:109C30001124C8018C54994F6AE270E00E94CCCA8A
:109C40009C01009709F43ECDFF2440E0C801F2CC0E
:109C500080913E04882309F06BCE6E960FB6F8947F
:109C6000DEBF0FBECDBFCF91DF911F910F91FF904F
:109C7000EF90DF90CF90BF90AF909F908F907F90AC
:109C80006F905F904F903F902F900895CF93DF9308
:109C900080913E0890913F0803970CF4F8DB8CE329
:109CA00094E060E00E94162380913E0890913F0866
:109CB000892B09F469C080913C04882309F44CC0C5
:109CC0002091A8063091A90680E690E0289FE00147
:109CD000299FD00D389FD00D1124CC54D94FCE01DF
:109CE0006CE879E00E9491CA892BE1F48CE394E05E
:109CF000BE010E94AE1D80913D04882369F5E9E80C
:109D0000F9E0949108C08091C00085FFFCCF90934A
:109D1000C600319694919923B1F78091C00085FFD8
:109D2000FCCF16C08CE394E00E94951DE7E7F9E0B4
:109D3000949108C08091C00085FFFCCF9093C6002D
:109D4000319694919923B1F78091C00085FFFCCFA3
:109D50008AE08093C60002C00E94183680913E08B7
:109D600090913F08019790933F0880933E0880911F
:109D7000A8069091A906019664E070E00E94E2D2E4
:109D80009093A9068093A8060E9482870E945A3069
:109D90000E94DF810E94D090DF91CF910895269A92
:109DA0002E9884EC98E040E950ED63E070E0AAD290
:109DB000E3E6FAE0949108C08091C00085FFFCCFF3
:109DC0009093C600319694919923B1F78091C00089
:109DD00085FFFCCF8AE08093C60044EE55E0FA018F
:109DE000949108C08091C00085FFFCCF9093C6007D
:109DF000319694919923B1F784B7282F80FF15C02D
:109E0000EBE5FAE0949108C08091C00085FFFCCF9B
:109E10009093C600319694919923B1F78091C00038
:109E200085FFFCCF8AE08093C60021FF15C0EBE4DC
:109E3000FAE0949108C08091C00085FFFCCF909318
:109E4000C600319694919923B1F78091C00085FFA7
:109E5000FCCF8AE08093C60022FF15C0EAE3FAE057
:109E6000949108C08091C00085FFFCCF9093C600FC
:109E7000319694919923B1F78091C00085FFFCCF72
:109E80008AE08093C60023FF15C0EAE2FAE09491CD
:109E900008C08091C00085FFFCCF9093C60031962A
:109EA00094919923B1F78091C00085FFFCCF8AE09F
:109EB0008093C60025FF15C0EAE1FAE0949108C03E
:109EC0008091C00085FFFCCF9093C600319694919D
:109ED0009923B1F78091C00085FFFCCF8AE0809381
:109EE000C60014BEE2E1FAE0949108C08091C0007F
:109EF00085FFFCCF9093C600319694919923B1F7DA
:109F0000ECE0FAE0949108C08091C00085FFFCCF9E
:109F10009093C600319694919923B1F78091C00037
:109F200085FFFCCF8AE08093C600FA019491E4EEAD
:109F3000F5E008C08091C00085FFFCCF9093C6007B
:109F4000319694919923B1F7ECEFF9E0949108C020
:109F50008091C00085FFFCCF9093C600319694910C
:109F60009923B1F7E7EEF9E0949108C08091C00021
:109F700085FFFCCF9093C600319694919923B1F759
:109F8000EBEDF9E0949108C08091C00085FFFCCF13
:109F90009093C600319694919923B1F7EDECF9E0D6
:109FA000949108C08091C00085FFFCCF9093C600BB
:109FB000319694919923B1F78091C00085FFFCCF31
:109FC0008AE08093C600E2ECF9E0949108C08091A9
:109FD000C00085FFFCCF9093C600319694919923E1
:109FE000B1F7E6EBF9E0949108C08091C00085FFDD
:109FF000FCCF9093C600319694919923B1F780914C
:10A00000C00085FFFCCF8AE08093C600FA019491DE
:10A01000E4EEF5E008C08091C00085FFFCCF90938E
:10A02000C600319694919923B1F7E7EAF9E094914B
:10A0300008C08091C00085FFFCCF9093C600319688
:10A0400094919923B1F70E94712EBC0184EC98E0A1
:10A050004AE050E098D2E0E9F9E0949108C080919C
:10A06000C00085FFFCCF9093C60031969491992350
:10A07000B1F784EC98E060ED74E04AE050E083D200
:10A080008091C00085FFFCCF8AE08093C6001092CB
:10A09000AA061092AB061092AC061092AD060E9472
:10A0A000712C0E9496860E94C9590E9477C70E940F
:10A0B000EF7A0C943291BC0180913E0890913F0858
:10A0C00004970CF070C0209138083091390880E670
:10A0D00090E0AC01249FC001259F900D349F900D0E
:10A0E00011248C54994F0E945BCAE4EEF5E09491E0
:10A0F00008C08091C00085FFFCCF9093C6003196C8
:10A1000094919923B1F7EBE6FAE0949108C080911D
:10A11000C00085FFFCCF9093C6003196949199239F
:10A12000B1F7209138083091390880E690E0289FF7
:10A13000F001299FF00D389FF00D1124EC54F94FD8
:10A1400007C08091C00085FFFCCF31969093C60078
:10A1500090819923B1F7E9E6FAE0949108C08091E3
:10A16000C00085FFFCCF9093C6003196949199234F
:10A17000B1F78091C00085FFFCCF8AE08093C600D4
:10A18000C901019664E070E00E94E2D29093390820
:10A190008093380880913E0890913F0801969093F3
:10A1A0003F0880933E080895BC0180913E0890913D
:10A1B0003F0804970CF070C020913808309139089E
:10A1C00080E690E0AC01249FC001259F900D349F54
:10A1D000900D11248C54994F0E94D7CAE4EEF5E0FB
:10A1E000949108C08091C00085FFFCCF9093C60079
:10A1F000319694919923B1F7E8E7FAE0949108C079
:10A200008091C00085FFFCCF9093C6003196949159
:10A210009923B1F7209138083091390880E690E011
:10A22000289FF001299FF00D389FF00D1124EC5468
:10A23000F94F07C08091C00085FFFCCF3196909305
:10A24000C60090819923B1F7E6E7FAE0949108C03F
:10A250008091C00085FFFCCF9093C6003196949109
:10A260009923B1F78091C00085FFFCCF8AE08093ED
:10A27000C600C901019664E070E00E94E2D29093AA
:10A2800039088093380880913E0890913F080196E4
:10A2900090933F0880933E0808951F920F920FB647
:10A2A0000F920BB60F9211242F933F934F938F93DE
:10A2B0009F93EF93FF934091C600E091C008F09107
:10A2C000C10831969F012F77307031978091C20875
:10A2D0009091C3082817390739F0E05CF74F4083A5
:10A2E0003093C1082093C008FF91EF919F918F9107
:10A2F0004F913F912F910F900BBE0F900FBE0F907B
:10A300001F9018959A01AB01203081EE380780E04C
:10A31000480780E0580729F182E08093C00060E0A0
:10A3200079E08DE390E00E94F5D22150304040402A
:10A33000504056954795379527953093C500209303
:10A34000C4008091C10080618093C1008091C100F0
:10A3500088608093C1008091C10080688093C100B3
:10A3600008951092C00020E130E0E7CF2091C208AC
:10A370003091C3088091C0089091C108821793075B
:10A3800019F42FEF3FEF0EC0F901E05CF74F808129
:10A390002F5F3F4F2F7730703093C3082093C20850
:10A3A000282F30E0C90108958091C2089091C30818
:10A3B0009093C1088093C008089508952F923F920A
:10A3C0004F925F926F927F928F929F92AF92BF92C5
:10A3D000CF92DF92EF92FF920F931F93DF93CF9371
:10A3E000CDB7DEB7A0970FB6F894DEBF0FBECDBFD6
:10A3F0001C016A017B01411551056105710541F49C
:10A4000040E350E060E070E020E030E089D053C0ED
:10A41000882499245401422E55246624772401E08F
:10A4200010E00C0F1D1F080D191DC701B601A30177
:10A4300092010E94F5D2F80160830894811C911C5E
:10A44000A11CB11CC701B601A30192010E94F5D263
:10A45000C901DA016C017D01C114D104E104F104E8
:10A46000F1F691E0E92EF12CEC0EFD1EE80CF91C42
:10A470003E010894611C711CD501C4010197A1091A
:10A48000B1096C01C818D90813C0F601EE0DFF1D03
:10A4900040814A3010F4405D01C0495C50E060E00A
:10A4A00070E0C10120E030E03BD00894E108F10801
:10A4B0006E147F0451F7A0960FB6F894DEBF0FBE5E
:10A4C000CDBFCF91DF911F910F91FF90EF90DF9063
:10A4D000CF90BF90AF909F908F907F906F905F9044
:10A4E0004F903F902F9008952115310539F48091B8
:10A4F000C00085FFFCCF4093C60008955FCFEF9268
:10A50000FF920F931F939A01E62EFF2400E010E0C4
:10A51000B801A701E9DF1F910F91FF90EF90089517
:10A52000EF92FF920F931F93CF93DF93EC017A0189
:10A530008B012115310539F48091C00085FFFCCFD6
:10A54000E092C60019C02A303105A9F477FF0FC088
:10A550004DE250E060E070E020E030E0E1DF109597
:10A560000095F094E094E11CF11C011D111DCE0139
:10A57000B801A7012AE022DFDF91CF911F910F914F
:10A58000FF90EF900895EF92FF920F931F937B013E
:10A590009A010027F7FC0095102FB801A701C0DF32
:10A5A0001F910F91FF90EF9008950F931F938C01CF
:10A5B0004DE050E060E070E020E030E0B1DFC80145
:10A5C0004AE050E060E070E020E030E0A9DF1F9159
:10A5D0000F910895CF92DF92EF92FF920F931F9306
:10A5E0008C019A016B01EE24FF24B701A6017CDFE8
:10A5F000C801DBDF1F910F91FF90EF90DF90CF90AC
:10A6000008959F92AF92BF92CF92DF92EF92FF9206
:10A610000F931F93CF93DF93EC017A018B01922E5E
:10A62000CB01BA0120E030E040E050E00E942BCCAA
:10A63000882364F4CE014DE250E060E070E020E059
:10A6400030E06EDF17FB109517F9109520E030E031
:10A6500040E05FE3AA240BC0CA01B90120E030E06A
:10A6600040E251E40E9432CC9B01AC01A394A914B6
:10A6700098F3C801B7010E9452CB7B018C010E9464
:10A680009FCC5B016C010E94CBCC9B01AC01C8014B
:10A69000B7010E9451CB7B018C01CE01B601A5010F
:10A6A0002AE030E021DF992099F1EEEDF2E007C0D9
:10A6B0008091C00085FFFCCF31969093C6009081B9
:10A6C0009923B1F725C0C801B70120E030E040E28E
:10A6D00051E40E9400CF7B018C010E949ACC5B0167
:10A6E0006C01CC24B7FCC094DC2CCE01B601A501D2
:10A6F0002AE030E015DFC601B5010E94CDCC9B01F8
:10A70000AC01C801B7010E9451CB7B018C019A9426
:10A710009920C9F6DF91CF911F910F91FF90EF9093
:10A72000DF90CF90BF90AF909F9008956ACF08952B
:10A730002F923F924F925F926F927F928F929F9251
:10A74000AF92BF92CF92DF92EF92FF920F931F933F
:10A75000DF93CF93CDB7DEB7CD55D0400FB6F89489
:10A76000DEBF0FBECDBF2F969FAF8EAF2F976196E6
:10A770007FAF6EAF61972A0162962FAF62976396A3
:10A780000FAF63976496EFAE64976896ACAEBDAEBC
:10A79000CEAEDFAE6897E22EFF24EE0CFF1CEE0C6F
:10A7A000FF1C9A012E0D3F1D2D963FAF2EAF2D970A
:10A7B000D9016D907D908D909C90FC01EE0DFF1D58
:10A7C000C401B30120813181428153810E9452CB67
:10A7D00069AF7AAF8BAF9CAF10E0000F111F000F75
:10A7E000111FF201E00FF11F2B96FFAFEEAF2B9779
:10A7F000A080B180C280D3802F96EEADFFAD2F97A1
:10A80000E00FF11FC601B5012081318142815381E2
:10A810000E9452CB6DAB7EAB8FAB98AF64962FADE1
:10A820006497E22FF0E0EE0FFF1FEE0FFF1F2F9651
:10A83000AEADBFAD2F97AE0FBF1F4D915D916D9126
:10A840007C9129964CAF5DAF6EAF7FAF2997619633
:10A850006EAD7FAD6197E60FF71F608171818281D8
:10A86000938129962CAD3DAD4EAD5FAD29970E94E9
:10A8700051CB69AB7AAB8BAB9CAB6196AEADBFAD48
:10A8800061971C968D919D910D90BC91A02D259660
:10A890008CAF9DAFAEAFBFAF25972F96AEADBFAD1E
:10A8A0002F971C962D913D914D915C911F9721966C
:10A8B0002CAF3DAF4EAF5FAF2197A401930150582D
:10A8C0002DA73EA74FA758ABB601A501705849A7C1
:10A8D0005AA76BA77CA761966EAD7FAD6197E60E18
:10A8E000F71ED7016D917D918D919C9129AD3AAD67
:10A8F0004BAD5CAD0E9451CB3B014C016196EEAD7E
:10A90000FFAD61970E0F1F1FD8016D917D918D9145
:10A910009C912DA93EA94FA958AD0E9451CB5B0136
:10A920006C016DA57EA58FA598A9A60195010E9431
:10A9300000CF7B018C0169A57AA58BA59CA5A401FC
:10A9400093010E9400CF9B01AC01C801B7010E9496
:10A9500051CB1B012C016DA57EA58FA598A9A40143
:10A9600093010E9400CF7B018C0169A57AA58BA57C
:10A970009CA5A60195010E9400CF9B01AC01C801D6
:10A98000B7010E9452CB9B01AC01C201B1010E94F0
:10A99000C5CB5B016C0120E030E040E050E00E945C
:10A9A0002BCC882354F4C601B5012BED3FE049ECD4
:10A9B00050E40E9452CB5B016C01E8968FADE897A2
:10A9C000882351F0C601B5012BED3FE049EC50E47E
:10A9D0000E9451CB5B016C01C601B501E7962CAD1D
:10A9E0003DAD4EAD5FADE7970E9400CF29A93AA9D2
:10A9F0004BA95CA95F770E943BCE7B018C012FE6BF
:10AA000032E143E85AE30E942BCC87FDF4C1C80130
:10AA1000B7010E9408CD0E949FCC78A76FA3672B37
:10AA200021F4E1E0F0E0F8A7EFA32FA138A5B901E8
:10AA300080E090E00E94CBCC7B018C01C601B50187
:10AA4000A80197010E9432CC6BA37CA38DA39EA387
:10AA500069A97AA98BA99CA9A80197010E9432CC67
:10AA60006F8F78A389A39AA325966CAD7DAD8EAD2B
:10AA70009FAD259721962CAD3DAD4EAD5FAD219795
:10AA80000E9451CBA80197010E9432CC6B8F7C8F22
:10AA90008D8F9E8F6BA17CA18DA19EA120E030E0C7
:10AAA00040E05FEB0E9400CF2BA13CA14DA15EA135
:10AAB0000E9400CF20E030E040E85FE30E9452CBEC
:10AAC0006F8B788F898F9A8F64963FAD6497E32F51
:10AAD000F0E0EE0FFF1FEE0FFF1F9E012F5F3F4FB5
:10AAE000E20FF31F29964CAD5DAD6EAD7FAD29979A
:10AAF00040835183628373832F96AEADBFAD2F9792
:10AB00001C964D915D916D917C911F974D875E874D
:10AB10006F87788B41E050E05A8B498B66246296B0
:10AB20007FAD6297672F70E0660F771F660F771F04
:10AB3000C901860F971F6A969FAF8EAF6A9763967B
:10AB4000BFAD6397AB2FB0E0AA0FBB1FAA0FBB1F0F
:10AB500021E030E02C0F3D1F2A0F3B1F6C963FAFCA
:10AB60002EAF6C976E96FFAFEEAF6E9719C138E1BE
:10AB700036150CF446C06DA57EA58FA598A92BA10E
:10AB80003CA14DA15EA10E9400CF7B018C0169A573
:10AB90007AA58BA59CA52F89388D498D5A8D0E9449
:10ABA00000CF9B01AC01C801B7010E9452CB7B01D1
:10ABB0008C016DA57EA58FA598A92F89388D498D0B
:10ABC0005A8D0E9400CF5B016C0169A57AA58BA507
:10ABD0009CA52BA13CA14DA15EA10E9400CF9B0191
:10ABE000AC01C601B5010E9451CB6DA77EA78FA70E
:10ABF00098AB6394C701D80189A79AA7ABA7BCA754
:10AC000065C049895A89BA0180E090E00E94CBCCA6
:10AC10002BA13CA14DA15EA10E9400CF7B018C0124
:10AC2000C8010E942FCC6B8B7C8B8D8B9E8BB701C8
:10AC3000C8010E9463CF3B014C012D96AEADBFAD64
:10AC40002D97ED90FD900D911C9117FB109517F924
:10AC500010952B96EEADFFAD2B9720803180428072
:10AC60005380C801B7012B893C894D895E890E94B8
:10AC700000CF5B016C01C201B101A40193010E94EC
:10AC800000CF9B01AC01C601B5010E9452CB6DA75C
:10AC90007EA78FA798ABC801B701A40193010E94BA
:10ACA00000CF7B018C01C201B1012B893C894D8908
:10ACB0005E890E9400CF9B01AC01C801B7010E94D0
:10ACC00051CB69A77AA78BA79CA7662469AD7AADFB
:10ACD0008BAD9CAD2DA53EA54FA558A90E9452CB8A
:10ACE0006A96AEADBFAD6A976D937D938D939C933D
:10ACF00013976DA97EA98FA998AD29A53AA54BA553
:10AD00005CA50E9452CB6C96EEADFFAD6C97608354
:10AD10007183828393836E96AEADBFAD6E976D9156
:10AD20007D918D919C912F8D38A149A15AA10E94AE
:10AD300052CB6E96EEADFFAD6E97608371838283CA
:10AD400093836D857E858F8598892B8D3C8D4D8D68
:10AD50005E8D0E9452CB6D877E878F87988BCE0148
:10AD600001960E94F42ECE010196BE016B5F7F4FCB
:10AD7000AE01475F5F4F9E01235F3F4F6896ECAC8B
:10AD8000FDAC0EAD1FAD6897F8E7CF2ED12CCC0EE1
:10AD9000DD1EC2D529893A892F5F3F4F3A8B298B17
:10ADA00049895A896FA178A54617570708F4DFCE5D
:10ADB00061964EAD5FAD6197485F5F4F61962EAD76
:10ADC0003FAD6197245F3F4F61968EAD9FAD619718
:10ADD000DC0114966196BFAFAEAF6197BD01689676
:10ADE000ECACFDAC0EAD1FAD6897E8E7CE2ED12CD4
:10ADF000CC0EDD1E91D5C35ADF4F0FB6F894DEBFDF
:10AE00000FBECDBFCF91DF911F910F91FF90EF90BB
:10AE1000DF90CF90BF90AF909F908F907F906F907A
:10AE20005F904F903F902F9008958091050E9091E4
:10AE3000060E891B8F7008956093750370937603D7
:10AE4000809377039093780308950F931F93CF9384
:10AE5000DF93C0E0D0E08E010B5E164FFE01E7519C
:10AE6000F74F60817181828193810E94CBCCFE017A
:10AE7000E752F74F20813181428153810E9400CFF8
:10AE80000E949FCCF8016083718382839383249610
:10AE9000C031D10501F7DF91CF911F910F91089536
:10AEA000FC0160817181828193812091E50830915C
:10AEB000E6084091E7085091E8080E9400CF2091F1
:10AEC00071033091720340917303509174030E9497
:10AED00000CF0E94D0CE60933109709332098093E5
:10AEE00033099093340981E399E00C943F7A8F926F
:10AEF0009F92AF92BF92CF92DF92EF92FF920F9309
:10AF00001F93FC018B015A0149016081718182818B
:10AF100093812091D9083091DA084091DB08509153
:10AF2000DC080E9400CF0E94D0CE35E2C32E39E06B
:10AF3000D32E609325097093260980932709909357
:10AF40002809F80160817181828193812091DD0857
:10AF50003091DE084091DF085091E0080E9400CF58
:10AF60000E94D0CE24E0E22EF12CEC0CFD1C60936C
:10AF70002909F701718382839383F50160817181CF
:10AF8000828193812091E1083091E2084091E308A9
:10AF90005091E4080E9400CF0E94D0CE8601085F45
:10AFA0001F4F60932D09F801718382839383F4010D
:10AFB00060817181828193812091E5083091E6085A
:10AFC0004091E7085091E8080E9400CF209171035A
:10AFD0003091720340917303509174030E9400CF2B
:10AFE0000E94D0CEF6013C96609331097183828332
:10AFF0009383C601B701A8019F010E94057A80E0F2
:10B0000090E0A0E0B0E08093070E9093080EA0932C
:10B01000090EB0930A0E80930B0E90930C0EA09322
:10B020000D0EB0930E0E80930F0E9093100EA09302
:10B03000110EB093120E8093130E9093140EA093E2
:10B04000150EB093160E8093170E9093180EA093C2
:10B05000190EB0931A0E1F910F91FF90EF90DF9091
:10B06000CF90BF90AF909F908F9008958F929F92B6
:10B07000AF92BF92CF92DF92EF92FF920F931F9306
:10B08000CF93DF93EC016B01009709F45CC08FA9AB
:10B09000882309F058C0EEA0FFA008A519A5FB0160
:10B0A000B6A0A7A090A481A4C801B7012B2D3A2D6A
:10B0B000492D582D0E942BCC88230CF044C0C80188
:10B0C000B701A80197010E9400CF7B018C016AA9FA
:10B0D0007BA98CA99DA9905820E030E040E050EC7D
:10B0E0000E9400CF2EA53FA548A959A90E9400CFD4
:10B0F0009B01AC01C801B7010E9452CB0E946DCFE9
:10B100007B018C016B2D7A2D892D982D9701A8013B
:10B110000E942BCC882324F4EB2CFA2C092D182D1B
:10B120006B2D7A2D892D982D9701A8010E942BCC8B
:10B13000882349F0C701D801F60186A397A3A0A7E9
:10B14000B1A781E086ABDF91CF911F910F91FF9066
:10B15000EF90DF90CF90BF90AF909F908F90089529
:10B16000EF92FF920F931F93CF93DF93F090060E11
:10B1700000E010E020E030E04DE4E42E11C0FE9C41
:10B18000E0011124CB5CD64FC901B801AE016EDFDE
:10B190008F2D8F5F803109F480E0F82E98018E01A9
:10B1A0008091050EF81659F7C901B80140E050E04A
:10B1B0005DDFDF91CF911F910F91FF90EF90089588
:10B1C000AF92BF92CF92DF92EF92FF920F931F93B5
:10B1D000CF93DF93EB018A016115710509F466C015
:10B1E0004115510509F462C0DAA4CBA4BCA4ADA4F6
:10B1F0006EA17FA188A599A52D2D3C2D4B2D5A2DF3
:10B200000E942BCC882309F451C08FA9882309F010
:10B2100043C0F801E6A0F7A000A511A56D2D7C2D77
:10B220008B2D9A2DA80197010E942ECE1816A4F5F9
:10B23000C801B701A80197010E9400CF7B018C01D2
:10B240006AA97BA98CA99DA9905820E030E040E034
:10B2500050EC0E9400CF2EA53FA548A959A90E94F5
:10B2600000CF9B01AC01C801B7010E9452CB0E94E4
:10B270006DCF7B018C016D2D7C2D8B2D9A2D97012F
:10B28000A8010E942BCC882324F4ED2CFC2C0B2D40
:10B290001A2DC701D80104C08D2D9C2DAB2DBA2DC0
:10B2A0008EA39FA3A8A7B9A781E08EABDF91CF9112
:10B2B0001F910F91FF90EF90DF90CF90BF90AF90D4
:10B2C0000895CF92DF92EF92FF920F93DF93CF9387
:10B2D0000F920F92CDB7DEB78091050E8FB7F8941D
:10B2E000F090060E8FBF8091050E90E040968F196A
:10B2F00091098F7090700497FCF00091050E035037
:10B300000F70CC24DD2440E050E06DE4E62E12C046
:10B31000802F002309F480E1082F01500E9DC00109
:10B3200011248B5C964F9A838983B60149DFA6016D
:10B33000C980DA800F1561F70F900F90CF91DF91E0
:10B340000F91FF90EF90DF90CF9008956091650688
:10B350009091060E8091050E9817B9F04091060E57
:10B36000242F30E08DE490E0289FF001299FF00D1C
:10B37000389FF00D1124E358F64F608102C04F5FF3
:10B380004F708091050E4817D1F787E070E00C945C
:10B390004E1A1092050E1092060E80E1E5E2F9E0D9
:10B3A000DF011D928A95E9F780E090E0A0E0B0E02F
:10B3B00080930B0E90930C0EA0930D0EB0930E0E77
:10B3C00080930F0E9093100EA093110EB093120E57
:10B3D0008093130E9093140EA093150EB093160E37
:10B3E0008093170E9093180EA093190EB0931A0E17
:10B3F0008093070E9093080EA093090EB0930A0E47
:10B4000008952F923F924F925F926F927F928F9208
:10B410009F92AF92BF92CF92DF92EF92FF920F93E3
:10B420001F93DF93CF93CDB7DEB766970FB6F8942F
:10B43000DEBF0FBECDBF9E8B8D8B6A017B014801A5
:10B440005901DC01D8966D917D918D919C91DB978E
:10B450000E94CBCC698B7A8B8B8B9C8BA70196013E
:10B460000E9400CF0E9418CC0E949FCC6D837E83E7
:10B470008F83988769897A898B899C89A501940132
:10B480000E9400CF0E9418CC0E949FCC69837A83CF
:10B490008B839C832D813E814F81588528373105D0
:10B4A0004105510540F448E750E060E070E04D830D
:10B4B0005E836F83788769817A818B819C8168370D
:10B4C00071058105910540F488E790E0A0E0B0E0C7
:10B4D00089839A83AB83BC83AD89BE89AC5BBF4F44
:10B4E000AD90BD90CD90DC901397A454B040BE8B2E
:10B4F000AD8BDC966D917D918D919C91DF970E9433
:10B50000CBCC6D877E878F87988BC601B5010E9453
:10B51000CDCC1B012C0120E030E040E050E00E9447
:10B520002BCC882321F4E0E070E060E028C069893A
:10B530007A898B899C899B01AC010E9400CF7B0199
:10B540008C016D857E858F8598899B01AC010E9459
:10B5500000CF9B01AC01C801B7010E9451CB7B0118
:10B560008C01C201B101A20191010E9452CB9B0149
:10B57000AC01C801B7010E9432CCE62F692F2E2FF3
:10B58000372F482F562FB901CA010E9418CC0E94AC
:10B590009ACC3B014C01ED89FE89E05CFF4F608154
:10B5A0007181828193810E94CBCC69877A878B8756
:10B5B0009C8766277727CB016A197B098C099D092F
:10B5C0000E94CDCC5B016C0120E030E040E050E017
:10B5D0000E942BCC882321F4E0E070E060E028C0DA
:10B5E00069857A858B859C859B01AC010E9400CF83
:10B5F0007B018C0169897A898B899C899B01AC01CB
:10B600000E9400CF9B01AC01C801B7010E9451CB41
:10B610007B018C01C601B501A60195010E9452CBA8
:10B620009B01AC01C801B7010E9432CCE62F692F03
:10B630002E2F372F482F562FB901CA010E9408CD4F
:10B64000ED89FE89A088B188C288D38886017501FA
:10B65000E618F708080919090E949ACCA801970171
:10B66000261B370B480B590B57FF71C0C201B101A4
:10B6700020E030E040E050E00E942BCC882321F411
:10B68000E0E070E060E044C0C201B101A2019101BC
:10B690000E9452CB7B018C01C601B5010E94CBCC2C
:10B6A0009B01AC01C801B7010E9400CF7B018C0156
:10B6B0006D857E858F8598899B01AC010E9400CFA6
:10B6C0009B01AC01C801B7010E9451CB7B018C01E9
:10B6D00069857A858B859C859B01AC010E9400CF92
:10B6E0009B01AC01C801B7010E9452CB7B018C01C8
:10B6F000C201B10120E030E040E850E40E9400CFF8
:10B700009B01AC01C801B7010E9432CCE62F692F22
:10B710002E2F372F482F562FB901CA010E9418CC5F
:10B720000E949ACCAC01CB01DA013C014D0197FE9D
:10B7300003C06624772443016A147B048C049D04AF
:10B7400010F03501460120E030E040E050E09FB7C6
:10B75000F8946D897E89645B7F4FDB018C91AC54DA
:10B76000B040BE8BAD8B882321F5FD01648A758ABC
:10B77000868A978A260D371D481D591D58962D9388
:10B780003D934D935C935B972D813E814F8158850E
:10B79000DC962D933D934D935C93DF97A05CBF4F58
:10B7A00029813A814B815C812D933D934D935C932C
:10B7B00013979FBF66960FB6F894DEBF0FBECDBF3E
:10B7C000CF91DF911F910F91FF90EF90DF90CF907D
:10B7D000BF90AF909F908F907F906F905F904F90B1
:10B7E0003F902F9008954F925F927F928F929F92F9
:10B7F000AF92BF92CF92DF92EF92FF920F931F937F
:10B80000CF93DF937090060EC0E0D0E07DE4472E2A
:10B81000512C45C02097A9F18EA9882361F4849CFE
:10B82000F001859CF00D949CF00D1124EB5CF64F1B
:10B8300086A9882331F1EAA0FBA00CA11DA16EA16D
:10B840007FA188A599A5A80197010E9432CC5B0130
:10B850006C01849CF001859CF00D949CF00D1124EA
:10B86000EB5CF64F66A177A180A591A5A801970191
:10B870000E9432CC8B019C01CE01B601A501C1DD35
:10B880001EAA739480E1781609F47724849CE00161
:10B89000859CD00D949CD00D1124CB5CD64F872C69
:10B8A000992487FC90948091050E90E08816990663
:10B8B00009F0B0CF2097E9F0EAA0FBA00CA11DA1F0
:10B8C0006EA17FA188A599A5A80197010E9432CCFD
:10B8D0005B016C016DEC7CEC8CE49DE3A8019701AD
:10B8E0000E9432CC8B019C01CE01B601A50189DDFD
:10B8F0001EAADF91CF911F910F91FF90EF90DF90E3
:10B90000CF90BF90AF909F908F907F905F904F901F
:10B910000895D7DC25DC67CF2F923F924F925F923C
:10B920006F927F928F929F92AF92BF92CF92DF924F
:10B93000EF92FF920F931F93DF93CF93CDB7DEB7B4
:10B94000C859D0400FB6F894DEBF0FBECDBF5C0122
:10B950004B013A012901CB56DF4FE882C559D0404F
:10B96000CA56DF4FF882C659D040C956DF4F088308
:10B97000C759D040C856DF4F1883C859D040E39606
:10B98000DFAECEAEE3978091050E8F5F803109F474
:10B9900080E0282F332727FD30953CA72BA706C032
:10B9A0000E9482870E945A300E94D0908091060E99
:10B9B00090E04BA55CA58417950791F36091D90899
:10B9C0007091DA088091DB089091DC08E1966CAF09
:10B9D0007DAF8EAF9FAFE197D5012D913D914D91F8
:10B9E0005C910E9400CF0E94D0CEC158DF4F688387
:10B9F000CF57D040C058DF4F7883C058D040CF5782
:10BA0000DF4F8883C158D040CE57DF4F9883C2584C
:10BA1000D0402091DD083091DE084091DF08509140
:10BA2000E008AD962CAF3DAF4EAF5FAFAD97CA010A
:10BA3000B901D4012D913D914D915C910E9400CFAF
:10BA40000E94D0CECD57DF4F6883C358D040CC572B
:10BA5000DF4F7883C458D040CB57DF4F8883C55819
:10BA6000D040CA57DF4F9883C658D0402091E10894
:10BA70003091E2084091E3085091E408A9962CAF78
:10BA80003DAF4EAF5FAFA997CA01B901D3012D9168
:10BA90003D914D915C910E9400CF0E94D0CEC9573C
:10BAA000DF4F6883C758D040C857DF4F7883C858E6
:10BAB000D040C757DF4F8883C958D040C657DF4FA3
:10BAC0009883CA58D0402091E5083091E60840910B
:10BAD000E7085091E808A5962CAF3DAF4EAF5FAF99
:10BAE000A597CA01B901D2012D913D914D915C916B
:10BAF0000E9400CF20917103309172034091730333
:10BB0000509174030E9400CF0E94D0CEC557DF4FE2
:10BB10006883CB58D040C457DF4F7883CC58D0408F
:10BB2000C357DF4F8883CD58D040C257DF4F98832B
:10BB3000CE58D0408091310990913209A0913309BB
:10BB4000B0913409C557DF4F288139814A815B8123
:10BB5000CB58D040281739074A075B0709F4B8C00B
:10BB6000E0916406F0E0EE0FFF1FEE0FFF1FEA58B2
:10BB7000FF4E6081718182819381209175033091A4
:10BB8000760340917703509178030E942BCC882351
:10BB90000CF033C0C557DF4F488159816A817B81E2
:10BBA000CB58D04040933109509332096093330908
:10BBB00070933409E3E8FAE0949108C08091C000E2
:10BBC00085FFFCCF9093C600319694919923B1F7ED
:10BBD000E7EAFAE0949108C08091C00085FFFCCFAD
:10BBE0009093C600319694919923B1F78091C0004B
:10BBF00085FFFCCF8AE08093C60080913109909147
:10BC00003209A0913309B0913409C557DF4F28811B
:10BC100039814A815B81CB58D040281B390B4A0BB4
:10BC20005B0BCA01B90157FF07C0909580957095CD
:10BC300061957F4F8F4F9F4F0E94CDCC7B018C0130
:10BC4000A5966CAD7DAD8EAD9FADA59720E030E89B
:10BC500043EE53E40E9400CF9B01AC01C801B70141
:10BC60000E942ECE18160CF033C0C557DF4F488106
:10BC700059816A817B81CB58D040409331095093E0
:10BC800032096093330970933409E3E8FAE0949140
:10BC900008C08091C00085FFFCCF9093C60031960C
:10BCA00094919923B1F7E9E8FAE0949108C0809162
:10BCB000C00085FFFCCF9093C600319694919923E4
:10BCC000B1F78091C00085FFFCCF8AE08093C60069
:10BCD0008091050E682F70E0A1967FAF6EAFA1979F
:10BCE0008DE490E0689FF001699FF00D789FF00D62
:10BCF0001124EB5CF64FE45BFF4F1082EC54F040F4
:10BD00008091250990912609A0912709B0912809D1
:10BD10006F968CAF9DAFAEAFBFAF6F97C158DF4F7F
:10BD2000288139814A815B81CF57D040281B390B4C
:10BD30004A0B5B0B6B962CAF3DAF4EAF5FAF6B9773
:10BD4000208331834283538357FF0DC0DA01C90139
:10BD5000B095A095909581959F4FAF4FBF4F808331
:10BD60009183A283B3834091290950912A0960915C
:10BD70002B0970912C0967964CAF5DAF6EAF7FAF0A
:10BD80006797CD57DF4F88819981AA81BB81C358BE
:10BD9000D040841B950BA60BB70B63968CAF9DAF61
:10BDA000AEAFBFAF63978DE490E0A196AEADBFADEF
:10BDB000A197A89FF001A99FF00DB89FF00D112445
:10BDC000EB5CF64F63962CAD3DAD4EAD5FAD63972A
:10BDD000248335834683578357FF0DC0DA01C90199
:10BDE000B095A095909581959F4FAF4FBF4F84839D
:10BDF0009583A683B78340912D0950912E096091B8
:10BE00002F09709130092F964CAF5DAF6EAF7FAFA9
:10BE10002F97C957DF4F88819981AA81BB81C75865
:10BE2000D040841B950BA60BB70B2B968CAF9DAF08
:10BE3000AEAFBFAF2B978DE490E0A196AEADBFAD96
:10BE4000A197A89FF001A99FF00DB89FF00D1124B4
:10BE5000EB5CF64F2B962CAD3DAD4EAD5FAD2B9709
:10BE6000208731874287538757FF0DC0DA01C90108
:10BE7000B095A095909581959F4FAF4FBF4F80870C
:10BE80009187A287B3872090310930903209409082
:10BE9000330950903409C557DF4F488159816A8171
:10BEA0007B81CB58D04042195309640975094DA3D1
:10BEB0005EA36FA378A76091490370914A03279608
:10BEC0007FAF6EAF27976DA17EA18FA198A597FF39
:10BED00007C090958095709561957F4F8F4F9F4FCC
:10BEE0002796AEADBFAD27979D01442737FD4095FE
:10BEF000542F0E94A3D224E630E040E050E00E949C
:10BF000017D38DE490E0A1966EAD7FADA197689FA9
:10BF1000F001699FF00D789FF00D1124EB5CF64F56
:10BF2000DF011C96248711963C93119712964C932F
:10BF3000129713965C936080718082809380A480B6
:10BF4000B580C680D780E084F18402851385C9015D
:10BF5000DA018E159F05A007B10714F4D801C701B7
:10BF60008A159B05AC05BD0514F4D601C5019C01DD
:10BF7000AD0186159705A805B90514F4A401930130
:10BF80008DE490E0A196AEADBFADA197A89FB001A2
:10BF9000A99F700DB89F700D11246B5C764FFB014B
:10BFA000208B318B428B538B263031054105510557
:10BFB00010F40C94C568E85BFF4F8091650690E033
:10BFC000A0E0B0E080839183A283B383DB019096ED
:10BFD0001C92C158DF4F288139814A815B81CF573C
:10BFE000D0406F968CAD9DADAEADBFAD6F972817AD
:10BFF00039074A075B0724F481E0DB0190968C93B4
:10C00000CD57DF4F288139814A815B81C358D040A9
:10C0100067966CAD7DAD8EAD9FAD679726173707E0
:10C020004807590794F48DE490E0A196AEADBFADFA
:10C03000A197A89FF001A99FF00DB89FF00D1124C2
:10C04000EB5CF64F80A1826080A3C957DF4F288147
:10C0500039814A815B81C758D0402F966CAD7DAD48
:10C060008EAD9FAD2F97261737074807590794F4D1
:10C070008DE490E0A196AEADBFADA197A89FF00171
:10C08000A99FF00DB89FF00D1124EB5CF64F80A135
:10C09000846080A3C557DF4F288139814A815B8145
:10C0A000CB58D040221533054405550594F48DE452
:10C0B00090E0A1964EAD5FADA197489FF001499FDA
:10C0C000F00D589FF00D1124EB5CF64F80A18860B5
:10C0D00080A38DE490E0A1966EAD7FADA197689F9F
:10C0E000F001699FF00D789FF00D1124EB5CF64F85
:10C0F000E396AEADBFADE3978C9181A320813181F2
:10C100004281538125962CAF3DAF4EAF5FAF25974F
:10C11000211531054105510509F015988DE490E090
:10C12000A1964EAD5FADA197489FF001499FF00DDC
:10C13000589FF00D1124EB5CF64F6480758086806B
:10C140009780611471048104910409F046988DE48C
:10C1500090E0A1966EAD7FADA197689FF001699FB9
:10C16000F00D789FF00D1124EB5CF64FA084B184A4
:10C17000C284D384A114B104C104D10409F043984A
:10C180008DE490E0A196AEADBFADA197A89FF00160
:10C19000A99FF00DB89FF00D1124EB5CF64F84853C
:10C1A0009585A685B7850097A105B10551F0409802
:10C1B0002090F9083090FA084090FB085090FC0855
:10C1C00008C0209011093090120940901309509036
:10C1D0001409CB56DF4F6881C559D040CA56DF4F8E
:10C1E0007881C659D040C956DF4F8881C759D040A1
:10C1F000C856DF4F9881C859D040A20191010E94D2
:10C200002BCC87FD16C0CB56DF4F8881C559D04057
:10C21000CA56DF4F9881C659D040C956DF4FA88112
:10C22000C759D040C856DF4FB881C859D0401C010B
:10C230002D016B966CAD7DAD8EAD9FAD6B970E9461
:10C24000CDCCE1962CAD3DAD4EAD5FADE1970E94FA
:10C2500032CCEC966FAFEC97ED967FAFED97EE9604
:10C260008FAFEE97EF969FAFEF97AC01CB01DA015E
:10C2700089839A83AB83BC8363966CAD7DAD8EADB1
:10C280009FAD63970E94CDCCAD962CAD3DAD4EAD2C
:10C290005FADAD970E9432CCE8966FAFE897E99614
:10C2A0007FAFE997EA968FAFEA97EB969FAFEB9750
:10C2B000AC01CB01DA018D839E83AF83B8872B96C7
:10C2C0006CAD7DAD8EAD9FAD2B970E94CDCCA99668
:10C2D0002CAD3DAD4EAD5FADA9970E9432CCE4963A
:10C2E0006FAFE497E5967FAFE597E6968FAFE69759
:10C2F000E7969FAFE797AC01CB01DA0189879A8770
:10C30000AB87BC876DA17EA18FA198A50E94CDCCE3
:10C31000A5962CAD3DAD4EAD5FADA5970E9432CC3C
:10C320007B018C012796EEADFFAD2797BF018827D3
:10C3300077FD8095982F0E94CDCC9B01AC01C80160
:10C34000B7010E9400CF20E030E048EC52E40E94A8
:10C3500032CC9B01AC016D877E878F87988B2596A9
:10C360006CAD7DAD8EAD9FAD2597663071058105B5
:10C3700091051CF576E06716710481049104ECF4D4
:10C3800086E0A816B104C104D104BCF48DE490E0A9
:10C39000A196AEADBFADA197A89FF001A99FF00DEA
:10C3A000B89FF00D1124EB5CF64FDA01C901BF779D
:10C3B00086A797A7A0ABB1AB55C0EC962FADEC9775
:10C3C000ED963FADED97EE964FADEE97EF965FADE4
:10C3D000EF97B901CA010E94ABCF3B014C01E8962F
:10C3E0002FADE897E9963FADE997EA964FADEA970A
:10C3F000EB965FADEB97B901CA010E94ABCF5B0131
:10C400006C01E4962FADE497E5963FADE597E6968F
:10C410004FADE697E7965FADE797B901CA010E9475
:10C42000ABCF7B018C01C401B301A60195010E9431
:10C4300052CBA80197010E9452CB0E946DCF2DE4F0
:10C4400030E0A1964EAD5FADA197429FF001439FB2
:10C45000F00D529FF00D1124EB5CF64F66A777A705
:10C4600080AB91AB8DE490E0A1966EAD7FADA197CE
:10C47000689FF001699FF00D789FF00D1124EB5C2F
:10C48000F64F86A597A5A0A9B1A921968CAF9DAF1F
:10C49000AEAFBFAF219760E070E080E89FE32196E8
:10C4A0002CAD3DAD4EAD5FAD21970E9432CC9B01CE
:10C4B000AC01C201B1010E9400CF2B013C0180916F
:10C4C000050E9091060EA82FB0E05096A91BB10959
:10C4D000AF70B070BAA7A9A7A230B1050CF451C0D3
:10C4E0005D01CC24B7FCC094DC2CC601B5010E94D0
:10C4F000CDCC20E030E040E051E40E942BCC8823FA
:10C500000CF03FC060E074E284E799E4A30192017B
:10C510000E9432CC0E94D0CE7B018C016091C50874
:10C520007091C6088091C7089091C808E616F70672
:10C530000807190730F56E197F09800B910B660FFC
:10C54000771F881F991FA60195010E94F5D2CA0185
:10C55000B9010E94CBCC0E94D0CE9B01AC012E0D24
:10C560003F1D401F511FCA01B9010E94CBCC9B0146
:10C57000AC0160E074E284E799E40E9432CC2B01C4
:10C580003C018DE490E0A196EEADFFADA197E89F50
:10C590008001E99F100DF89F100D11240B5C164FC0
:10C5A00021966CAD7DAD8EAD9FAD2197A30192011B
:10C5B0000E9400CFD80192966D937D938D939C93AA
:10C5C000959750966D917D918D919C9153970E9476
:10C5D000CBCCA30192010E9400CF0E9418CC0E94F4
:10C5E0009FCCF80160AF71AF82AF93AFC157DF4FFF
:10C5F0001882CF58D040C057DF4F1882C059D04062
:10C6000020E8222E9FE3392E88249924E1E0F0E0EF
:10C61000EC0FFD1FE80DF91DC301B201208131812E
:10C62000428153810E9400CFE1E1F0E0EC0FFD1F59
:10C63000E80DF91D60837183828393835B016C0134
:10C64000E894D7F8F401E753F74FE080F1800281D6
:10C650001381C601B501A80197010E942ECE1816BC
:10C66000CCF4C801B701A60195010E9432CC6B0140
:10C670007C01C157DF4F6881CF58D040C057DF4F92
:10C680007881C059D040C101A70196010E942BCCEE
:10C6900088236CF4C157DF4F8881CF58D040C057F2
:10C6A000DF4F9881C059D040D1016C017D0124E059
:10C6B00030E0820E931E30E18316910471F0D701B1
:10C6C000C601C157DF4FC882CF58D040C057DF4F97
:10C6D0009883C059D0401D0199CFC701B60120E011
:10C6E00030E040E85FE30E942BCC88230CF04CC084
:10C6F0008E010F5E1F4F81E2A82EB12CAC0EBD1E25
:10C70000D8016D917D918D919C91A70196010E9418
:10C7100000CFF80161937193819391938F01EA1592
:10C72000FB0571F78DE490E0A1962EAD3FADA1978A
:10C73000289F8001299F100D389F100D11240B5C3C
:10C74000164FD80192966D917D918D919C91959700
:10C75000A70196010E9400CFF80162A373A384A3EE
:10C7600095A360AD71AD82AD93AD0E94CBCCA70116
:10C7700096010E9400CF0E949FCCD801D8966D935D
:10C780007D938D939C93DB978DE490E0A196EEAD25
:10C79000FFADA197E89F8001E99F100DF89F100D54
:10C7A00011240B5C164FD80150966D917D918D919F
:10C7B0009C9153970E94CBCCF80126A537A540A9A0
:10C7C00051A90E9432CC1B012C01F801808191817A
:10C7D000A281B3810097A105B10549F584819581B6
:10C7E000A681B7810097A105B10509F580859185DE
:10C7F000A285B3850097A105B105C9F4C201B101B5
:10C8000020910109309102094091030950910409D6
:10C810000E9400CF0E9418CC0C5B1F4F0E949FCC3F
:10C82000D8016D937D938D939C93139771C1C20131
:10C83000B1012091FD083091FE084091FF08509110
:10C8400000090E9400CF0E9418CC0E949FCC2DE4CA
:10C8500030E0A196EEADFFADA197E29F6001E39FAE
:10C86000D00CF29FD00C112425E339E0C20ED31E68
:10C87000B4E46B2E712C6C0C7D1CD3016D937D93F5
:10C880008D939C9313978090150990901609A09012
:10C890001709B09018090E94CBCC7B018C01F601DE
:10C8A00060817181828193810E94CDCC9B01AC011A
:10C8B000C801B7010E9400CF7B018C01D6015096C0
:10C8C0006D917D918D919C9153970E94CBCC9B0152
:10C8D000AC01C801B7010E9432CC7B018C01C501BB
:10C8E000B4010E94CBCC9B01AC01C801B7010E94EE
:10C8F0002ECE18162CF4F30180829182A282B3828C
:10C900008090190990901A09A0901B09B0901C09F9
:10C910008DE490E0A1962EAD3FADA197289F6001D8
:10C92000299FD00C389FD00C112445E359E0C40E48
:10C93000D51EA4E46A2E712C6C0C7D1CD3016D9164
:10C940007D918D919C910E94CBCC7B018C01F60155
:10C9500064817581868197810E94CDCC9B01AC0159
:10C96000C801B7010E9400CF7B018C01D60150960F
:10C970006D917D918D919C9153970E94CBCC9B01A1
:10C98000AC01C801B7010E9432CC7B018C01C5010A
:10C99000B4010E94CBCC9B01AC01C801B7010E943D
:10C9A0002ECE18162CF4F30180829182A282B382DB
:10C9B0008090210990902209A0902309B090240929
:10C9C0008DE490E0A1962EAD3FADA197289F600128
:10C9D000299FD00C389FD00C112445E359E0C40E98
:10C9E000D51EF4E46F2E712C6C0C7D1CD3016D915F
:10C9F0007D918D919C910E94CBCC7B018C01F601A5
:10CA000064857585868597850E94CDCC9B01AC0198
:10CA1000C801B7010E9400CF7B018C01D60150965E
:10CA20006D917D918D919C9153970E94CBCC9B01F0
:10CA3000AC01C801B7010E9432CC7B018C01C50159
:10CA4000B4010E94CBCC9B01AC01C801B7010E948C
:10CA50002ECE18162CF4F30180829182A282B3822A
:10CA600080901D0990901E09A0901F09B090200988
:10CA70008DE490E0A1962EAD3FADA197289F600177
:10CA8000299FD00C389FD00C112445E359E0C40EE7
:10CA9000D51EE4E46E2E712C6C0C7D1CD3016D91BF
:10CAA0007D918D919C910E94CBCC7B018C01F601F4
:10CAB00060857185828593850E94CDCC9B01AC01F8
:10CAC000C801B7010E9400CF7B018C01D6015096AE
:10CAD0006D917D918D919C9153970E94CBCC9B0140
:10CAE000AC01C801B7010E9432CC7B018C01C501A9
:10CAF000B4010E94CBCC9B01AC01C801B7010E94DC
:10CB00002ECE18162CF4F30180829182A282B38279
:10CB10008DE490E0A1962EAD3FADA197289F6001D6
:10CB2000299FD00C389FD00C112445E359E0C40E46
:10CB3000D51EF601EC5BFF4F60817181828193818C
:10CB40000E94CBCC7B018C01A20191010E9432CCCE
:10CB5000D601D2966D937D938D939C93D597C80102
:10CB6000B7012DEB37E346E051E40E9400CF0E946D
:10CB70009ACCF601648F758F868F978F6090050928
:10CB8000709006098090070990900809C401B301CC
:10CB900020E030E040E05FE30E9400CF5B016C01E9
:10CBA000298D3A8D4B8D5C8D29AF3AAF4BAF5CAF81
:10CBB0004091090950910A0960910B0970910C0983
:10CBC0004DAB5EAB6FAB78AFCB01BA0120E030E08C
:10CBD00040E05FE30E9400CF7B018C0169AD7AAD3C
:10CBE0008BAD9CAD9F77A80197010E942ECE1816A1
:10CBF00044F4C601B501A80197010E942BCC8823FB
:10CC000014F4860175016D8D7E8D8F8D98A169ABB1
:10CC10007AAB8BAB9CAB80910D0990910E09A091E2
:10CC20000F09B09110098DA79EA7AFA7B8ABBC01A3
:10CC3000CD0120E030E040E05FE30E9400CF1B0127
:10CC40002C0169A97AA98BA99CA99F77A2019101BE
:10CC50000E942ECE181644F4C801B701A20191011A
:10CC60000E942BCC882314F4170128018DE490E056
:10CC7000A196AEADBFADA197A89FF001A99FF00D01
:10CC8000B89FF00D1124EB5CF64F22A133A144A113
:10CC900055A129A33AA34BA35CA3C201B1010E94F1
:10CCA0002BCC87FD04C029A03AA04BA05CA049A5CD
:10CCB0005AA5423051050CF405C15091070ECF56CC
:10CCC000DF4F5883C159D0406091080ECE56DF4FD8
:10CCD0006883C259D0407091090ECD56DF4F7883DA
:10CCE000C359D04080910A0ECC56DF4F8883C45977
:10CCF000D040652FCE56DF4F7881C259D040CD56F7
:10CD0000DF4F8881C359D040CC56DF4F9881C4593A
:10CD1000D04027E137EB41ED58E30E942ECE1816A4
:10CD20000CF0D0C069897A898B899C8920910B0E7F
:10CD300030910C0E40910D0E50910E0E0E9451CB71
:10CD40009B01AC010E9400CF7B018C016D897E8923
:10CD50008F89988D20910F0E3091100E4091110EF9
:10CD60005091120E0E9451CB9B01AC010E9400CF4A
:10CD70009B01AC01C801B7010E9452CB0E946DCF4C
:10CD80007B018C01A40193010E942ECE18165CF049
:10CD90000F2EF0E06F2EF0E07F2EF0E88F2EFFE3F5
:10CDA0009F2EF02D08C0C401B301A80197010E9475
:10CDB00032CC3B014C0169AD7AAD8BAD9CAD20917D
:10CDC000130E3091140E4091150E5091160E0E94C4
:10CDD00051CB7B018C01E89417F9C801B7012DA94B
:10CDE0003EA94FA958AD0E942ECE181694F46DA9F5
:10CDF0007EA98FA998ADA80197010E9432CC5B0152
:10CE00006C01C401B301A60195010E942BCC8823BB
:10CE100014F46401530169A97AA98BA99CA92091F2
:10CE2000170E3091180E4091190E50911A0E0E9453
:10CE300051CB7B018C01E89417F9C801B7012DA5EE
:10CE40003EA54FA558A90E942ECE181694F46DA5A4
:10CE50007EA58FA598A9A80197010E9432CC7B01DD
:10CE60008C01C601B501A80197010E942BCC882333
:10CE700014F48601750169A17AA18BA19CA1A80176
:10CE800097010E9400CF7B018C01CF56DF4F688154
:10CE9000C159D040CE56DF4F7881C259D040CD56CF
:10CEA000DF4F8881C359D040CC56DF4F9881C45999
:10CEB000D040A80197010E942BCC87FD19C0D80152
:10CEC000C70102C0D201C101CF56DF4F8883C159CB
:10CED000D040CE56DF4F9883C259D040CD56DF4F59
:10CEE000A883C359D040CC56DF4FB883C459D04033
:10CEF0008DE490E0A196AEADBFADA197A89F800153
:10CF0000A99F100DB89F100D11240B5C164FCF5622
:10CF1000DF4F8881C159D040CE56DF4F9881C2592A
:10CF2000D040CD56DF4FA881C359D040CC56DF4FFB
:10CF3000B881C459D040F80182A793A7A4A7B5A788
:10CF400062A973A984A995A9905820E030E040E037
:10CF500050EC0E9400CFD8019E962D913D914D91AD
:10CF60005C91D1970E9400CF2BE037ED43E25BE369
:10CF70000E9452CB0E946DCFF62EE72ED82EC92EDE
:10CF8000CF56DF4F6881C159D040CE56DF4F7881F0
:10CF9000C259D040CD56DF4F8881C359D040CC56BE
:10CFA000DF4F9881C459D0402F2D3E2D4D2D5C2D43
:10CFB0000E942BCC87FD14C0CF56DF4FF882C15999
:10CFC000D040CE56DF4FE882C259D040CD56DF4F19
:10CFD000D882C359D040CC56DF4FC882C459D04004
:10CFE0008DE490E0A196EEADFFADA197E89F8001A2
:10CFF000E99F100DF89F100D11240B5C164FCF56B2
:10D00000DF4F8881C159D040CE56DF4F9881C25939
:10D01000D040CD56DF4FA881C359D040CC56DF4F0A
:10D02000B881C459D040F80186A397A3A0A7B1A79F
:10D0300062A173A184A195A12F2D3E2D4D2D5C2DB4
:10D040000E942BCC18162CF081E0D801D7968C9337
:10D0500002C0F80117AA8DE490E0A1962EAD3FAD75
:10D06000A197289FF001299FF00D389FF00D112402
:10D07000EB5CF64F81E086ABABE0BEE0FE01719663
:10D0800080E101900D928150E1F78DE490E0A1964E
:10D090004EAD5FADA197489F6001499FD00C589F4E
:10D0A000D00C112465E379E0C60ED71ED601929606
:10D0B000ED90FD900D911C919597E092070EF092E6
:10D0C000080E0093090E10930A0E96966D917D91AD
:10D0D0008D919C919997A80197010E9432CC4B01A8
:10D0E0005C01C201B101A80197010E9432CC8B0101
:10D0F0009C01C601B501A4010E94015ABBA5B093D1
:10D10000050EC557DF4F288139814A815B81CB5895
:10D11000D040209331093093320940933309509322
:10D120003409C957DF4F488159816A817B81C758CB
:10D13000D04040932D0950932E0960932F0970938E
:10D140003009CD57DF4F688179818A819B81C3582F
:10D15000D0406093290970932A0980932B099093FA
:10D160002C09C158DF4F88819981AA81BB81CF5793
:10D17000D0408093250990932609A0932709B09366
:10D1800028090E94895C0E94FF79C856DF4F0FB6BC
:10D19000F894DEBF0FBECDBFCF91DF911F910F91ED
:10D1A000FF90EF90DF90CF90BF90AF909F908F90C7
:10D1B0007F906F905F904F903F902F900895FF92D7
:10D1C0000F931F93CF93DF938B010E94DE19EB0126
:10D1D000FF24FA9409C00E94DE196C1B7D0B6017B6
:10D1E000710710F080E008C0FEBC0DB407FEFDCF53
:10D1F0008EB58F3F81F781E0DF91CF911F910F9125
:10D20000FF900895FC014281242F30E0C9019595DB
:10D21000879580658CBD40FF02C080E004C080E03F
:10D22000463009F081E08DBD808160E00C94DF1B09
:10D23000DF92EF92FF920F931F93CF93DF93EC0156
:10D24000D62E79018A01DEDFCE016CE271E0B7DF14
:10D250008D2D80648EBD0DB407FEFDCF28E130E03A
:10D26000D801C701022E04C0B695A795979587955A
:10D270000A94D2F78EBD0DB407FEFDCF2850304082
:10D280008FEF283F380761F7DD2011F485E906C0EC
:10D2900088E0D81611F487E801C08FEF8EBD0DB479
:10D2A00007FEFDCF8CE0D81631F48FEF8EBD0DB4A4
:10D2B00007FEFDCF8EB59FEF2FEF2EBD0DB407FEFD
:10D2C000FDCF8EB587FF04C0992311F09150F5CFA3
:10D2D0008B83DF91CF911F910F91FF90EF90DF90A3
:10D2E0000895FC01808161E00C94DF1BDC016EBDC0
:10D2F000FA0120E030E00DB407FEFDCF80818EBD45
:10D300000DB407FEFDCF81818EBD2E5F3F4F32965B
:10D3100082E02030380779F70DB407FEFDCF8FEF9C
:10D320008EBD0DB407FEFDCF8FEF8EBD0DB407FE91
:10D33000FDCF8FEF8EBD0DB407FEFDCF8EB51396DA
:10D340008C9313978F71853011F481E0089583E1F8
:10D3500011968C931197CD01C4DF80E00895CF9290
:10D36000DF92EF92FF920F931F93CF93DF93EC0125
:10D370007A018B0169018C81833039F059E0EE0C20
:10D38000FF1C001F111F5A95D1F7CE0168E1A801BB
:10D3900097014EDF882311F086E020C0CE016EEFAA
:10D3A000A601A4DF8823D9F0CE0168E572E007DF8B
:10D3B000882311F487E112C0CE016DE020E030E057
:10D3C00040E050E035DF882341F48FEF8EBD0DB48F
:10D3D00007FEFDCF8EB5882371F086E18983CE01EB
:10D3E00080DF80E0DF91CF911F910F91FF90EF9050
:10D3F000DF90CF900895CE0174DF81E0F3CFBF922C
:10D40000CF92DF92EF92FF920F931F93CF93DF9310
:10D41000EC016B018A010E94DE197B01BB24BA94E6
:10D4200009C00E94DE196E197F096D52714010F01B
:10D4300081E15FC0BEBC0DB407FEFDCF8EB58B830E
:10D440008F3F79F38E3F11F08FE053C0D8011197D1
:10D4500001151105D9F08FEF8EBD20E030E09FEF70
:10D460000BC00DB407FEFDCF8EB5F601E20FF31F22
:10D4700080839EBD2F5F3F4F2A173B0790F30DB46B
:10D4800007FEFDCF8EB5AC0DBD1D8C9340E050E086
:10D4900060E070E016C0272F3327F601E40FF51F78
:10D4A000808190E028273927220F331F2F53354FD3
:10D4B000F90185919491762F6627682779274F5F28
:10D4C0005F4F4017510738F38FEF8EBD0DB407FE45
:10D4D000FDCF3EB58FEF8EBD0DB407FEFDCF2EB54F
:10D4E000932F80E030E0822B932B6817790731F07F
:10D4F00080E28983CE01F5DE80E003C0CE01F1DE5B
:10D5000081E0DF91CF911F910F91FF90EF90DF901D
:10D51000CF90BF900895AF92BF92DF92EF92FF92AB
:10D520000F931F93CF93DF93EC017A018B01590185
:10D530008C81833039F099E0EE0CFF1C001F111F25
:10D540009A95D1F783E0D82EDA94CE0161E1A80153
:10D5500097016EDE882329F0DD2071F484E0898351
:10D5600016C0CE01B50140E052E049DF882311F03A
:10D5700081E010C0DD2059F0CE01B3DECE016CE0B9
:10D5800020E030E040E050E053DE1982DDCFCE01F4
:10D59000A8DE80E0DF91CF911F910F91FF90EF9077
:10D5A000DF90BF90AF900895BF92CF92DF92EF923D
:10D5B000FF920F931F93CF93DF93EC01B62E1C8243
:10D5C000198248830E94DE196B01888161E00E9404
:10D5D0002C1BCE0186DE82E360E00E942C1B83E3DD
:10D5E00061E00E942C1B84E361E00E942C1B85E318
:10D5F00061E00E942C1B85E361E00E94DF1B85E057
:10D600008A8382E58CBD1DBC80E09FEF9EBD0DB47A
:10D6100007FEFDCF8F5F8A30C9F709C00E94DE196F
:10D620006C197D09615D774010F081E059C0CE0131
:10D6300060E020E030E040E050E0FADD182F8B831E
:10D64000813061F7CE0168E02AEA31E040E050E045
:10D65000EFDD82FF02C01C8311C080E02FEF2EBDE2
:10D660000DB407FEFDCF9EB58F5F8430C1F79B835D
:10D670009A3A11F082E034C082E08C838C8182304F
:10D6800021F0EE24FF2487010FC0E12CF12C012DA5
:10D6900040E4142F09C00E94DE196C197D09615DF8
:10D6A000774010F08AE01CC0CE0167E320E030E054
:10D6B00040E050E0BDDDCE0169E2A8019701B8DD90
:10D6C0008B83882341F78C81823019F5CE016AE380
:10D6D00020E030E040E050E0ABDD882329F088E036
:10D6E0008983CE01FEDD20C08FEF8EBD0DB407FE15
:10D6F000FDCF8EB5807C803C11F483E08C8380E08C
:10D700009FEF9EBD0DB407FEFDCF2EB58F5F83301A
:10D71000C1F7CE01E6DD86E08B1518F488E1898338
:10D7200003C0BA8281E001C080E0DF91CF911F91F8
:10D730000F91FF90EF90DF90CF90BF900895CF931F
:10D74000DF93DC01EB01BA0180E090E020E2FE0112
:10D75000E80FF91F208301968B309105C1F757E040
:10D7600040E022C02E3219F081EC9CE007C05A3014
:10D7700049F15AE048E017C0321721F1FC01019647
:10D7800034913323C9F75417E8F02132D8F02F37FA
:10D79000C8F4822F81568A3108F42052FE01E40F2A
:10D7A000F11D20834F5F11962C91222311F02F320F
:10D7B000C9F6FB01B183A08390E08881803219F023
:10D7C00091E001C090E0892FDF91CF9108956F9291
:10D7D0007F928F929F92AF92BF92CF92DF92EF9201
:10D7E000FF920F931F93CF93DF93EC017A018B018C
:10D7F0002B81222309F480C089899A89AB89BC894D
:10D8000084179507A607B70708F476C085C0E1140A
:10D81000F1040105110551F41C821D821E821F8234
:10D82000188619861A861B8681E067C02885398587
:10D830004A855B85E98DFA8D858590E009962150B2
:10D8400030404040504039014A01082E04C09694AF
:10D850008794779467940A94D2F72F5F3F4F4F4F86
:10D860005F4F0894E108F1080109110957016801A7
:10D8700004C0D694C794B794A7948A95D2F7089415
:10D88000E11CF11C011D111DA614B704C804D90424
:10D8900028F0211531054105510549F48D899E89EE
:10D8A000AF89B88D8C839D83AE83BF8316C0A618C5
:10D8B000B708C808D90811C04C815D816E817F818D
:10D8C000898D9A8D94010E94AE770894A108B108C1
:10D8D000C108D108882331F40FC084E0882E912C30
:10D8E0008C0E9D1EA114B104C104D10429F7E88651
:10D8F000F9860A871B8798CF80E0DF91CF911F912F
:10D900000F91FF90EF90DF90CF90BF90AF909F90DE
:10D910008F907F906F900895223009F078CFE7CFF5
:10D92000CF93DF93EC018C859D85AE85BF8540E06C
:10D93000611141E0BC01CD010E948875882319F472
:10D9400020E030E00AC08889282F30E095E0220FDF
:10D95000331F9A95E1F72F5D314FC901DF91CF91C8
:10D9600008950F931F93CF93DF938C01FC01838164
:10D970008823E9F1818187FF37C0C80161E0D0DFEA
:10D98000EC010097A1F18881853E89F1F80183813E
:10D99000823040F481899289A389B4898C8F9D8FCC
:10D9A000AE8FBF8FF801858996899B8F8A8F858975
:10D9B0009689A789B08DCD01AA27BB279D8B8C8B1B
:10D9C000E0911B0EF0911C0E309751F0BE016A5E83
:10D9D0007F4FCE0148961995888D998D9B8B8A8BA8
:10D9E000F80181818F7781830E944D7504C081E0A9
:10D9F000F801808380E0DF91CF911F910F9108950E
:10DA00000F931F938C01ADDFF80113821F910F91CB
:10DA10000895FC018381882311F0CF01F1CF08958F
:10DA20006F927F928F929F92AF92BF92CF92DF922E
:10DA3000EF92FF920F931F93DF93CF9300D00F923B
:10DA4000CDB7DEB77C015A016B01DC0113968C91D6
:10DA50001397813009F08EC011968C9181FF8AC096
:10DA60009DC00097A105B10511F481E084C0F701C4
:10DA70006084718482849384C701B601A501A7DE06
:10DA8000882309F477C0D70159968D919C915A97B4
:10DA9000A114B104C104D10489F455964D915D914E
:10DAA0006D917C9158970E942378882309F462C075
:10DAB000F701158A168A178A108E44C0D70114966A
:10DAC0004D915D916D917C9117979E012F5F3F4F16
:10DAD0000E94AE77882309F44DC0D7015996ED9185
:10DAE000FC915A9749815A816B817C818789803169
:10DAF00049F4483FBFEF5B07B0E06B07B0E07B073E
:10DB000048F020C0483F8FEF58078FEF68078FE03D
:10DB10007807C0F4CF010E942378882359F1D701F8
:10DB200014964D915D916D917C91179759968D91B9
:10DB30009C915A970FEF1FEF2FEF3FE00E9428773D
:10DB40008823C1F0F701A18AB28AC38AD48A81816D
:10DB500080688183C70105DF882361F0B601A501D4
:10DB60006A147B048C049D0410F4B401A301C70162
:10DB70002EDE01C080E00F900F900F900F90CF919C
:10DB8000DF911F910F91FF90EF90DF90CF90BF90AA
:10DB9000AF909F908F907F906F900895F70181894B
:10DBA0009289A389B48984179507A607B70708F057
:10DBB00058CFE0CFCF93DF93EC0140E050E060E03E
:10DBC00070E02EDF882359F0CE0161E0A9DEFC0170
:10DBD000009729F085EE80831B825FD701C080E02B
:10DBE000DF91CF9108952F923F924F925F926F9263
:10DBF0007F928F929F92AF92BF92CF92DF92EF92DD
:10DC0000FF920F931F93CF93DF93EC012A018B8137
:10DC1000882309F4B5C0898180FFB2C0C7C025013F
:10DC20004E185F083B0174E0272E312C2C0E3D1E50
:10DC30004201A0C0288539854A855B856FEFA62EF5
:10DC400061E0B62EA222B3228B8179018A0199E08C
:10DC500016950795F794E7949A95D1F7E98DFA8D83
:10DC6000823049F4428D538D648D758D4E0D5F1D4C
:10DC7000601F711F3FC0D480DA94DE20A114B1046C
:10DC8000D9F4DD20C9F4211531054105510549F4C8
:10DC90008D899E89AF89B88D8C839D83AE83BF8328
:10DCA0000BC04C815D816E817F81CF0191010E940B
:10DCB000AE77882309F464C0E98DFA8D4C815D81CB
:10DCC0006E817F814250504060407040058404C0A6
:10DCD000440F551F661F771F0A94D2F786859785D4
:10DCE000A089B189480F591F6A1F7B1F4D0D511D17
:10DCF000611D711D80E092E08A199B0984018815DD
:10DD0000990508F48C0182E00030180709F066C01C
:10DD100080911D0E90911E0EA0911F0EB091200EAD
:10DD2000481759076A077B0709F458C080912110EA
:10DD3000909122109301EFDB882349F421C09501D3
:10DD40002F5D314FC301B901A8010E94B8CA600E0E
:10DD5000711E980140E050E088859985AA85BB85B1
:10DD6000820F931FA41FB51F88879987AA87BB8737
:10DD7000801A910A8114910409F05CCFA20102C0BB
:10DD80004FEF5FEFCA01DF91CF911F910F91FF908D
:10DD9000EF90DF90CF90BF90AF909F908F907F904B
:10DDA0006F905F904F903F902F900895A988BA8808
:10DDB000CB88DC88E884F9840A851B859A0140E0D9
:10DDC00050E0D601C5018E199F09A00BB10B281791
:10DDD00039074A075B0708F022CF24CFCB01BA01ED
:10DDE00040E096D6882309F0AACFCACFCF92DF921F
:10DDF000EF92FF920F931F93CF93DF937C01EB0180
:10DE00008A01FC018381823008F46EC0808591858F
:10DE1000A285B3858F719070A070B0700097A10536
:10DE2000B10509F061C06CC0F8011082EDE0CE2EA2
:10DE3000D12CC701BE0140E250E0D5DE9C0180320A
:10DE4000910521F0009709F04FC050C0488144234C
:10DE500009F44CC0453E69F34E3259F38B858F73FC
:10DE60008F30E9F501151105D1F18A8D9B8D892B34
:10DE7000B1F5842F90E08F719070009781F183301D
:10DE800091056CF58C9D90018D9D300D9C9D300D04
:10DE900011242D503040F801E20FF31F8981808357
:10DEA0008B8181838D8182838F8183838985848324
:10DEB0008E858583888986838A8987838C898087F4
:10DEC0008E898187888D82878C8D83878E8D8487CC
:10DED000888186FF04C0F801E20FF31F15868B8549
:10DEE00083FDA7CF822F03C08FEF01C080E0DF91B9
:10DEF000CF911F910F91FF90EF90DF90CF900895F9
:10DF00004115510509F090CF91CFDF93CF930F9238
:10DF1000CDB7DEB7BE016F5F7F4F41E050E063DEFB
:10DF2000019719F02FEF3FEF03C08981282F30E0D0
:10DF3000C9010F90CF91DF910895EF92FF920F9357
:10DF40001F93CF93DF93EC018B81823030F1E88413
:10DF5000F9840A851B85CE01D8DF97FD1EC0888510
:10DF60009985AA85BB854F96A11DB11D8887998784
:10DF7000AA87BB87A5E016950795F794E794AA951D
:10DF8000D1F72E2D30E02F703070F5E0220F331FC7
:10DF9000FA95E1F72F5D314F02C020E030E0C90172
:10DFA000DF91CF911F910F91FF90EF9008950F9304
:10DFB0001F93CF93DF93EC018B018B81882309F0B2
:10DFC00040C0FB018789803109F041C082E08B832A
:10DFD0001D8A1E8A1F8A188E808D918DA0E0B0E068
:10DFE00045E0880F991FAA1FBB1F4A95D1F7898B5F
:10DFF0009A8BAB8BBC8B13C083E08B83F801428D73
:10E00000538D648D758D4D8B5E8B6F8B788F9E01DC
:10E010002F5E3F4FC8010E947F78882391F01A8FAE
:10E02000098F81E089831C821D821E821F821886CF
:10E0300019861A861B861C861D861E861F86188AD0
:10E0400001C080E0DF91CF911F910F910895803240
:10E05000C1F7D2CF1F93CF93DF93EC01142F262F5C
:10E0600030E0F90175E0EE0FFF1F7A95E1F7EF5D03
:10E07000F14F8385817121F0842F827109F066C090
:10E0800080911D0E90911E0EA0911F0EB091200E3A
:10E090008C879D87AE87BF87688BF90165E0EE0F9F
:10E0A000FF1F6A95E1F7EF5DF14F84899589A0E044
:10E0B000B0E0DC01992788278D8B9E8BAF8BB88FC2
:10E0C000228D338DA90160E070E0482B592B6A2B1B
:10E0D0007B2B4D8B5E8B6F8B788F838590E0887167
:10E0E0009070009751F4848D958DA68DB78D898B96
:10E0F0009A8BAB8BBC8B81E00BC0409739F59E01AE
:10E100002F5E3F4F898D9A8DFAD78823F9F084E0EE
:10E110008B83812F8F7089831C821D821E821F82B8
:10E12000188619861A861B8614FF16C0CE0140E099
:10E1300050E060E070E074DC882371F409C0498924
:10E140005A896B897C89CE0142DB02C01B8280E048
:10E15000DF91CF911F91089515FDF1CF81E0F8CFA8
:10E160002F923F924F925F926F927F928F929F92E7
:10E17000AF92BF92CF92DF92EF92FF920F931F93D5
:10E18000DF93CF930F92CDB7DEB72C015B013A013D
:10E19000490100E010E0EE24EA94FE2C1E010894F0
:10E1A000211C311C11C00A0D1B1DF8016083811454
:10E1B000910419F46A3039F41BC0C40170E00E9464
:10E1C000CCCA0097A9F4860168010894C11CD11C2F
:10E1D000C614D7043CF5C201B10141E050E003DDB3
:10E1E0007C0181309105F1F469816D30E1F6ECCF6D
:10E1F0008601A00EB11EF5011082C8010F90CF91CB
:10E20000DF911F910F91FF90EF90DF90CF90BF9023
:10E21000AF909F908F907F906F905F904F903F90C6
:10E220002F900895F7FEE5CF0FEF1FEFE6CFCF93C6
:10E23000DF93EC019C012C5F3F4F898D9A8D41E06B
:10E2400050E060E070E0C6D78823A1F08D899E89F8
:10E25000AF89B88D0097A105B10559F48C819D81D6
:10E26000AE81BF818D8B9E8BAF8BB88F898180688B
:10E27000898381E0DF91CF9108952F923F924F9251
:10E280005F927F928F929F92AF92BF92CF92DF92D6
:10E29000EF92FF920F931F93DF93CF9300D000D0A4
:10E2A000CDB7DEB76C01162F072F5E834D83DC01DF
:10E2B00013968C911397813009F069C111968C9156
:10E2C00081FF65C182C1F6014189528963897489E0
:10E2D00080859185A285B38584179507A607B70722
:10E2E00029F0C60174DA882309F451C1812F902FD7
:10E2F0009C0119014D805E800FC1D6015996ED91A8
:10E30000FC915A97DA01C90149E0B695A79597950E
:10E3100087954A95D1F774807A9478228FEF882E6A
:10E3200081E0982E82229322772009F051C0811437
:10E33000910409F04DC0D60114964D915D916D91F7
:10E340007C911797411551056105710581F455962A
:10E350008D919D910D90BC91A02D0097A105B105C7
:10E3600059F1F60184839583A683B78331C0CF0129
:10E370009E012F5F3F4FF2D5882309F408C1298100
:10E380003A814B815C81D6015996ED91FC915A9767
:10E390008789803149F4283FBFEF3B07B0E04B0746
:10E3A000B0E05B0770F008C0283FEFEF3E07EFEFEB
:10E3B0004E07EFE05E0728F0C60139DF882341F4FD
:10E3C000E6C0D60114962D933D934D935C93179719
:10E3D00080E092E08819990952018415950508F4A6
:10E3E0005C01D6015996ED91FC915A971496ED90E7
:10E3F000FD900D911C9117978EEF9FEFAFEFBFEF40
:10E40000E80EF91E0A1F1B1F058404C0EE0CFF1C3A
:10E41000001F111F0A94D2F786859785A089B189BC
:10E42000E80EF91E0A1F1B1FE70CF11C011D111D30
:10E4300090E0A91692E0B90639F580911D0E9091F1
:10E440001E0EA0911F0EB091200E8E159F05A007E5
:10E45000B10771F4109223108FEF9FEFAFEFBFEF72
:10E4600080931D0E90931E0EA0931F0EB093200E4E
:10E470008091211090912210B801A70191010E9472
:10E48000AF698823A9F583C08114910411F5D601E1
:10E4900018962D913D914D915C911B9751968D91C0
:10E4A0009D910D90BC91A02D281739074A075B0755
:10E4B00080F0F3D2882309F46AC081E080932310AE
:10E4C000E0921D0EF0921E0E00931F0E1093200E70
:10E4D00007C0C801B70141E01BD3882309F457C026
:10E4E00094012F5D314FC901B101A5010E94B8CA45
:10E4F000950140E050E0F60180859185A285B385C5
:10E50000820F931FA41FB51F80879187A287B387AF
:10E510002A0C3B1C4A185B08D60118962D913D9198
:10E520004D915C911B974114510409F0E6CE519630
:10E530008D919D910D90BC91A02D82179307A407FA
:10E54000B50748F4F601218B328B438B548B8181C4
:10E550008068818311C080911B0E90911C0E892BC5
:10E5600059F08D819E81892B39F0D60111968C91BD
:10E570001197806811968C93F601818183FF04C006
:10E58000C601EFD9882319F04D815E8105C081E075
:10E59000D6018C934FEF5FEFCA0126960FB6F89421
:10E5A000DEBF0FBECDBFCF91DF911F910F91FF90C6
:10E5B000EF90DF90CF90BF90AF909F908F907F9023
:10E5C0005F904F903F902F90089582FD7CCE8ECE2D
:10E5D000DF92EF92FF920F931F93CF93DF93EC01A3
:10E5E00089899A89AB89BC89805E9F4FAF41B040D1
:10E5F00008F06FC0CE011BDE882309F46AC04DD23B
:10E60000882309F466C0E98DFA8DEC80FD800E81C7
:10E610001F818EEF9FEFAFEFBFEFE80EF91E0A1FCD
:10E620001B1F058404C0EE0CFF1C001F111F0A9461
:10E63000D2F786859785A089B189E80EF91E0A1F51
:10E640001B1F81E080932310E0921D0EF0921E0E9E
:10E6500000931F0E1093200E80E092E0E1E2FEE0B6
:10E66000DF019C011D9221503040E1F7DD24D3945D
:10E6700011C0B801A7014D0D511D611D711D809183
:10E6800021109091221021E23EE00E94AF69882380
:10E6900001F1D394E98DFA8D8481D81650F320E0EE
:10E6A00032E040E050E0058404C0220F331F441FD5
:10E6B000551F0A94D2F789899A89AB89BC89820F40
:10E6C000931FA41FB51F898B9A8BAB8BBC8B81E0EA
:10E6D00001C080E0DF91CF911F910F91FF90EF90EB
:10E6E000DF9008958F929F92AF92BF92CF92DF9268
:10E6F000EF92FF920F931F93CF93DF936C01EB0187
:10E70000942E852EA22E898D9A8DD6015A969C9391
:10E710008E935997CB0140E050E060E070E057D80D
:10E72000BB2437C0CE0109DCFC01009709F48FC07F
:10E7300055E016950795F794E7945A95D1F71E2D55
:10E740001F708081882311F0853EC9F4BB2099F4A5
:10E7500020911D0E30911E0E40911F0E5091200EE3
:10E76000D6011C962D933D934D935C931F97509625
:10E770001C93BB24B3948081882359F418C0892D3D
:10E78000982DBF014BE050E00E94ABCA009709F4FE
:10E790006CC0E884F9840A851B8589899A89AB89CC
:10E7A000BC89E816F9060A071B0708F4BBCFA6FECA
:10E7B0004EC0A1FE4CC0BB2049F0F6011089C60135
:10E7C00061E0AED8EC01009761F441C08B818230EA
:10E7D00009F43DC0CE01FCDE8823C9F110E0C1E29E
:10E7E000DEE080E2DE011D928A95E9F7DE01292D47
:10E7F000382DC901FC018BE001900D928150E1F7A9
:10E80000E0911B0EF0911C0E309739F0BE01625F53
:10E810007F4FCE014096199508C081E298E2998B0E
:10E82000888B80E098E09F878E87888999899B8B69
:10E830008A8B998F888F8E859F859F8B8E8B2DD10C
:10E84000882329F0C601612F4A2D04DC01C080E035
:10E85000DF91CF911F910F91FF90EF90DF90CF90BC
:10E86000BF90AF909F908F900895A7FEEBCFEFCF12
:10E870002F923F924F925F926F927F928F929F92D0
:10E88000AF92BF92CF92DF92EF92FF920F931F93BE
:10E89000DF93CF93CDB7DEB7C654D0400FB6F89410
:10E8A000DEBF0FBECDBF3C016B01DE01AE5BBF4FD3
:10E8B00011965C934E9325962FAF25971C861F8645
:10E8C0001FA21AA66115710509F47CC0FC018381A1
:10E8D000882309F077C0FA0180818F32F1F0860138
:10E8E000ECE0EE2EF12CEC0EFD1E72E4A72EB12C06
:10E8F000AC0EBD1E4E010894811C911C2796FFAEE4
:10E90000EEAE279767E2262E312C2C0E3D1E2701F6
:10E9100023C01196B183A08301C0FD01A081B18104
:10E920008C918F32B1F3D60113968C91139782504C
:10E930008230A8F28E01095D1F4F59966D917C912E
:10E940005A97C80134DB882359F63CC0342D252D55
:10E950008701832F922F7C01F50180819181B40181
:10E96000A5010E949F6B882329F42CC03196D50104
:10E97000ED93FC93D501ED91FC9180818F32B1F341
:10E980008823B9F0C701B801A40121E0ABDE8823D8
:10E99000C9F00C151D0511F0C80132D82796EEAD4F
:10E9A000FFAD2797EE16FF0689F6C101322D292FFC
:10E9B000CFCFC301B801A40125962FAD259792DED4
:10E9C000182F01C010E0CE01879623D8CE010C96F7
:10E9D00020D8812FCA5BDF4F0FB6F894DEBF0FBE81
:10E9E000CDBFCF91DF911F910F91FF90EF90DF90FE
:10E9F000CF90BF90AF909F908F907F906F905F90DF
:10EA00004F903F902F9008950F931F93DF93CF93D4
:10EA1000CDB7DEB76B970FB6F894DEBF0FBECDBF94
:10EA20009C01AB0119821C828E010F5F1F4FC80130
:10EA3000B90122E01DDF882311F410E003C0C801F2
:10EA4000B9D8182FCE0101960E94096D812F6B96BF
:10EA50000FB6F894DEBF0FBECDBFCF91DF911F91EF
:10EA60000F910895DB010D900020E9F71197A61B87
:10EA7000B70B0496AD0101CCDF93CF930F92CDB7C6
:10EA8000DEB769830496BE016F5F7F4F41E050E0BF
:10EA9000F4DB0F90CF91DF910895809123108823AC
:10EAA00099F140911D0E50911E0E60911F0E7091B4
:10EAB000200E809121109091221021E23EE00E94D0
:10EAC000AF69882319F1409124105091251060916D
:10EAD000261070912710411551056105710591F0BF
:10EAE000809121109091221021E23EE00E94AF69B6
:10EAF000882361F010922410109225101092261095
:10EB0000109227101092231081E0089580E008955C
:10EB1000DF92EF92FF920F931F937B018C01D42E13
:10EB200080911D0E90911E0EA0911F0EB091200E8F
:10EB30008E159F05A007B107B9F0AFDF8823E1F07C
:10EB40008091211090912210B801A70121E23EE0AE
:10EB50000E948B6A882381F0E0921D0EF0921E0EB7
:10EB600000931F0E1093200EDD2011F481E005C0EC
:10EB700081E08093231001C080E01F910F91FF90EE
:10EB8000EF90DF9008958F929F92AF92BF92CF92B5
:10EB9000DF92EF92FF920F931F93CF93DF936C015D
:10EBA000142F7093221060932110FC01178A82E0C9
:10EBB00090E0A0E0B0E080839183A283B3831092C1
:10EBC00023101092241010922510109226101092EB
:10EBD00027108FEF9FEFAFEFBFEF80931D0E909345
:10EBE0001E0EA0931F0EB093200E442321F4882400
:10EBF000992454013FC0453008F01CC160E070E02A
:10EC000080E090E040E084DF882309F413C1C12F45
:10EC1000D0E02197FE0174E0EE0FFF1F7A95E1F737
:10EC2000EF5DF14FE254FE4F8081EE5BF14090E0EA
:10EC30008F779070892B09F0FDC0E653FE4F8081DD
:10EC40009181A281B38184369105A105B10508F4B3
:10EC5000F1C064E0CC0FDD1F6A95E1F7C951D04FD8
:10EC600088809980AA80BB8081149104A104B1049A
:10EC700009F4E0C0C501B40140E04ADF882309F48B
:10EC8000D9C080912C0E90912D0E8050924009F0A9
:10EC9000D1C02091310E222309F4CCC080912F0ED7
:10ECA0009091300E892B09F4C5C080912E0E8823D7
:10ECB00009F4C0C0F601228B80912E0E8483158644
:10ECC00061E070E007C04F5FF60145874150483072
:10ECD00008F0B0C0F6014585848190E09B01042EC8
:10ECE00002C0220F331F0A94E2F78217930759F7E5
:10ECF0002091370E3091380E2115310519F040E082
:10ED000050E008C02091450E3091460E4091470ECC
:10ED10005091480EF6012583368347835087E09053
:10ED20002F0EF090300E00E010E0E80CF91C0A1DE8
:10ED30001B1DE38AF48A058B168B8091320E90910D
:10ED4000330E918F808F6091310E70E080E090E003
:10ED50000E94A3D26E0D7F1D801F911FF601628F4E
:10ED6000738F848F958F2091320E3091330E55E042
:10ED7000220F331F5A95E1F721503E4F232F33279F
:10ED8000269540E050E0260F371F481F591F268761
:10ED90003787408B518B8091340E9091350E0097C0
:10EDA00019F0A0E0B0E008C08091410E9091420EB1
:10EDB000A091430EB091440E85017401E21AF30A4A
:10EDC000040B150BA8019701280F391F4A1F5B1F61
:10EDD000F601058404C056954795379527950A9402
:10EDE000D2F72187328743875487253FFFE03F07CB
:10EDF000F0E04F07F0E05F0720F48CE0F601878B2E
:10EE000019C0255F3F4F4040504018F480E1F601A3
:10EE10000EC080914D0E90914E0EA0914F0EB0916C
:10EE2000500EF601828F938FA48FB58F80E2878B6F
:10EE300081E001C080E0DF91CF911F910F91FF90A1
:10EE4000EF90DF90CF90BF90AF909F908F900895FC
:10EE50006F927F928F929F92AF92BF92CF92DF92EA
:10EE6000EF92FF920F931F93CF93DF93EC015A0120
:10EE70006B0138014901423051056105710508F403
:10EE80005DC089859A85AB85BC850196A11DB11DA4
:10EE900084179507A607B70708F450C08F898031FB
:10EEA00029F4E52EF62E072F11270CC0803209F029
:10EEB00045C07A018B0187E016950795F794E79492
:10EEC0008A95D1F78B899C89AD89BE89E80EF91E98
:10EED0000A1F1B1FC801B70141E01ADE882371F128
:10EEE0008F89803149F4F501F070EE0FFF1FEF5D5F
:10EEF000F14F718260820DC0F501EF77F070EE0F77
:10EF0000FF1FEE0FFF1FEF5DF14F60827182828263
:10EF100093828A89823080F08D819E81AF81B8850D
:10EF2000E80EF91E0A1F1B1FE0922410F092251014
:10EF3000009326101093271081E001C080E0DF913C
:10EF4000CF911F910F91FF90EF90DF90CF90BF90E6
:10EF5000AF909F908F907F906F900895CF92DF92A7
:10EF6000EF92FF920F931F93CF93DF93EC017A01FF
:10EF70008B01690189859A85AB85BC850196A11DA8
:10EF8000B11D84179507A607B70708F452C08F89EB
:10EF9000803129F45527412F302F2F2D0CC080327E
:10EFA00009F047C09A01AB0167E056954795379540
:10EFB00027956A95D1F78B899C89AD89BE89280FE1
:10EFC000391F4A1F5B1F80911D0E90911E0EA0914C
:10EFD0001F0EB091200E281739074A075B0731F042
:10EFE000CA01B90140E094DD882319F18F8980318D
:10EFF00059F4F701F070EE0FFF1FEF5DF14F8081C4
:10F000009181A0E0B0E00EC0F701EF77F070EE0F55
:10F01000FF1FEE0FFF1FEF5DF14F80819181A281F5
:10F02000B381BF70F60180839183A283B38381E0B3
:10F0300001C080E0DF91CF911F910F91FF90EF9081
:10F04000DF90CF900895AF92BF92CF92DF92EF9270
:10F05000FF920F931F93DF93CF9300D00F92CDB702
:10F06000DEB76C017A018B0182E090E0A0E0B0E0B5
:10F07000F60180839183A283B3835E010894A11C6F
:10F08000B11CC601B801A701950168DF882339F1D9
:10F09000C601B801A70100E010E020E030E0D8DEB2
:10F0A0008823E9F0E980FA800B811C81F6018789C9
:10F0B000803151F4F8EFEF16FFEFFF06F0E00F0795
:10F0C000F0E01F07F0F209C088EFE8168FEFF806AE
:10F0D0008FEF08078FE01807A0F281E001C080E001
:10F0E0000F900F900F900F90CF91DF911F910F9184
:10F0F000FF90EF90DF90CF90BF90AF9008954F9228
:10F100005F926F927F928F929F92AF92BF92CF92B7
:10F11000DF92EF92FF920F931F93DF93CF9300D074
:10F120000F92CDB7DEB76C0149835A836B837C8322
:10F130003901EE24FF2487012E010894411C511C43
:10F14000812CE2E09E2EA12CB12C49815A816B8149
:10F150007C81C601920102DF882339F1D501C40107
:10F16000F601058404C0880F991FAA1FBB1F0A94CB
:10F17000D2F7E80EF91E0A1F1B1F29813A814B8125
:10F180005C818789803131F4285F3F4F4040504097
:10F19000E0F205C0285F3F4F4F4F5F40B0F2F301F0
:10F1A000E082F1820283138381E00F900F900F9031
:10F1B0000F90CF91DF911F910F91FF90EF90DF9013
:10F1C000CF90BF90AF909F908F907F906F905F9007
:10F1D0004F9008952F923F924F925F926F927F923D
:10F1E0008F929F92AF92BF92CF92DF92EF92FF9257
:10F1F0000F931F93DF93CF93CDB7DEB72F970FB643
:10F20000F894DEBF0FBECDBF1C014A875B876C87B9
:10F210007D873F872E87DC0119968D919D910D90FA
:10F22000BC91A02D0196A11DB11D8E839F83A8873F
:10F23000B987F901008111812281338101151105FE
:10F240002105310549F0480159010894811C911CA0
:10F25000A11CB11C1D8210C0D1018D909D90AD905C
:10F26000BC901D828A859B85AC85BD850197A105D3
:10F27000B10511F491E09D83750164014424552486
:10F2800032018E010F5F1F4FF10181859285A385A9
:10F29000B485481659066A067B0608F08CC08E8134
:10F2A0009F81A885B9858C159D05AE05BF0550F4D5
:10F2B000A2E08A2E912CA12CB12CF2E0CF2ED12CE1
:10F2C000E12CF12CC101B701A601980147DE88238A
:10F2D00009F471C089819A81AB81BC81A701960133
:10F2E0002F5F3F4F4F4F5F4F0097A105B10519F0BA
:10F2F00049015A010DC0281939094A095B098A8553
:10F300009B85AC85BD85281739074A075B0759F0EF
:10F310000894411C511C611C711C0894C11CD11C17
:10F32000E11CF11CB1CFC101A601B7010FEF1FEF26
:10F330002FEF3FE08DDD882391F43DC0260137019A
:10F3400008944108510861087108C101B301A20184
:10F35000970186017DDD882371F1730162018C14B0
:10F360009D04AE04BF0450F3AE85BF854D915D9101
:10F370006D917C91411551056105710531F0C10117
:10F380009501840165DD8823B1F0EE85FF858082DB
:10F390009182A282B382FD81FF2359F00894811CDF
:10F3A000911CA11CB11CD1018D929D92AD92BC9279
:10F3B000139781E001C080E02F960FB6F894DEBF6E
:10F3C0000FBECDBFCF91DF911F910F91FF90EF90B6
:10F3D000DF90CF90BF90AF909F908F907F906F9075
:10F3E0005F904F903F902F90089510925C10109274
:10F3F0005E10109260100895809383030895EFE6E5
:10F40000F0E080818260808308951F93FC011FB724
:10F41000F89480819181A281B3818093361090937A
:10F420003710A0933810B0933910FB01808191817F
:10F43000A281B38180933A1090933B10A0933C102B
:10F44000B0933D10FA0180819181A281B3818093B4
:10F450003E1090933F10A0934010B0934110F901DB
:10F4600080819181A281B381809342109093431057
:10F47000A0934410B09345101FBF1F910895FC0145
:10F480002FB7F89480819181A281B381809342103B
:10F4900090934310A0934410B09345102FBF08954C
:10F4A000E82F8FB7F894F0E0EE0FFF1FEE0FFF1F6D
:10F4B000EA5CFF4E20813181428153818FBFB901C7
:10F4C000CA01089580916F008D7F80936F0006C000
:10F4D0008091060E8F5F8F708093060E9091050EBF
:10F4E0008091060E981751F410922910109228104E
:10F4F00080916F00826080936F0008959091050E57
:10F500008091060E981751F3E3CF9B01882399F45D
:10F51000B901882777FD8095982F2FEF30E040E0E4
:10F5200050E00E94A3D220ED37E040E050E00E947E
:10F5300017D38CE214C08130A9F4B901882777FD74
:10F540008095982F2FEF30E040E050E00E94A3D24A
:10F5500020ED37E040E050E00E9417D38DE2B90182
:10F560000C944E1A8230A9F4B901882777FD809552
:10F57000982F2FEF30E040E050E00E94A3D220ED22
:10F5800037E040E050E00E9417D38EE2B9010C94BE
:10F590004E1A08958CE261E00E942C1B8DE261E01E
:10F5A0000E942C1B8EE261E00E942C1B609179036B
:10F5B00070917A0380E0A9DF60917B0370917C03F6
:10F5C00081E0A3DF60917D0370917E0382E09DDF87
:10F5D000E1E2F1E08081887F816080830895DADF55
:10F5E000099A3C9A399AEAE0F1E08081806480834C
:10F5F0008081846080830D9A159A3E9A469A3B9A40
:10F60000439A389A409A8081826080839FB7F894A9
:10F61000EBE0F1E08081826080839FBF0898109AC0
:10F620000C98149A0F98179A0B9A1398159A3D9A5A
:10F630004598469A3A9A4298439AEAE0F1E08081E6
:10F64000806880839FB7F894EBE0F1E080818F774A
:10F6500080839FBF409AEAE0F1E0808181608083EF
:10F660009FB7F894EBE0F1E080818E7F80839FBFAD
:10F67000A1E8B0E08C918F7E8C938C9188608C9304
:10F68000E0E8F0E080818D7F808380818E7F8083C1
:10F6900080818F73808380818F7C80838C91887F31
:10F6A00082608C9380E090E490938900809388003E
:10F6B0001092850010928400EFE6F0E08081826075
:10F6C000808381E080938303789408959091050E60
:10F6D0008091060E981739F00E9482870E945A3056
:10F6E0000E94D090F3CF0895F1DF159A469A439A7D
:10F6F000409A08951F920F920FB60F920BB60F9279
:10F700001124AF92BF92CF92DF92EF92FF920F93AC
:10F710001F932F933F934F935F936F937F938F9399
:10F720009F93AF93BF93CF93DF93EF93FF9380911A
:10F73000281090912910892B09F094C19091050E01
:10F740008091060E981719F4E0E0F0E014C0809163
:10F75000060E90E02DE430E0829FF001839FF00DD3
:10F76000929FF00D1124EB5CF64FE45BFF4F81E0BC
:10F770008083EC54F040F0932910E09328103097E8
:10F7800009F46AC1E45BFF4F81E08083EC54F040F0
:10F79000109268101092691010926A1010926B10FB
:10F7A00060AD71AD2CE96134720718F060E47CE95A
:10F7B00004C03EE46132730730F076956795769524
:10F7C000679584E007C047E26131740730F07695B1
:10F7D000679582E08093611007C08093611060326A
:10F7E000710510F460E270E06052704058E06030E3
:10F7F0007507E8F0472F50E0440F551F440F551F81
:10F800004B50534F9A012E5F3F4FF90185919491D0
:10F810009C01AA27639FC001629F810D9A1F0694D5
:10F820008A1F9A1F1124FA01459154911EC0CB01E1
:10F83000969587958C7F8B509F4EFC0145915491F6
:10F84000FC01329625913491862F90E0877090705C
:10F85000FC012E9FC0012F9F900D3E9F900D112403
:10F86000B3E096958795BA95E1F7481B590B443656
:10F870005105A8F4E0EEF2E007C08091C00085FFDA
:10F88000FCCF31969093C60090819923B1F784EC18
:10F8900098E04AE050E00E94EA5244E650E050937B
:10F8A0006D1040936C108091611080936E101092D7
:10F8B0006F10E0912810F091291064AD75AD709330
:10F8C000671060936610FCE961347F0718F060E40C
:10F8D0007CE904C02EE46132720730F076956795BA
:10F8E0007695679584E007C037E26131730730F0A1
:10F8F0007695679582E08093611008C081E08093DF
:10F9000061106032710510F460E270E06052704086
:10F9100048E060307407E8F0472F50E0440F551F6F
:10F92000440F551F4B50534F9A012E5F3F4FF90123
:10F93000859194919C01AA27639FC001629F810DCC
:10F940009A1F06948A1F9A1F1124FA014591549117
:10F950001EC0CB01969587958C7F8B509F4EFC01E6
:10F9600045915491FC01329625913491862F90E077
:10F9700087709070FC012E9FC0012F9F900D3E9FBD
:10F98000900D112433E0969587953A95E1F7481B41
:10F99000590B44365105A8F4E0EEF2E007C080911F
:10F9A000C00085FFFCCF31969093C60090819923CB
:10F9B000B1F784EC98E04AE050E00E94EA5244E655
:10F9C00050E0CA01A0E0B0E0809362109093631011
:10F9D000A0936410B0936510509389004093880001
:10F9E000E0912810F091291080899189A289B3892A
:10F9F000B695A79597958795B095A0959095819583
:10FA00009F4FAF4FBF4F8093461090934710A093E6
:10FA10004810B093491080934A1090934B10A093D4
:10FA20004C10B0934D1080934E1090934F10A093B4
:10FA30005010B09351108093521090935310A09394
:10FA40005410B093551010925610109257101092F7
:10FA500058101092591006C080ED97E090938900DD
:10FA600080938800C0912810D0912910209709F424
:10FA700089C488A180935A1080FF03C0119A8FEF28
:10FA800002C0119881E080937F0380915A1081FF1A
:10FA900003C044988FEF02C0449A81E080938003B2
:10FAA00080915A1080FF36C080918303882391F1A2
:10FAB00020B1217031E0232759F180915B10882318
:10FAC00039F188819981AA81BB81181619061A0615
:10FAD0001B06F4F48091361090913710A0913810E5
:10FAE000B091391080932A1090932B10A0932C1072
:10FAF000B0932D1030935C1088899989AA89BB89AD
:10FB00008093561090935710A0935810B0935910AB
:10FB100020935B1080915A1081FD3AC0809183033D
:10FB20008823B1F180B182958F708095282F217044
:10FB300080FF2CC080915D10882341F18C819D81D4
:10FB4000AE81BF81181619061A061B06FCF48091B7
:10FB50003A1090913B10A0913C10B0913D108093D1
:10FB60002E1090932F10A0933010B093311081E09D
:10FB700080935E1088899989AA89BB8980935610E1
:10FB800090935710A0935810B093591020935D1084
:10FB900080915A1082FF05C0419A8FEF80938103B4
:10FBA00039C0419881E08093810380918303882349
:10FBB00089F120E007992CC021E080915F10882313
:10FBC00039F188859985AA85BB85181619061A0604
:10FBD0001B06F4F480913E1090913F10A0914010CC
:10FBE000B09141108093321090933310A093341051
:10FBF000B09335102093601088899989AA89BB89B0
:10FC00008093561090935710A0935810B0935910AA
:10FC100020935F1080915A1083FF0AC08FB7F89429
:10FC200090910B019F7B90930B018FBF8FEF09C0C9
:10FC30008FB7F89490910B01906490930B018FBF54
:10FC400081E08093820360E070E079C18091C00020
:10FC500087FF19C04091C600E091C008F091C1082B
:10FC600031969F012F77307031978091C208909123
:10FC7000C3082817390739F0E05CF74F4083309309
:10FC8000C1082093C008288139814A815B81809115
:10FC9000461090914710A0914810B0914910280F3C
:10FCA000391F4A1F5B1F2093461030934710409323
:10FCB00048105093491012161306140615066CF5D9
:10FCC000139A88899989AA89BB89281B390B4A0B01
:10FCD0005B0B20934610309347104093481050938D
:10FCE00049102091361030913710409138105091C2
:10FCF000391080917F03992787FD9095A92FB92FFF
:10FD0000820F931FA41FB51F809336109093371056
:10FD1000A0933810B093391013982C813D814E81F7
:10FD20005F8180914A1090914B10A0914C10B0913E
:10FD30004D10280F391F4A1F5B1F20934A10309324
:10FD40004B1040934C1050934D101216130614068E
:10FD500015066CF5459A88899989AA89BB89281B5B
:10FD6000390B4A0B5B0B20934A1030934B10409396
:10FD70004C1050934D1020913A1030913B1040910F
:10FD80003C1050913D1080918003992787FD9095FC
:10FD9000A92FB92F820F931FA41FB51F80933A106C
:10FDA00090933B10A0933C10B0933D10459828854C
:10FDB00039854A855B8580914E1090914F10A091B6
:10FDC0005010B0915110280F391F4A1F5B1F20930C
:10FDD0004E1030934F104093501050935110121604
:10FDE0001306140615066CF5429A88899989AA8922
:10FDF000BB89281B390B4A0B5B0B20934E103093A9
:10FE00004F10409350105093511020913E1030915C
:10FE10003F104091401050914110809181039927EB
:10FE200087FD9095A92FB92F820F931FA41FB51F8F
:10FE300080933E1090933F10A0934010B0934110D8
:10FE400042982C853D854E855F858091521090911A
:10FE50005310A0915410B0915510280F391F4A1F0C
:10FE60005B1F2093521030935310409354105093C3
:10FE700055101216130614061506DCF59FB7F894F4
:10FE800080910B01806880930B019FBF88899989BD
:10FE9000AA89BB89281B390B4A0B5B0B2093521094
:10FEA00030935310409354105093551020914210AA
:10FEB000309143104091441050914510809182033D
:10FEC000992787FD9095A92FB92F820F931FA41F03
:10FED000B51F8093421090934310A0934410B093A9
:10FEE00045109FB7F89480910B018F7780930B0199
:10FEF0009FBF8091561090915710A0915810B091CB
:10FF000059100196A11DB11D809356109093571062
:10FF1000A0935810B093591020915610309157105B
:10FF200040915810509159106F5F7F4F888999897F
:10FF3000AA89BB89281739074A075B0738F48091DB
:10FF4000611090E0681779070CF480CE209156106C
:10FF50003091571040915810509159108C899D89BB
:10FF6000AE89BF8982179307A407B50708F4E3C0D9
:10FF7000E0906210F0906310009164101091651091
:10FF8000AC8CBD8CCE8CDF8CA8019701C601B5016D
:10FF9000AA27279FB12D389FF001489FF00D479F5A
:10FFA000E00DF11D289FB00DE11DFA1F379FB00D28
:10FFB000E11DFA1F469FB00DE11DFA1F369FB10DDE
:10FFC000EA1FFA1FB695EA1FFA1F11248CAD9DADEA
:10FFD0008E0F9F1F909367108093661028AD39ADE8
:10FFE0004AAD5BADA0E0B0E0281739074A075B07D0
:10FFF00020F4309367102093661060916610709122
:020000021000EC
:1000000067108CE96134780718F060E47CE904C07B
:100010009EE46132790730F076956795769567951D
:1000200084E007C0E7E261317E0730F0769567959E
:1000300082E08093611008C081E08093611060329B
:10004000710510F460E270E060527040F8E06030DA
:100050007F07E8F0472F50E0440F551F440F551F0E
:100060004B50534F9A012E5F3F4FF9018591949168
:100070009C01AA27639FC001629F810D9A1F06946D
:100080008A1F9A1F1124FA01459154911EC0CB0179
:10009000969587958C7F8B509F4EFC01459154918E
:1000A000FC01329625913491862F90E087709070F4
:1000B000FC012E9FC0012F9F900D3E9F900D11249B
:1000C000B3E096958795BA95E1F7481B590B4436EE
:1000D0005105A8F4E0EEF2E007C08091C00085FF72
:1000E000FCCF31969093C60090819923B1F784ECB0
:1000F00098E04AE050E00E94EA5244E650E0509313
:100100008900409388009A0140E050E0809162109D
:1001100090916310A0916410B0916510820F931FAD
:10012000A41FB51F8093621090936310A093641076
:10013000B093651002C12091561030915710409134
:10014000581050915910888D998DAA8DBB8D8217AA
:100150009307A407B50708F0E4C060916810709198
:10016000691080916A1090916B102C8D3D8D4E8D91
:100170005F8DAA27639FB12D749FF001849FF00DBE
:10018000839FE00DF11D649FB00DE11DFA1F739F69
:10019000B00DE11DFA1F829FB00DE11DFA1F729F85
:1001A000B10DEA1FFA1FB695EA1FFA1F11248091BC
:1001B0006610909167108E179F0738F4C05CDF4F70
:1001C00068817981C054D04003C0BC016E1B7F0B95
:1001D000C05CDF4F288139814A815B81CB01A0E07F
:1001E000B0E082179307A407B50708F4B901FCE94A
:1001F00061347F0718F060E47CE904C02EE46132CA
:10020000720730F0769567957695679584E007C01C
:1002100037E26131730730F07695679582E080931D
:10022000611008C081E0809361106032710510F4A4
:1002300060E270E06052704048E060307407E8F0BF
:10024000472F50E0440F551F440F551F4B50534F3D
:100250009A012E5F3F4FF901859194919C01AA2745
:10026000639FC001629F810D9A1F06948A1F9A1F87
:100270001124FA01459154911EC0CB0196958795A2
:100280008C7F8B509F4EFC0145915491FC0132961E
:1002900025913491862F90E087709070FC012E9FFD
:1002A000C0012F9F900D3E9F900D112423E0969545
:1002B00087952A95E1F7481B590B44365105A8F458
:1002C000E0EEF2E007C08091C00085FFFCCF3196E0
:1002D0009093C60090819923B1F784EC98E04AE0AE
:1002E00050E00E94EA5244E650E050938900409367
:1002F00088009A0140E050E0809168109091691068
:10030000A0916A10B0916B10820F931FA41FB51FAC
:100310008093681090936910A0936A10B0936B104B
:100320000CC080916C1090916D1090938900809317
:10033000880080916E10809361102091561030914A
:1003400057104091581050915910E0912810F09199
:10035000291080899189A289B389281739074A070A
:100360005B0780F010922910109228109091050ED2
:100370008091060E981731F08091060E8F5F8F7076
:100380008093060EFF91EF91DF91CF91BF91AF91D6
:100390009F918F917F916F915F914F913F912F919D
:1003A0001F910F91FF90EF90DF90CF90BF90AF9093
:1003B0000F900BBE0F900FBE0F901F90189580915D
:1003C0005C10882349F480915E10882329F4809181
:1003D0006010882309F490C0E5EFF4E1949108C01F
:1003E0008091C00085FFFCCF9093C6003196949118
:1003F0009923B1F7E7E0F5E1949108C08091C0003E
:1004000085FFFCCF9093C600319694919923B1F764
:1004100080915C108823D1F060912A1070912B108C
:1004200080912C1090912D100E94CDCC2091D90854
:100430003091DA084091DB085091DC080E9432CC00
:10044000AB01BC0183E095E10E94C23380915E1054
:100450008823D1F060912E1070912F108091301070
:10046000909131100E94CDCC2091DD083091DE08B2
:100470004091DF085091E0080E9432CCAB01BC01F2
:100480008FEF94E10E94C233809160108823D1F0F5
:10049000609132107091331080913410909135102A
:1004A0000E94CDCC2091E1083091E2084091E30810
:1004B0005091E4080E9432CCAB01BC018BEF94E177
:1004C0000E94C233E4EFF2E007C08091C00085FFD4
:1004D000FCCF31969093C60090819923B1F780911B
:1004E000C00085FFFCCF8AE08093C60010925C10AC
:1004F00010925E1010926010089560E070E08FE737
:1005000093E4209188033091890340918A035091AC
:100510008B030E9432CC60939C1070939D1080934B
:100520009E1090939F1060E070E08FE793E420911D
:1005300098033091990340919A0350919B030E9434
:1005400032CC6093A4107093A5108093A610909362
:10055000A7100895FC0197FF03C08091811003C08C
:10056000E058FF4E808190E008952F923F924F9285
:100570005F926F927F928F929F92AF92BF92CF9233
:10058000DF92EF92FF920F931F93CF93DF93EC01D3
:1005900021E030E0A901440F551F440F551FFA0117
:1005A000E253FA4E85919491C817D9070CF059C0BF
:1005B000B90161507040660F771F660F771FCB013E
:1005C00080539A4EFC010591149162537A4EFB01BF
:1005D000C590D490FA01E053FA4EE590F490FA01F8
:1005E000E253FA4EA590B490B801882777FD809524
:1005F000982F0E94CDCC1B012C01CC19DD09BE0126
:10060000882777FD8095982F0E94CDCC3B014C0127
:10061000E01AF10A0027F7FC0095102FC801B70176
:100620000E94CDCC9B01AC01C401B3010E9400CF5C
:100630007B018C01AC18BD08CC24B7FCC094DC2C29
:10064000C601B5010E94CDCC9B01AC01C801B70128
:100650000E9432CC9B01AC01C201B1010E9452CB7D
:1006600019C0822F8F5F2F5F3F4F2133310509F073
:1006700091CF813329F0E0E070E080E060E00CC0D1
:10068000E0E9F6E165917491882777FD8095982FD0
:100690000E94CDCCE62F692F2E2F372F482F562FB3
:1006A000B901CA01DF91CF911F910F91FF90EF9097
:1006B000DF90CF90BF90AF909F908F907F906F9082
:1006C0005F904F903F902F90089508951092711071
:1006D00010927010109280107498109273101092F3
:1006E000721010928110A59808952DEB37E346E023
:1006F0005EE30C9400CF2DEB37E346E05EE30C9411
:1007000032CC2DEB37E346E05EE30C9432CC2DEB9C
:1007100037E346E05EE30C9400CFA5980E94862F55
:10072000882319F5E6E1F5E1949108C08091C000B5
:1007300085FFFCCF9093C600319694919923B1F731
:10074000EDE1F5E1949108C08091C00085FFFCCFF8
:100750009093C600319694919923B1F78091C0008F
:1007600085FFFCCF8AE08093C60083E00C94C22F03
:100770001F93182FABDF0E94862F882391F5E6E1A7
:10078000F5E1949108C08091C00085FFFCCF909363
:10079000C600319694919923B1F784EC98E0612FCB
:1007A00070E04AE050E00E94C3528091C00085FF93
:1007B000FCCF8AE08093C600E7E5F5E1949108C09C
:1007C0008091C00085FFFCCF9093C6003196949134
:1007D0009923B1F78091C00085FFFCCF8AE0809318
:1007E000C60082E00E94C22F1F9108951F93182F08
:1007F0006DDF0E94862F882391F5E6E1F5E1949163
:1008000008C08091C00085FFFCCF9093C600319650
:1008100094919923B1F784EC98E0612F70E04AE05D
:1008200050E00E94C3528091C00085FFFCCF8AE057
:100830008093C600E4E8F5E1949108C08091C0007F
:1008400085FFFCCF9093C600319694919923B1F720
:100850008091C00085FFFCCF8AE08093C60081E0D4
:100860000E94C22F1F9108951F920F920FB60F92F0
:100870000BB60F9211242F933F934F935F936F9377
:100880007F938F939F93AF93BF93EF93FF93909139
:10089000A403992361F480918010809386108111C4
:1008A000749A80918110809385108111A59A80910E
:1008B0008610981708F0749880918510981708F0A2
:1008C000A5989F5F9F779093A4038091A5038430A0
:1008D00009F471C0853050F4813021F1813098F0F5
:1008E0008230F1F1833009F07AC049C0863009F4D2
:1008F00068C0863008F463C0873009F466C0883069
:1009000009F06DC06AC088E080937B0080E480932A
:100910007C0080917A00806480937A000E94938E9C
:1009200081E01BC08091780090917900A0E0B0E058
:100930002091931030919410409195105091961001
:10094000280F391F4A1F5B1F209393103093941078
:10095000409395105093961082E08093A5033FC07A
:1009600088E080937B0082E480937C0080917A0011
:10097000806480937A000E94938E83E0EECF809112
:10098000780090917900A0E0B0E02091871030913C
:1009900088104091891050918A10280F391F4A1FE2
:1009A0005B1F2093871030938810409389105093D9
:1009B0008A1084E0D2CF0E94938E85E0CECF86E06D
:1009C000CCCF0E94938E87E0C8CF1092A503809170
:1009D00097108F5F8093971002C01092A5038091AB
:1009E0009710803108F463C080918210882381F4CD
:1009F000809193109091941090937510809374103F
:100A0000809187109091881090937B1080937A103A
:100A100081E08093821010929710109293101092A0
:100A20009410109295101092961010928F101092B0
:100A30009010109291101092921010928B101092B0
:100A40008C1010928D1010928E10109287101092B0
:100A500088101092891010928A1020917410309191
:100A600075108091A0039091A1032817390714F005
:100A700080E0BCDE2091741030917510809183105D
:100A8000909184108217930714F080E071DE20911A
:100A90007A1030917B108091A2039091A3032817C4
:100AA00039072CF0109273101092721036DEFF91FD
:100AB000EF91BF91AF919F918F917F916F915F91D6
:100AC0004F913F912F910F900BBE0F900FBE0F9043
:100AD0001F9018952F926F927F928F929F92AF9254
:100AE000BF92CF92DF92EF92FF920F931F93DF930B
:100AF000CF93CDB7DEB729970FB6F894DEBF0FBE00
:100B0000CDBF8C01E62E662369F1E6E1F5E1949113
:100B100008C08091C00085FFFCCF9093C60031963D
:100B200094919923B1F784EC98E06E2D70E04AE03F
:100B300050E00E94C352E1EBF5E1949108C080912E
:100B4000C00085FFFCCF9093C60031969491992305
:100B5000B1F78091C00085FFFCCF8AE08093C6008A
:100B60000E940230AE2DB0E0FD01EE0FFF1FE85DE8
:100B7000FB4F6081718179876887672B09F49FC07B
:100B8000A65DBB4F7C917B832224239479C0222DC8
:100B900030E0A901440F551F440F551FE885F98522
:100BA000E40FF51F85919491081719070CF067C0A1
:100BB000C9010197880F991F880F991FFC01329670
:100BC000A885B985EA0FFB1FC590D4908A0F9B1F9B
:100BD000FC01659174917A836983FA013296EA0F78
:100BE000FB1FE590F490FD01E40FF51FA590B49074
:100BF000B601882777FD8095982F0E94CDCC6C8315
:100C00007D838E839F8389819A81081B190BB8018C
:100C1000882777FD8095982F0E94CDCC3B014C0111
:100C2000EC18FD080027F7FC0095102FC801B7014C
:100C30000E94CDCC9B01AC01C401B3010E9400CF46
:100C40007B018C01A981BA81AA1ABB0ACC24B7FC0A
:100C5000C094DC2CC601B5010E94CDCC9B01AC0137
:100C6000C801B7010E9432CC9B01AC016C817D812F
:100C70008E819F810E9452CBE62F692F09C0239459
:100C8000BB812B1608F483CFE0E070E080E060E0E9
:100C9000FB812F1679F5E22DF0E0EE0FFF1FEE0F2E
:100CA000FF1F329768857985E60FF71F659174916C
:100CB000882777FD8095982F0E94CDCC19C0B80168
:100CC000882777FD8095982F0E94CDCC20E030E0DA
:100CD0004AEF5EE30E9400CF20E030E040E85DE3B1
:100CE0000E9400CF20E030E040E050E00E9452CB74
:100CF000E62F692F2E2F372F482F562FB901CA0103
:100D000029960FB6F894DEBF0FBECDBFCF91DF910D
:100D10001F910F91FF90EF90DF90CF90BF90AF9019
:100D20009F908F907F906F902F900895EF92FF92F9
:100D30000F931F93CF93DF930F2EF0E0EF2EF0E091
:100D4000FF2EF0E00F2FF0E01F2FF02DE092981013
:100D5000F092991000939A1010939B1060E070E04D
:100D60008FE793E4209188033091890340918A03AF
:100D700050918B030E9432CC60939C1070939D1015
:100D800080939E1090939F10E092A010F092A1107B
:100D90000093A2101093A31060E070E08FE793E43B
:100DA000209198033091990340919A0350919B03AD
:100DB0000E9432CC6093A4107093A5108093A6106B
:100DC0009093A7106C9A6D9A9D9A80910101806111
:100DD0008093010187ED80937A0010927E0010923B
:100DE0007D0080917D00816080937D0080917D00F9
:100DF000826080937D0080917D00846080937D007F
:100E000080E888BD80916E00846080936E0085E0EC
:100E100090E09093A9108093A81009C0809183104E
:100E200090918410409690938410809383108091C9
:100E300083109091841060E04DDE20E030E040EAC5
:100E400050E40E942BCC87FDE9CF83E191E09093A1
:100E5000A7038093A60309C08091A0039091A103EA
:100E600040979093A1038093A0038091A003909159
:100E7000A10360E02FDE20E030E849E853E40E945F
:100E80002ECE18164CF3C091A203D091A303EC2EE2
:100E90001D2FCE016ADB609720E030E048E453E488
:100EA0000E942ECE18169CF3E092A2031093A30387
:100EB000DF91CF911F910F91FF90EF900895809156
:100EC00074109091751060E005DE60937610709359
:100ED0007710809378109093791080917A10909188
:100EE0007B1043DB60937C1070937D1080937E10A9
:100EF00090937F100E9483C78FB7F894109282104E
:100F00008FBF08952F923F924F925F926F927F9280
:100F10008F929F92AF92BF92CF92DF92EF92FF9209
:100F20000F931F9380918210882309F46EC2C7DF4C
:100F30006090761070907710809078109090791073
:100F4000C0907010D0907110B601882777FD809501
:100F5000982F0E94CDCCA40193010E9451CB7B011C
:100F60008C016093AA107093AB108093AC10909397
:100F7000AD1020E030E04AE754E40E942ECE18166F
:100F800024F481E08093AE10E9C0C801B70120E0ED
:100F900030E04AE754EC0E942BCC87FD02C0CD28FC
:100FA00021F481E08093AE10C4C08091AE108823FC
:100FB00071F080E090E0A0E0B0E08093AF109093FB
:100FC000B010A093B110B093B2101092AE10C8013F
:100FD000B70120918403309185034091860350919D
:100FE00087030E9400CF1B012C016093B310709304
:100FF000B4108093B5109093B610C801B70120913A
:10100000AF103091B0104091B1105091B2100E94C9
:1010100052CB5B016C01E0909810F0909910009118
:101020009A1010919B10A80197010E942BCC87FD6C
:1010300012C0E0909C10F0909D1000919E101091B5
:101040009F10C601B501A80197010E942ECE181667
:1010500014F086017501E092AF10F092B010009389
:10106000B1101093B210C801B701209188033091DC
:10107000890340918A0350918B030E9400CF5B014A
:101080006C016093B7107093B8108093B91090936F
:10109000BA10C401B3012091BB103091BC10409133
:1010A000BD105091BE100E9451CB20918C03309105
:1010B0008D0340918E0350918F030E9400CF20E05A
:1010C00037ED43E25CE30E9400CF7B018C0160912D
:1010D000BF107091C0108091C1109091C21024EA8D
:1010E00030E74DE75FE30E9400CF9B01AC01C801F0
:1010F000B7010E9452CB7B018C016093BF107093AB
:10110000C0108093C1109093C210C201B101A6011A
:1011100095010E9452CBA80197010E9451CB7B01FF
:101120008C0120E030E040E050E00E942BCC88238E
:101130005CF40F2EF0E0EF2EF0E0FF2EF0E00F2F2A
:10114000F0E01F2FF02D14C0C801B70120E030E0FF
:101150004FE753E40E942ECE181654F40F2EF0E001
:10116000EF2EF0E0FF2EFFE70F2FF3E41F2FF02DFF
:101170006092BB107092BC108092BD109092BE1015
:101180006091A8107091A910882777FD8095982FFD
:101190000E94CDCC9B01AC01C401B3010E942ECEB4
:1011A0001816DCF46091A6037091A703882777FDD9
:1011B0008095982F0E94CDCC9B01AC01C401B30156
:1011C0000E942BCC88234CF4C801B7010E949ACC12
:1011D000759567956093801002C0109280106090A2
:1011E0007C1070907D1080907E1090907F106091A8
:1011F000721070917310882777FD8095982F0E9448
:10120000CDCCA40193010E9451CB7B018C01609352
:10121000C3107093C4108093C5109093C610209192
:1012200094033091950340919603509197030E9447
:1012300000CF1B012C016093C7107093C8108093DE
:10124000C9109093CA10C801B7012091CB103091FA
:10125000CC104091CD105091CE100E9452CB5B012A
:101260006C01E090A010F090A1100091A2101091DC
:10127000A310A80197010E942BCC87FD12C0E0901B
:10128000A410F090A5100091A6101091A710C6010F
:10129000B501A80197010E942ECE181614F0860100
:1012A0007501E092CB10F092CC100093CD1010930A
:1012B000CE10C801B7012091980330919903409155
:1012C0009A0350919B030E9400CF5B016C016093D5
:1012D000CF107093D0108093D1109093D210C4018E
:1012E000B3012091D3103091D4104091D51050917A
:1012F000D6100E9451CB20919C0330919D034091C8
:101300009E0350919F030E9400CF20E037ED43E2FF
:101310005CE30E9400CF7B018C016091D71070913B
:10132000D8108091D9109091DA1024EA30E74DE777
:101330005FE30E9400CF9B01AC01C801B7010E948E
:1013400052CB7B018C016093D7107093D81080939F
:10135000D9109093DA106092D3107092D4108092CA
:10136000D5109092D610C201B101A60195010E943C
:1013700052CBA80197010E9451CB7B018C0120E048
:1013800030E040E050E00E942BCC88235CF40F2E2C
:10139000F0E0EF2EF0E0FF2EF0E00F2FF0E01F2F37
:1013A000F02D14C0C801B70120E030E04FE753E44E
:1013B0000E942ECE181654F40F2EF0E0EF2EF0E01F
:1013C000FF2EFFE70F2FF3E41F2FF02DC401B30111
:1013D00020E030E040EA50E40E942ECE18169CF443
:1013E000C401B30120E030E048E453E40E942BCC78
:1013F00088234CF4C801B7010E949ACC7595679573
:101400006093811002C0109281101F910F91FF9084
:10141000EF90DF90CF90BF90AF909F908F907F9094
:101420006F905F904F903F902F9008952F923F9232
:101430004F925F926F927F928F929F92AF92BF92E4
:10144000CF92DF92EF92FF920F931F93DF93CF9390
:10145000CDB7DEB7E6970FB6F894DEBF0FBECDBFAF
:101460006C8F7D8F8E8F9F8F5EAB4DAB39A328A382
:101470000E94DE19698B7A8B8B8B9C8B2DA93EA9E0
:10148000223031051CF4E5EFF2E019C0E8E0F3E0AA
:1014900007C08091C00085FFFCCF31969093C600B5
:1014A00090819923B1F78091C00085FFFCCF12C4D1
:1014B0008091C00085FFFCCF31969093C60090814B
:1014C0009923B1F78091C00085FFFCCF8AE080931B
:1014D000C600FCD84DA95EA957FF74C08FE7809362
:1014E000811089899A89AB89BC898D879E87AF874E
:1014F000B88B89879A87AB87BC8719AA1AAA1BAAB7
:101500001CAA1F8A1E8A91E09D8B1D821E821F824B
:1015100018869FE7A92EB12CC12CD12C8FE7282E3D
:10152000312C412C512C20E030E040E050E0298368
:101530003A834B835C830F2EF0E06F2EF0E47F2E16
:10154000FCE18F2EF6E49F2EF02D4DA95EA94058A8
:101550005F4E5BA34AA3E3E7F7E154915CA3EEE699
:10156000F7E184918DA3E7E6F7E194919EA3E0E68D
:10157000F7E1A491AFA3EAE5F7E1B491B8A7E4E5F8
:10158000F7E1249129A7E7E4F7E134913AA7E1E4F0
:10159000F7E144914BA7EBE3F7E154915CA7E5E356
:1015A000F7E184918DA7ADA9BEA9AA0FBB1FAA0F11
:1015B000BB1FAA58BF4EBFA7AEA7EBEFF6E1B49191
:1015C000B8AB07C0EDA9FEA9E058FF4E8FE78083B6
:1015D00088CF80918210882309F4A2C270DCEDA923
:1015E000FEA9F7FF0DC0F0917C10F9AB20917D10A2
:1015F0002AAB30917E103BAB40917F104CAB11C0B9
:10160000AEA5BFA5BC91B9ABEEA5FFA5F181FAAB24
:10161000AEA5BFA51296BC91BBABEEA5FFA5F3810D
:10162000FCAB69817A818B819C8129A93AA94BA95C
:101630005CA90E942ECE181644F089A99AA9ABA9DC
:10164000BCA989839A83AB83BC83C401B30129A954
:101650003AA94BA95CA90E942BCC87FD06C089A999
:101660009AA9ABA9BCA93C014D012D89222309F4FB
:1016700051C069A97AA98BA99CA92C8D3D8D4E8D4D
:101680005F8D0E942ECE18160CF04AC20E94DE1901
:1016900029853A854B855C85621B730B840B950B02
:1016A000695873418040904008F43AC2D601C501A0
:1016B00082199309A409B5094DA95EA957FF07C06E
:1016C000B595A795979587958093811007C0B59597
:1016D000A79597958795EAA1FBA180830E94DE19C3
:1016E0006D877E878F87988B9B01AC0189859A8552
:1016F000AB85BC85281B390B4A0B5B0B2D833E83C6
:101700004F8358872C8D3D8D4E8D5F8D29833A8375
:101710004B835C8369A97AA98BA99CA92C8D3D8DEB
:101720004E8D5F8D0E942BCC88230CF0F8C10E9457
:10173000DE192D853E854F855889621B730B840BFE
:10174000950B695873418040904008F4E8C10E94AD
:10175000DE1969877A878B879C874E895F89452B3D
:1017600009F4B8C1DC01CB012D853E854F85588930
:10177000821B930BA40BB50B2D813E814F815885A5
:10178000280F391F4A1F5B1F288F398F4A8F5B8FA5
:101790002D813E814F815885281B390B4A0B5B0BED
:1017A000CA01B901A20191010E94A3D2288D398DED
:1017B0004A8D5B8D0E9417D32A0D3B1D4C1D5D1D6C
:1017C00024313105410551055CF4E4E12E2E312C24
:1017D000412C512C74E1A72EB12CC12CD12C1FC04F
:1017E00059016A013CEEA316B104C104D1042CF0E6
:1017F0006BEEA62EB12CC12CD12C40E8A416B1045E
:10180000C104D1041CF41501260109C05EEF252E88
:10181000312C412C512C2A183B084C085D089CA106
:10182000E3E7F7E108C08091C00085FFFCCF90930B
:10183000C600319694919923B1F784EC98E0B601F3
:10184000A5012AE030E00E9490529DA1EEE6F7E16A
:1018500008C08091C00085FFFCCF9093C6003196F0
:1018600094919923B1F784EC98E0B201A1012AE0A8
:1018700030E00E9490529EA1E7E6F7E108C0809117
:10188000C00085FFFCCF9093C600319694919923B8
:10189000B1F784EC98E0B401A30122E030E00E94AB
:1018A00096539FA1E0E6F7E108C08091C00085FF54
:1018B000FCCF9093C600319694919923B1F784ECB4
:1018C00098E049815A816B817C8122E030E00E945E
:1018D00096538091C00085FFFCCF8AE08093C600BC
:1018E0008E899F8903970CF4F5C0C201B1010E9453
:1018F000CDCC20E030E040E850E40E9400CF7B01F6
:101900008C0169817A818B819C81A40193010E9461
:1019100051CB20ED3FE049E450E40E9400CF20E0AD
:1019200030E040E05FE30E9400CF9B01AC01C801C2
:10193000B7010E9432CC7B018C01688D798D8A8D34
:101940009B8D0E94CDCC20E030E04AE754E40E9419
:1019500032CC3B014C0198A5EAE5F7E108C0809143
:10196000C00085FFFCCF9093C600319694919923D7
:10197000B1F784EC98E0B801A70122E030E00E94C2
:10198000965399A5E4E5F7E108C08091C00085FF72
:10199000FCCF9093C600319694919923B1F784ECD3
:1019A00098E0B401A30122E030E00E9496538091B8
:1019B000C00085FFFCCF8AE08093C600C801B70154
:1019C0002AE939E949E15FE30E9400CF7B018C01FC
:1019D0009AA5E7E4F7E108C08091C00085FFFCCF3D
:1019E0009093C600319694919923B1F78091C000ED
:1019F00085FFFCCF8AE08093C6009BA5E1E4F7E178
:101A000008C08091C00085FFFCCF9093C60031963E
:101A100094919923B1F784EC98E0B801A70122E0F2
:101A200030E00E9496538091C00085FFFCCF8AE091
:101A30008093C6009CA5EBE3F7E108C08091C0004D
:101A400085FFFCCF9093C600319694919923B1F70E
:101A5000C801B701A80197010E9452CBA4019301CC
:101A60000E9432CCAB01BC0184EC98E022E030E073
:101A70000E9496538091C00085FFFCCF8AE080933E
:101A8000C6009DA5E5E3F7E108C08091C00085FF91
:101A9000FCCF9093C600319694919923B1F7C80179
:101AA000B701A40193010E9400CF20E030E040E0A4
:101AB0005EE30E9400CFAB01BC0184EC98E022E021
:101AC00030E00E9496538091C00085FFFCCF8AE0F1
:101AD0008093C600D201C1018A0D9B1DAC1DBD1DA6
:101AE000EDA9FEA9F7FF07C0B595A795979587952E
:101AF0008093811007C0B595A79597958795EAA122
:101B0000FBA180832E893F892F5F3F4F3F8B2E8B18
:101B10006C8C7D8C8E8C9F8C31E03D8B01C01D8A3E
:101B20006C8D7D8D8E8D9F8D20E030E040EA51E4FC
:101B30000E9452CB9B01AC0169A97AA98BA99CA9EF
:101B40000E942ECE18169CF4EBE0F7E1949108C0A9
:101B50008091C00085FFFCCF9093C6003196949190
:101B60009923B1F78091C00085FFFCCFB3C00E94DC
:101B7000DE1929893A894B895C89621B730B840BB6
:101B8000950B615D77408040904008F454C04DA9AA
:101B90005EA957FF11C060918110E5E0F7E19491D3
:101BA00008C08091C00085FFFCCF9093C60031969D
:101BB00094919923B1F711C0AAA1BBA16C91EFEF49
:101BC000F6E1949108C08091C00085FFFCCF90930E
:101BD000C600319694919923B1F7162F84EC98E0C2
:101BE00049A95AA96BA97CA922E030E00E9496532A
:101BF00098A9EBEFF6E108C08091C00085FFFCCF0B
:101C00009093C600319694919923B1F784EC98E0B3
